:100000000C94441D0C94751D0C94751D0C94751D59
:100010000C94751D0C94751D0C94751D0C94751D18
:100020000C94751D0C94751D0C94751D0C94751D08
:100030000C94751D0C94751D0C94751D0C94751DF8
:100040000C94751D0C9442930C94751D0C94751DA5
:100050000C94751D0C94751D0C9457D50D947F143C
:100060000C94751D0C94DA5A0C94D05A0C94751D8E
:100070000C94751D0C94751D0C94751D0C94751DB8
:100080000C948B520C94751D0C94751D0C94751D5D
:100090000C94751D0C94751D0C94751D0C94751D98
:1000A0000C94751D0C94751D0C945D520C94751D6B
:1000B0000C94751D0C94751D0C94751D0C942F5289
:1000C0000C94751D0C94751D0C94751D0C947F5D1E
:1000D0000C94555D0C94751D0C94751D0C94751D38
:1000E0000C94751D241F6A1F701F971FA41FAD1F3E
:1000F000B81F7C279C287829AB2908350835C62AE3
:10010000692B782808350835062D9F2ED72E0835FF
:10011000D53008350835263208350835B032E33297
:1001200008355F331B34E62EEE2E122F362F6A2F42
:100130000D3021303A304730543068300D5B135B5E
:10014000255B355B3D5B6A5B415B6A5B455B495B9D
:100150006A5B4D5B515B555B5D5B6A5B675B129EE7
:10016000349E549E799E9E9E55A0C39EE69E099FF6
:100170002E9F539F789F9D9FC29F55A0E79F0CA0E5
:1001800031A0E3A1E6A1EAA1EDA1F0A11AA2F4A198
:10019000F7A1FBA1FEA101A205A208A20BA21AA22F
:1001A0000FA212A215A2FFE702E8F1E7F5E7FBE7CD
:1001B00039E806E80AE810E814E818E81EE822E83A
:1001C00026E839E82CE830E834E8F8EDFDED02EEF9
:1001D0000CEE16EE8FEE20EE28EE30EE3AEE44EE08
:1001E0004EEE5DEE67EE8FEE71EE7BEE85EE084A29
:1001F000D73B3BCE016E84BCBFFDC12F3D6C74313B
:100200009ABD56833DDA3D00C77F11BED9E4BB4C91
:100210003E916BAAAABE000000803F05A84CCDB25B
:10022000D44EB93836A9020C50B9918688083CA63C
:10023000AAAA2ABE000000803F000C9416EE0C947F
:1002400022E80C94A41F0C940D5B0C94D5300C94F4
:10025000C29F0C9478290D94281E0C94F8ED0C94F0
:1002600067EE0C940FA20C9430E80C94F0A10C945F
:10027000B81F0C94799E0C94FEA10C943AEE0C9449
:10028000241F0C9468300C941B340C94E69E0C9440
:10029000515B0C94E3320C94062D0C94F5E70C940E
:1002A000B45C0C9402EE0C94F7A10C940CEE0C943C
:1002B000AD1F0C94FFE70C94EAA10C9426320C9429
:1002C00006E80C9408350C94495B0C94692B0C944B
:1002D00026E80C940AE80C94122F0C940D5C0C94F4
:1002E00028EE0C94D05B0C9454300C94FE5B0C9470
:1002F0000CA00C94215C0C9410E80C94FDED0C9473
:1003000008A20C949E9E0C9415A20C940D300C9493
:1003100002E80C94E3A10C94135B0C94E79F0C94FB
:10032000455B0C94539F0C9439E80C94F1E70C94C2
:10033000F4A10C946A5B0C94789F0C9420EE0C94BE
:10034000FBE70C942CE80C946A2F0C9418E80C949E
:100350009C280C94AB290C9471EE0C9421300C94D5
:10036000675B0C940BA20C942F5C0C945F330C9481
:10037000355B0C942E9F0C944D5B0C946A1F0C946F
:100380008FEE0C949D9F0C94099F0C94B0320C94AA
:10039000549E0C9412A20C9455A00C944EEE0C9406
:1003A0009F2E0C94675C0C947C270C943A300C9430
:1003B00044EE0C94415B0C94C39E0C94555B0C94DE
:1003C000362F0C9414E80C94FBA10C94255B0C9430
:1003D000E62E0C9431A00C943D5B0C9401A20C947D
:1003E0001AA20C941EE80C9478280C94129E0C947B
:1003F00034E80C945D5B0C945DEE0C947BEE0C94F5
:10040000E6A10D94831D0C94EE2E0C94701F0C9499
:1004100047300C9485EE0C94D72E0C9430EE0C944F
:10042000349E0C94C62A0C94971F0C9405A20C942D
:10043000EDA14E414E494E495459494E46CDCCCC82
:100440003D0AD7233C17B7D13877CC2B329595E6A8
:10045000241FB14F0A000020410000C84200401C88
:100460004620BCBE4CCA1B0E5AAEC59D7400407AD5
:1004700010F35A00A0724E18090010A5D4E800002D
:10048000E87648170000E40B54020000CA9A3B00CB
:100490000000E1F505000080969800000040420F42
:1004A000000000A08601000000102700000000E806
:1004B00003000000006400000000000A00000000CB
:1004C000000100000000002C76D888DC674F08236C
:1004D000DFC1DFAE59E1B1B796E5E3E453C63AE6D2
:1004E00051997696E8E6C28426EB898C9B62ED40B2
:1004F0007C6FFCEFBC9C9F40F2BAA56FA5F4900501
:100500005A2AF75C936B6CF9676DC11BFCE0E40D34
:1005100047FEF520E6B500D0ED902E030094357728
:10052000050080841E080000204E0A000000C80C50
:10053000333333330F986E12831141EF8D211489B9
:100540003BE65516CFFEE6DB18D1844B381BF77C13
:100550001D901DA4BBE424203284725E228100C958
:10056000F124ECA1E53D274D323520500A4D3234BF
:10057000005072696E742050617573656400526535
:1005800073756D65005549205061757365004E6F38
:10059000204D61746368203A004D333033452D316E
:1005A000533635433455004D393939004D353032E5
:1005B0000A4D353030004D3330334530533231350C
:1005C000433855000A202A2A2A7265636461742E12
:1005D000646174615B305D203D004732380A473109
:1005E000204631303030205A313000556E737570EE
:1005F000706F72746564204F7074696F6E205365FC
:100600006C6563746564004D3139305335350A4784
:1006100032380A4732390A4D3430300A4D313034DD
:10062000533231350A4732380A4D3130395332317D
:10063000350A4D34323053310A4731583130305950
:1006400031303046353030300A47315A300A4D3576
:1006500030300A4D31313720536574205A204F66AF
:1006600066736574004731204631303030205A308F
:100670002E30004732380A473120463130303020A2
:100680005A302E30004D353030005A204F66667398
:100690006574203A202573004D353030005A204FC4
:1006A0006666736574203A202573004732385A0A0B
:1006B000473146313530305A302E30004732380A13
:1006C000473146313530305A302E30004D38340005
:1006D000473146313030305A302E30004732380AF8
:1006E000473146313030305A302E30005A204F6674
:1006F00066736574203A202573004D353030004D07
:10070000383400426567696E5377697463680072B4
:1007100065636461742E61646472203D3D0072659E
:10072000636461742E646174615B305D203D3D00E3
:1007300077616974776179203D3D000A202A2A2A71
:100740004E6F7A7A6C6554656D705374617475730D
:100750005B325D203D00434F4D4D554E4943415462
:10076000494F4E0044525952554E004552524F5235
:100770005300494E464F004543484F0047322F47EC
:10078000332062616420706172616D65746572739B
:100790000A00536C6565702E2E2E005A2050726F21
:1007A00062652050617374204265640A005A2050CB
:1007B000726F626520506173742042656400486FF7
:1007C0006D652058592046697273740A00486F6D30
:1007D00065205859204669727374004D31313720B5
:1007E00050726F6265206661696C65642E0A4732DB
:1007F000380A0070726F62655F72657769706500B4
:10080000473239205265747279696E670050726F91
:1008100062696E67204661696C6564004D313137ED
:1008200020426564206C6576656C696E6720666140
:10083000696C65642E0A4730205A31300A4D3330D6
:10084000302050323520533838300A4D3330302084
:100850005035302053300A4D33303020503235205F
:10086000533838300A4D3330302050353020533033
:100870000A4D3330302050323520533838300A4D4D
:10088000333030205035302053300A473420533134
:100890000070726F62655F6661696C6564004D31FE
:1008A000313720426564206C6576656C696E67201F
:1008B000646F6E652E00205A3A200020593A2000BD
:1008C00042656420583A20004D65736820706F6956
:1008D0006E742063616E6E6F742062652072657342
:1008E0006F6C7665640A004E6F204D6F76652E0042
:1008F000456E642066696C65206C6973740A0042F9
:100900006567696E2066696C65206C6973740A009E
:10091000526573756D6520534400286E6F206669BB
:100920006C65290043757272656E742066696C652A
:100930003A20002E0A0044656C6574696F6E20666B
:1009400061696C65642C2046696C653A20004669D3
:100950006C652064656C657465643A005072696EFC
:10096000742074696D653A20000A53746174733A97
:100970002046696C616D656E7420757365643A20FC
:10098000002C204C6F6E67657374206A6F623A208A
:1009900000546F74616C2074696D653A2000537463
:1009A0006174733A20002C204661696C65643A20BA
:1009B000002C2046696E69736865643A20005072A5
:1009C000696E74733A200053746174733A20004561
:1009D00020436F6F6C696E672E2E2E004520486590
:1009E0006174696E672E2E2E006F6666007707723F
:1009F000076B076407560744454255473A004D3197
:100A0000313320530042656420436F6F6C696E6719
:100A10002E2E2E004265642048656174696E672E33
:100A20002E2E006F6B004348414D4245525F5445A6
:100A30004D5045524154555245004D4F54494F4E2B
:100A40005F4D4F44455300544845524D414C5F5013
:100A5000524F54454354494F4E004155544F52450F
:100A6000504F52545F53445F5354415455530050B8
:100A7000524F4D50545F535550504F525400454DB6
:100A8000455247454E43595F5041525345520043EA
:100A90004153455F4C494748545F42524947485487
:100AA0004E45535300544F47474C455F4C494748C8
:100AB000545300534F4654574152455F504F57458A
:100AC00052004255494C445F50455243454E5400F4
:100AD0004C4556454C494E475F44415441005A5F8E
:100AE00050524F4245004155544F4C4556454C00DD
:100AF0005052494E545F4A4F420050524F47524560
:100B00005353004155544F5245504F52545F544532
:100B10004D5000564F4C554D4554524943004545A4
:100B200050524F4D0042494E4152595F46494C4543
:100B30005F5452414E534645520053455249414C31
:100B40005F584F4E5F584F4646004649524D5741F9
:100B500052455F4E414D453A4D61726C696E20328F
:100B60002E305F44573320544D3344204535505385
:100B70004D44424220534F555243455F434F4445F5
:100B80005F55524C3A68747470733A2F2F676974CA
:100B90006875622E636F6D2F496E73616E6974792B
:100BA0004175746F6D6174696F6E2F4D61726C6900
:100BB0006E2F747265652F437265616C6974795F1D
:100BC0004D61726C696E322E302E782050524F5427
:100BD0004F434F4C5F56455253494F4E3A312E309A
:100BE000204D414348494E455F545950453A544D74
:100BF000334420453520506C757320455854525568
:100C00004445525F434F554E543A3120555549445F
:100C10003A63656465326132662D343161322D3458
:100C20003734382D396231322D63353563363266CB
:100C300033363766660A002F2F200020466C6F7708
:100C40003A200050726F7465637465642050696E59
:100C50000A00206F7574206F662072616E67650AE6
:100C600000536572766F20003A200020536572763B
:100C70006F200050726F6265205A204F6666736560
:100C8000743A2000496E76616C69642065787472EC
:100C9000756465720A0020643A0020693A00207089
:100CA0003A0020643A0020693A0020703A006469F2
:100CB0007300656E0043290A0061626C6564202838
:100CC0006D696E2074656D702000436F6C642065E3
:100CD000787472756465732061726520004F4646B2
:100CE000004F4E0046696C616D656E742072756EC2
:100CF0006F75742064697374616E636520286D6D0F
:100D0000293A200046696C616D656E742072756EBB
:100D10006F757420004D65736820706F696E742064
:100D200063616E6E6F74206265207265736F6C769E
:100D300065640A004D34323120696E636F727265EA
:100D4000637420706172616D657465722075736182
:100D500067650A004F666673657473204170706C36
:100D6000696564004572723A20546F6F2066617243
:100D70002100546F6F206661722066726F6D207261
:100D800065666572656E636520706F696E740A00D2
:100D9000454550524F4D204F4B0A003F4B20766146
:100DA0006C7565206F7574206F662072616E676563
:100DB0002028302D3130292E0A00416476616E637F
:100DC00065204B3D004572726F72207772697469BD
:100DD0006E6720746F20454550524F4D210A0036F2
:100DE0003726033C3D380E2E303E121A1C1808449C
:100DF0000AFF430809070001627573793A207061A0
:100E00007573656420666F7220696E7075740A0070
:100E1000627573793A2070617573656420666F72CC
:100E200020757365720A00627573793A2070726F6B
:100E300063657373696E670A007061757365004D51
:100E4000363030200A204D313137200A00206669C3
:100E50006C616D656E745F72756E6F75742000667F
:100E6000696C616D656E745F72756E6F7574205418
:100E70000046696C616D656E7452756E6F75742095
:100E8000540053544F505045442E20005072696E08
:100E90007465722073746F7070656420647565206A
:100EA000746F206572726F72732E20466978207499
:100EB0006865206572726F7220616E64207573655B
:100EC000204D39393920746F2072657374617274E2
:100ED0002E202854656D7065726174757265206985
:100EE000732072657365742E2053657420697420B5
:100EF00061667465722072657374617274696E677D
:100F0000290A004E6F20436865636B73756D207707
:100F1000697468206C696E65206E756D6265722CEF
:100F2000204C617374204C696E653A20004E6F202E
:100F3000436865636B73756D2077697468206C69AD
:100F40006E65206E756D6265722C204C6173742025
:100F50004C696E653A2000636865636B73756D203C
:100F60006D69736D617463682C204C617374204CDF
:100F7000696E653A20004C696E65204E756D62653C
:100F800072206973206E6F74204C617374204C69F9
:100F90006E65204E756D6265722B312C204C61732D
:100FA00074204C696E653A20004D31313000776114
:100FB00069740A004D313137004D333100534420FC
:100FC00072656164206572726F720A00446F6E65AB
:100FD000207072696E74696E672066696C650A00BC
:100FE0004B494C4C206361757365642062792074B1
:100FF0006F6F206D75636820696E616374697665D3
:101000002074696D65202D2063757272656E742081
:10101000636F6D6D616E643A20002020506C616ECC
:101020006E657242756666657242797465733A20C0
:10103000002046726565204D656D6F72793A20001B
:10104000436F6D70696C65643A2053657020203879
:1010500020323031390A00207C20417574686F726B
:101060003A2054696E794D616368696E65733344E3
:101070000A00323031392D30372D333000204C61A9
:10108000737420557064617465643A2000322E30A8
:101090005F4457330A004D61726C696E0020536FD4
:1010A0006674776172652052657365740A00205713
:1010B00061746368646F672052657365740A002009
:1010C00042726F776E206F75742052657365740A73
:1010D000002045787465726E616C2052657365748A
:1010E0000A00506F77657255700A007374617274EC
:1010F0000A006175746F25632E67006572726F72E6
:101100002077726974696E6720746F2066696C65F8
:101110000A00446F6E6520736176696E67206669A8
:101120006C652E0A004D323900205A3A0020593A97
:101130000020583A00656E6473746F70732068699C
:10114000743A200047323858590043616E6E6F740C
:10115000206F70656E20737562646972200053445D
:101160002063617264206F6B0A006F70656E526F4E
:101170006F74206661696C65640A00766F6C756DCA
:10118000652E696E6974206661696C65640A005336
:101190004420696E6974206661696C0A004D3234BE
:1011A000004D32332025730057726974696E6720D1
:1011B000746F2066696C653A20002E0A006F7065B6
:1011C0006E206661696C65642C2046696C653A2006
:1011D000002E0A006F70656E206661696C65642C74
:1011E0002046696C653A200046696C652073656C21
:1011F00065637465640A002053697A653A20004685
:10120000696C65206F70656E65643A200066726572
:10121000736800646F696E67002066696C653A20C8
:10122000004E6F772000454E4420535542524F5593
:1012300054494E450A002220706F730022207061CD
:1012400072656E743A2200535542524F5554494EBE
:10125000452043414C4C207461726765743A22000A
:10126000747279696E6720746F2063616C6C20738F
:1012700075622D67636F64652066696C657320779E
:1012800069746820746F6F206D616E79206C65766B
:10129000656C732E204D4158206C6576656C206915
:1012A000733A310A005344207072696E74696E6734
:1012B000206279746520004E6F7420534420707250
:1012C000696E74696E670A00496E76616C696420A4
:1012D00065787472756465720A007C3C3E5E2B3DD5
:1012E0003F2F5B5D3B2C2A225C00220A00556E6B6F
:1012F0006E6F776E20636F6D6D616E643A202200B1
:1013000020746F6F206C6F6E6720657874727573D0
:10131000696F6E2070726576656E7465640A002070
:10132000636F6C6420657874727573696F6E20707A
:10133000726576656E7465640A004D3238302050EF
:1013400030205339300050726F62696E6720506FE1
:10135000696E742025692F2569002E0A002F005020
:10136000726F62696E67206D65736820706F696E59
:10137000742000202844525952554E2900473239D2
:10138000204175746F20426564204C6576656C69F8
:101390006E67003F20284C2C522C462C4229206F8F
:1013A0007574206F6620626F756E64732E0A003F3D
:1013B0002856296572626F7365206C6576656C20AE
:1013C000697320696D706C61757369626C65202842
:1013D000302D34292E0A00426164205A2076616C37
:1013E00075650A004E6F2062696C696E65617220D6
:1013F000677269640A0046696E6973686564210AE8
:1014000000206F662000205A00205900476F696E47
:101410006720746F3A20580043570A0020646972AD
:101420003A0020616E676C653A00537461727420F3
:101430007261646975733A00506F736974696F6E95
:10144000696E67207468652070726F62652E2E2E3B
:101450000A003F4E756D626572206F66206C65678D
:101460007320696E206D6F76656D656E74206E6F8A
:101470007420706C61757369626C652028302D3141
:1014800035292E0A003F2028582C5929206F7574C1
:10149000206F6620626F756E64732E0A003F536181
:1014A0006D706C652073697A65206E6F7420706C46
:1014B00061757369626C652028342D3530292E0AD8
:1014C000004D3438205A2D50726F6265205265707D
:1014D0006561746162696C69747920546573740A1A
:1014E000003F2856296572626F7365206C657665CA
:1014F0006C20697320696D706C61757369626C65CD
:101500002028302D34292E0A0053544F5020636177
:101510006C6C65642062656361757365206F66201D
:10152000424C546F756368206572726F72202D2073
:10153000726573746172742077697468204D3939EB
:10154000390A0053544F502063616C6C656420620B
:10155000656361757365206F6620424C546F7563D7
:1015600068206572726F72202D20726573746172CB
:10157000742077697468204D3939390A002F2F613A
:101580006374696F6E3A00627574746F6E00656E95
:10159000640070726F6D70745F0073686F77004DD8
:1015A00038373620526573706F6E64696E672050ED
:1015B000524F4D50545F00554E4B4E4F574E205397
:1015C000544154450047434F44455F494E464F0000
:1015D0004C43445F50415553455F524553554D452B
:1015E0000046494C414D454E545F52554E4F55545F
:1015F0005F434F4E54494E55450046494C414D4579
:101600004E545F52554E4F5554004D323400436F87
:101610006E74696E75650044697361626C655275BC
:101620006E6F7574005075726765204D6F7265003E
:101630005061757365640070617573656400486F0F
:1016400074656E6420746F6F20636F6C640A005061
:101650006175736500507265737320627574746F81
:101660006E20286F72204D3130382920746F20721F
:101670006573756D650A00496E73657274206669DD
:101680006C616D656E7420616E6420707265737339
:1016900020627574746F6E20286F72204D3130385F
:1016A000290A00436F6E74696E756500526568653E
:1016B000617420446F6E6500526568656174696E7F
:1016C000672E2E2E00526568656174696E6700484A
:1016D000656174657254696D656F757400526568F3
:1016E0006561740048656174657254696D656F75F4
:1016F0007400507265737320627574746F6E202865
:101700006F72204D3130382920746F206865617404
:10171000206E6F7A7A6C650A004E6F7A7A6C65205B
:101720005061726B656400436F6E74696E7565001D
:101730004E6F7A7A6C65205061726B656400486FF9
:1017400074656E6420746F6F20636F6C640A00723E
:101750006573756D656400626567696E00436F6EE1
:1017600074696E75650044697361626C6552756E6B
:101770006F75740050757267654D6F7265005061CA
:1017800075736564004C6F61642046696C616D65BA
:101790006E7400436F6E74696E7565004C6F6164A2
:1017A0002046696C616D656E74205400496E7365E6
:1017B00072742066696C616D656E7420616E642060
:1017C000707265737320627574746F6E20286F7207
:1017D000204D313038290A00526573756D6500243B
:1017E000F4D43050C38E20C2A24017828B701112E5
:1017F0007A910D816CD90AA861E108C75866076122
:101800005143061E4B5D05C145A7041A4111040949
:101810003D9803713931034036DB0265339102D4C0
:10182000305402802E1D02632CEE01752AC501B0D2
:1018300028A001102781018F2564012B244B01E092
:10184000223401AC211F018D200D01801FFC00847A
:101850001EED00971DDF00B81CD200E61BC600205D
:101860001BBC00641AB200B219A8000A19A0006AD1
:10187000189900D117910040178B00B516840031DC
:10188000167E00B31579003A157300C7146F00581F
:10189000146A00EE1366008813630025135E00C708
:1018A000125B006C12570015125400C111510070E8
:1018B000114F0021114B00D61049008D10470046F2
:1018C00010440002104200C00F4000800F3E004252
:1018D0000F3C00060F3B00CB0E3800930E37005C28
:1018E0000E3500270E3400F30D3200C10D3100908B
:1018F0000D3000600D2E00320D2D00050D2C00D98D
:101900000C2B00AE0C2900850C29005C0C2700353F
:101910000C27000E0C2600E80B2400C40B2400A0AA
:101920000B23007D0B23005A0B2100390B210018DB
:101930000B2000F80A1F00D90A1E00BB0A1E009DDA
:101940000A1D00800A1D00630A1C00470A1B002CA8
:101950000A1B00110A1A00F7091A00DD091900C450
:10196000091900AB091900920917007B09180063D7
:101970000917004C09160036091600200916000A3E
:10198000091500F5081500E0081400CC081400B88B
:10199000081400A4081400900813007D0812006BBE
:1019A00008130058081200460812003408110023DA
:1019B0000811001208110001081100F0071000E0E2
:1019C000071000D0071000C0071000B0070F00A1DB
:1019D00007100091070E0083070F0074070F0065C2
:1019E000070E0057070E0049070E003B070D002E9B
:1019F000070E0020070D0013070D0006070D00F964
:101A0000060C00ED060D00E0060C00D4060C00C824
:101A1000060C00BC060C00B0060C00A4060B0099D6
:101A2000060C008D060B0082060B0077060B006C7F
:101A3000060B0061060A0057060B004C060A00421E
:101A4000060A0038060A002E060A0024060A001AB2
:101A5000060A001006090007060A00FD050900F441
:101A6000050900EB050900E2050900D9050900D0C8
:101A7000050900C7050900BE050900B5050800AD48
:101A8000050800A50509009C050800940508008CC0
:101A9000050800840508007C050800740508006C32
:101AA000050700650508005D050700560508004E9E
:101AB0000507004705070040050800380507003105
:101AC0000507002A050700230507001C0506001668
:101AD0000507000F0507000805060002050700FBC3
:101AE000040600F5040700EE040600E8040600E220
:101AF000040700DB040600D5040600CF040600C975
:101B0000040600C3040600BD040600B7040600B1C5
:101B1000040500AC040600A6040600A00405009B12
:101B200004060095040500900406008A040500855B
:101B3000040500800406007A0405007504050070A1
:101B40000405006B04050066040500610405005CE3
:101B500004050057040500520405004D0405004823
:101B6000040500430405003E0404003A0405003562
:101B7000040500300404002C04050027040400239D
:101B80000405001E0404001A0404001604050011D4
:101B90000404000D0404000904050004040400000A
:101BA000040400FC030400F8030400F4030400F040
:101BB000030400EC030400E8030400E4030400E071
:101BC000030400DC030400D8030400D4030400D0A1
:101BD000030400CC030400C8030300C5030300246E
:101BE000F404D9201BC40C5C0E9804C4095F026580
:101BF000077101F405F900FB04B30048048700C134
:101C00000369005803550003034500BE023A0084EF
:101C100002310053022A002902250004022000E4B8
:101C2000011C00C8011900AF0117009801140084BD
:101C3000011300710110006101100051010E0043F9
:101C4000010D0036010B002B010B0020010B0015CC
:101C50000109000C01090003010800FB000800F362
:101C6000000800EB000700E4000600DE000600D8D4
:101C7000000600D2000600CC000500C7000500C227
:101C8000000500BD000400B9000400B5000400B167
:101C9000000400AD000400A9000400A5000300A298
:101CA0000003009F0004009B0003009800030095C0
:101CB00000020093000300900003008D0002008BDF
:101CC00000030088000200860002008400030081F7
:101CD0000002007F0002007D0002007B000200790C
:101CE000000200770001007600020074000200721A
:101CF000000100710002006F0002006D0001006C25
:101D00000002006A0001006900020067000100662D
:101D10000001006500010064000200620001006132
:101D2000000100600001005F0002005D0001005C36
:101D30000001005B0001005A000100590001005839
:101D40000001005700010056000100550001005439
:101D50000001005300000053000100520001005137
:101D6000000100500001004F0001004E0000004E35
:101D70000001004D0001004C0001004B0000004B31
:101D80000001004A0001004900010048000000482D
:101D90000001004700010046000000460001004528
:101DA0000000004500010044000100430000004322
:101DB000000100420000004200010041000000411B
:101DC000000100400001003F0000003F0001003E14
:101DD0000000003E0001003D0000003D0001003C0D
:101DE0000000003C0000003C0001003B0000003B04
:101DF0000001003A0000003A0001003900000039FB
:101E000000010038000000380000003800010037F1
:101E100000000037000100360000003600000036E8
:101E200000010035000000350000003500010034DD
:101E300000000034000000340001003300000033D3
:101E400000000033000100320000003200000032C8
:101E500000010031000000310000003100010030BD
:101E600000000030000000300001002F0000002FB3
:101E70000000002F0000002F0001002E0000002EA7
:101E80000000002E0001002D0000002D0000002D9C
:101E90000000002D0001002C0000002C0000002C90
:101EA0000000002C0001002B0000002B0000002B84
:101EB0000000002B0001002A0000002A0000002A78
:101EC0000000002A0001002900000029000000296C
:101ED000000000290000002900010028000000285F
:101EE0000000002800000028000000280001002752
:101EF0000000002700000027000000270000002746
:101F00000001002600000026000000260000002638
:101F1000000000260001002500000025000000252B
:101F2000000000250000002500000025000100241D
:101F30000000002400000024000000240000002411
:101F40000001002300000023000000230000002304
:101F500000000023000000230000002300010022F5
:101F600000000022000000220000002200000022E9
:101F700000000022000100210000002100000021DB
:101F800000000021000000210000002100000021CD
:101F900000010020000000200000002000000020C0
:101FA00000000020000000200000002000000020B1
:101FB0000001001F0000001F0000001F0000001FA4
:101FC0000000001F0000001F0000001F0001001E95
:101FD0000000001E0000001E0000001E000000C2E5
:101FE0003100001C260000F4190000D80F0000EB9F
:101FF000080000C004000075020000400100005A03
:102000005F53544F505F50494E005A5F53544550F0
:102010005F50494E005A5F4D494E5F50494E005A3D
:102020005F454E41424C455F50494E005A5F44491E
:10203000525F50494E005A5F43535F50494E00591A
:102040005F53544F505F50494E00595F53544550B1
:102050005F50494E00595F4D41585F50494E0059FD
:102060005F454E41424C455F50494E00595F4449DF
:10207000525F50494E00595F43535F50494E0058DC
:102080005F53544F505F50494E00585F5354455072
:102090005F50494E00585F4D41585F50494E0058BF
:1020A0005F454E41424C455F50494E00585F4449A0
:1020B000525F50494E00585F43535F50494E0053A2
:1020C000535F50494E00534552564F335F50494E6F
:1020D00000534552564F325F50494E0053455256B9
:1020E0004F315F50494E00534552564F305F504973
:1020F0004E00534453530053445F444554454354A6
:102100005F50494E0053434B5F50494E0052414D82
:1021100050535F44395F50494E0052414D50535F18
:1021200044385F50494E0052414D50535F44313066
:102130005F50494E004D4F53495F50494E004D4F3F
:10214000534645545F445F50494E004D49534F5FDD
:1021500050494E004D4158363637355F53535F5026
:10216000494E004C45445F50494E00484541544556
:10217000525F4245445F50494E00484541544552E4
:102180005F305F50494E0046494C5F52554E4F55A7
:10219000545F50494E0046414E315F50494E004613
:1021A000414E5F50494E0045315F535445505F509A
:1021B000494E0045315F454E41424C455F50494EC6
:1021C0000045315F4449525F50494E0045315F43FD
:1021D000535F50494E0045305F535445505F50495E
:1021E0004E0045305F454E41424C455F50494E00E0
:1021F00045305F4449525F50494E0045305F43537C
:102200005F50494E00455F4D5558325F50494E0072
:10221000455F4D5558315F50494E00455F4D55580B
:10222000305F50494E004156525F53535F50494E04
:10223000004156525F53434B5F50494E0041565246
:102240005F4D4F53495F50494E004156525F4D49D3
:10225000534F5F50494E0054454D505F4245445FD7
:1022600050494E0054454D505F315F50494E005427
:10227000454D505F305F50494E0046494C574944E8
:1022800054485F50494E005458440052584400206E
:102290005400205200416363656C65726174696F1C
:1022A0006E3A2050003F4A206F7574206F6620728E
:1022B000616E67652028302E303120746F20302EFB
:1022C00033290A0050574D3A2020253464005057D6
:1022D0004D3A20202534640050574D3A20202534B3
:1022E000640050574D3A20202534640050574D3A31
:1022F00020202534640050574D3A202025346400B6
:1023000050574D3A20202534640050574D3A202034
:102310002534640050574D3A20202534640050572E
:102320004D3A20202534640050574D3A2020253462
:10233000640050574D3A20202534640050574D3AE0
:1023400020202534640050574D3A20202534640065
:1023500050574D3A20202534640050574D3A2020E4
:1023600025346400433A2000423A2000413A2000DC
:1023700020202020434F4D002020206E6F6E2D73B3
:1023800074616E646172642050574D206D6F646596
:1023900000202020636F6D7061726520696E746526
:1023A000727275707420656E61626C6564002020C5
:1023B000206F766572666C6F7720696E74657272D5
:1023C00075707420656E61626C6564003A2000204F
:1023D00020202054494D534B00423A200020202019
:1023E000205443435200413A2000202020205443EF
:1023F0004352002020202043533A20002020202058
:1024000057474D3A200050574D3A2020253464005C
:1024100050574D3A20202534640047004800000002
:1024200088008A008C00B300B400000098009A0075
:102430009C00A800AA00AC0028012A012C01202041
:10244000202054494D455200440045006E00800054
:1024500081006F00B000B100700090009100710029
:10246000A000A100720020012101730020697320E7
:10247000616C736F207469656420746F207468697F
:10248000732070696E0054494D45523143000A2053
:102490002E002020002020506F72743A200020204F
:1024A0002000202020416E616C6F6720696E203D06
:1024B0002025356C64003C756E757365642F756EF0
:1024C0006B6E6F776E3E00202841253264292020F4
:1024D000002533642000257350494E3A20004F7583
:1024E00074707574203D2000496E70757420203D15
:1024F0002000416E616C6F6720696E203D2025359C
:102500006C640070726F74656374656420002028C9
:102510004125326429202000253364200025735092
:10252000494E3A20008B220001872201017A223B8A
:10253000006F22430064224500572244004A2232A1
:10254000013D22330131223401262235011B22288C
:102550000110222A0105222C01FB212A01F0211C55
:1025600001E2211801D6211A01CC212C01C121221E
:1025700001B3211E01A72124019F210901962107F2
:1025800001872102017A210A016B21080163210DD3
:1025900001542142014B2132013E210701352133F3
:1025A0000127210A011A2108010D21090105213401
:1025B00001F7203101F2203501E7200B01DC200674
:1025C00001D1200501C6200401BF203501B6203508
:1025D00001AC2037019F202601952003018A203677
:1025E000017F200301762031016C203D015F2038FE
:1025F0000155200E014A203C013F200E01362028C3
:10260000012C2030011F203E01152012010A202E2E
:1026100001FF1F120157616974696E6720666F724E
:10262000206865617475702E0A004C656176696E6C
:102630006720473236003F53706563696669656499
:1026400020582C5920636F6F7264696E6174652025
:102650006F7574206F6620626F756E64732E0A004A
:102660003F28522965706561742076616C7565201C
:102670006E6F7420706C61757369626C653B206D60
:10268000757374206265206174206C6561737420B9
:10269000312E0A003F2852296570656174206D75DE
:1026A0007374206265207370656369666965642070
:1026B0007768656E206E6F74207573696E67206130
:1026C0006E204C43442E0A003F537065636966696F
:1026D0006564206E6F7A7A6C652074656D706572C2
:1026E0006174757265206E6F7420706C61757369AA
:1026F000626C652E0A003F537065636966696564A4
:102700002066696C616D656E742073697A65206EF0
:102710006F7420706C61757369626C652E0A003F7E
:10272000537065636966696564207072696D6520C0
:102730006C656E677468206E6F7420706C61757361
:1027400069626C652E0A003F5072696D65206C6588
:102750006E677468206D7573742062652073706590
:10276000636966696564207768656E206E6F7420A2
:102770007573696E6720616E204C43442E0A003FDA
:10278000537065636966696564206E6F7A7A6C65FB
:102790002073697A65206E6F7420706C617573693F
:1027A000626C652E0A003F52657472616374696FD2
:1027B0006E204D756C7469706C696572206D7573EF
:1027C00074206265207370656369666965642E0AAA
:1027D000003F537065636966696564205265747271
:1027E000616374696F6E204D756C7469706C696596
:1027F00072206E6F7420706C61757369626C652EE7
:102800000A003F537065636966696564206C61798D
:10281000657220686569676874206E6F7420706CDB
:1028200061757369626C652E0A0043292E0A003FA8
:1028300053706563696669656420626564207465C8
:102840006D7065726174757265206E6F7420706C46
:1028500061757369626C65202834302D004732360B
:10286000207374617274696E672E2E2E0A004F46B3
:10287000460A0046616465204865696768742000FF
:10288000426564204C6576656C696E672000466120
:10289000696C656420746F20656E61626C652042AE
:1028A0006564204C6576656C696E670A00496E76D2
:1028B000616C6964206D6573682E0A004469666600
:1028C00065723A200046726F6D5374703A0053740B
:1028D00065707065723A00556E4C6576656C3A00AD
:1028E0004C6576656C65643A005261773A20202029
:1028F00020000A4C6F676963616C3A004361703A6B
:10290000004D302F3120427265616B2043616C6C49
:10291000656400436F6E74696E7565004D302F31CC
:1029200020427265616B2043616C6C65640050727B
:102930006F6265205A204F66667365743A200050B6
:10294000726F62652059204F66667365743A200085
:1029500050726F62652058204F66667365743A2026
:10296000003F59206F7574206F662072616E676535
:102970002028302D33363020746F20333630290A2A
:10298000003F58206F7574206F662072616E676516
:102990002028302D33363020746F20333630290A0A
:1029A000003F5A206F7574206F662072616E6765F4
:1029B00020282D323020746F203230290A00220A5C
:1029C00000656E7175657565696E6720220020422D
:1029D000002050006F6B000000B4430000B44300BF
:1029E00000000000004842000048420000804057BC
:1029F00061726E696E673A20486F6D696E6720423A
:102A0000756D702044697669736F72203C20310ABD
:102A1000000202040000A0400000A04000000040AE
:102A20000000B4430000B4430000C8430101FF525A
:102A30006573656E643A200043616E6E6F74206F3B
:102A400070656E2073756264697220002569730079
:102A500025696D20256973002569682025696D2029
:102A600025697300256964202569682025696D2022
:102A70002569730025697920256964202569682006
:102A800025696D202569730023646566696E65207C
:102A900044454641554C545F0000626564004B64F8
:102AA00020004B6920004B702000504944204175A4
:102AB000746F74756E652066696E697368656421EC
:102AC0002050757420746865206C617374204B709D
:102AD0002C204B6920616E64204B6420636F6E7301
:102AE00074616E74732066726F6D2062656C6F77AF
:102AF00020696E746F20436F6E66696775726174CA
:102B0000696F6E2E680A00504944204175746F74D5
:102B1000756E65206661696C6564212074696D65F8
:102B20006F75740A00453120544845524D414C2080
:102B300052554E4157415900424544205448455250
:102B40004D414C2052554E415741590054686572D1
:102B50006D616C2052756E61776179004531204856
:102B6000656174696E67204661696C6564004265E1
:102B7000642048656174696E67204661696C6564AC
:102B80000048656174696E67206661696C65640000
:102B9000504944204175746F74756E652066616993
:102BA0006C6564212054656D706572617475726521
:102BB00020746F6F20686967680A00204B643A20B0
:102BC00000204B693A2000204B703A20000A204335
:102BD0006C617373696320504944200A00204B6480
:102BE0003A2000204B693A2000204B703A20000A1E
:102BF000204E6F206F76657273686F6F740A0020C5
:102C000054753A2000204B753A2000206D61783AC7
:102C10002000206D696E3A200020643A2000206276
:102C20006961733A2000504944204175746F74758E
:102C30006E652073746172740A00504944204175B6
:102C4000746F74756E65206661696C6564212054CB
:102C5000656D706572617475726520746F6F206840
:102C60006967680A00504944204175746F74756E35
:102C700065206661696C6564212042616420657825
:102C8000747275646572206E756D6265720A00708B
:102C9000012C0190012701B0012201C0011D01F0AA
:102CA0000118011002130130020E016002090190A7
:102CB000020401C002FF000003FA004003F5008097
:102CC00003F000D003EB002004E6007004E100E014
:102CD00004DC004005D700C005D2004006CD00D07E
:102CE00006C8008007C3003008BE00F008B900C065
:102CF00009B400B00AAF00B00BAA00D00CA50000C8
:102D00000EA000500F9B00C01096005012910000C2
:102D1000148C00C0158700B0178200B0197D00D058
:102D20001B7800001E730040206E0090226900F0A6
:102D300024640040275F0090295A00E02B550010C2
:102D40002E500020304B0010324600E033410090FE
:102D5000353C001037370070383200A0392D00B0F4
:102D60003A2800A03B2300603C1E00103D19009053
:102D70003D1400103E0F00703E0A00C03E050000EA
:102D80003F0000403FFBFF803FF6FFC03FF1FF20C8
:102D90002D20496E76616C69642065787472756463
:102DA0006572206E756D62657220210A001000C97F
:102DB0000210012C014001220170011801B0010E26
:102DC00001F00104015002FA00B002F0003003E605
:102DD00000D003DC009004D2007005C800A006BE3D
:102DE000000008B400B009AA00D00BA000600E9645
:102DF0000060118C000015820020197800C01D6E43
:102E000000A0226400B0275A00902C5000003146E8
:102E100000E0343C0010383200903A2800603C1E3C
:102E200000A03D1400803E0A00203F0000453120F4
:102E3000544845524D414C2052554E41574159003E
:102E400042454420544845524D414C2052554E4134
:102E500057415900546865726D616C2052756E61FE
:102E6000776179004531204572723A204D415854BE
:102E7000454D50004572723A204D415854454D50D1
:102E800020424544004D415854454D5020747269CC
:102E9000676765726564004531204572723A204D5E
:102EA000494E54454D50004572723A204D494E549A
:102EB000454D5020424544004D494E54454D50200B
:102EC000747269676765726564000A0A0020205A97
:102ED0005F4D494E3A002020595F4D41583A00203D
:102EE00020585F4D41583A004D3834205820592021
:102EF0005A204500202F002042403A0020403A004E
:102F000020573A0020573A006F70656E00545249BE
:102F1000474745524544003A200066696C616D653B
:102F20006E74007A5F6D696E00795F6D617800780C
:102F30005F6D6178005265706F7274696E672065AD
:102F40006E6473746F70207374617475730A0020FB
:102F50005A3A0020593A0020436F756E7420583A4F
:102F60000020453A00205A3A0020593A00583A00C9
:102F700020746F6F206C6F6E672065787472757344
:102F8000696F6E2070726576656E7465640A0020E4
:102F9000636F6C6420657874727573696F6E2070EE
:102FA000726576656E7465640A00446F6E652E0AFC
:102FB0000066616C7365004641494C3A204E6F20B3
:102FC00074726967676572206465746563746564AB
:102FD0000A004641494C3A204E6F6973652064658A
:102FE000746563746564202D20706C656173652061
:102FF00072652D72756E20746573740A00206465A5
:103000007465637465642E0A003D20424C546F75EC
:103010006368207072652056332E3120286F72202D
:10302000636F6D70617469626C6529003D205A2080
:10303000536572766F2050726F6265003D20424C7E
:10304000546F7563682056332E310020282B2F2DA6
:1030500020346D73293A20003A2033306D73206F8D
:1030600072206D6F72650A002E2050756C7365209A
:103070007769647468002A2A20506C656173652042
:10308000747269676765722070726F626520776914
:103090007468696E20333020736563202A2A0A0021
:1030A0004641494C3A20424C544F55434820656EA6
:1030B00061626C6564202D205365742075702074E6
:1030C0006869732064657669636520617320612097
:1030D000536572766F2050726F62652077697468ED
:1030E00020494E56455254494E472073657420740A
:1030F0006F202774727565272E0A002020444550E2
:103100004C4F5945442073746174653A204C4F57B5
:1031100020286C6F676963203029002020444550C7
:103120004C4F5945442073746174653A20484947AF
:103130004820286C6F676963203129003D204D6568
:103140006368616E6963616C20537769746368209A
:1031500064657465637465640A005741524E494E54
:10316000473A20494E56455254494E47207365749C
:1031700074696E672070726F6261626C792062613F
:10318000636B77617264732E0A002E204465706C45
:103190006F7920262073746F7720342074696D65F1
:1031A000730A003D20424C546F75636820436C6184
:1031B0007373696320312E322C20312E332C20532F
:1031C0006D61727420312E302C20322E302C203242
:1031D0002E322C20332E302C20332E312064657477
:1031E00065637465642E0A002E20436865636B2056
:1031F000666F7220424C544F5543480A002E205AA5
:103200005F4D494E5F454E4453544F505F494E56B3
:10321000455254494E473A20002E2050726F626545
:10322000205A5F4D494E5F50494E3A20002C207382
:10323000746F7720616E676C653A202020002C2027
:103240006465706C6F7920616E676C653A2000531D
:103250006572766F2070726F626520746573740A90
:103260002E207573696E6720696E6465783A202038
:10327000004D343320576169742043616C6C656480
:1032800000436F6E74696E7565004D34332057616D
:1032900069742043616C6C6564005761746368698C
:1032A0006E672070696E730A0064697300656E0052
:1032B00061626C65640A00656E6473746F70206D82
:1032C0006F6E69746F722000204500205A002059EB
:1032D00000204D3932205800205A00205900580053
:1032E00020204D61783A2000205A002059005800D3
:1032F00020204D696E3A2000536F667420656E641D
:1033000073746F70733A20004732380020496E762C
:10331000616C696420657874727564657220000060
:10332000002100240027002A002D00300033000176
:10333000010000040107010A010000220025002805
:10334000002B002E003100340002010000050108AE
:10335000010B01000020002300260029002C002F73
:103360000032000001000003010601090105050506
:1033700005070508080808020202020A0A080804EC
:10338000040404010101010101010103030303031A
:10339000030303040707070C0C0C0C0C0C0C0C02A9
:1033A00002020206060606060606060B0B0B0B0BB0
:1033B0000B0B0B01021020200808102040102040A9
:1033C00080020102010804020101020408102040E9
:1033D0008080402010080402018004020180402007
:1033E0001008040201080402010102040810204030
:1033F00080010204081020408000000A0B02090C22
:103400000D0E08070304010000000000000000008A
:1034100000000000000000000000000000000000AC
:103420000000000000121110000000000000000069
:10343000000000000000000000000000000000503C
:10344000726F62696E67204661696C65640A00503C
:10345000726F62696E67204661696C656400486FCF
:103460006D6520257325732573204669727374007A
:103470002046697273740A00486F6D652000544DD0
:10348000334420453520506C757320526561647952
:103490002E005072696E74696E672E2E2E00507267
:1034A000696E74205061757365640063616E636555
:1034B0006C005072696E742041626F7274656400B2
:1034C00055492041626F727400726573756D6500B5
:1034D0004D3234000000B4430000B4430000C84340
:1034E000000000000000000000000000290A002089
:1034F00062797465733B2063726320005365747452
:10350000696E67732053746F7265642028004545A7
:1035100050524F4D206461746173697A6520657201
:10352000726F722E0A00290A002062797465733B5B
:103530002063726320002073746F7265642073656A
:103540007474696E677320726574726965766564F8
:10355000202800202863616C63756C6174656429A0
:10356000210A0020213D2000454550524F4D204367
:103570005243206D69736D61746368202D20287338
:10358000746F7265642920002053697A653A2000BF
:10359000496E6465783A2000204D61726C696E3D19
:1035A000563730290A00454550524F4D20766572F6
:1035B00073696F6E206D69736D617463682028454F
:1035C0004550524F4D3D000A20696E6974207A7053
:1035D000726F62655F7A6F6666736574203D200066
:1035E000454550524F4D20496E697469616C697A46
:1035F00065640A0048617264636F646564204465B1
:103600006661756C742053657474696E6773204CC1
:103610006F616465640A00D0070000D00700006491
:103620000000004B00000000803B4400803B440051
:10363000002041000096420000A0420000A042008D
:103640000048440000BE423A0A0020204D36303384
:10365000200020440020204D3431322053004669A0
:103660006C616D656E742072756E6F757420736514
:103670006E736F723A0A002055004C0046696C6107
:103680006D656E74206C6F61642F756E6C6F616414
:10369000206C656E677468733A0A0020204D3930DB
:1036A00030204B004C696E65617220416476616E1A
:1036B00063653A0A0020204D383531205A00202019
:1036C0004D38353120590020204D383531205800F3
:1036D0005A2D50726F6265204F66667365740020C4
:1036E000440020490020204D333034205000204435
:1036F0000020490020204D333031205000504944F3
:103700002073657474696E67733A0A00204A00205A
:10371000204732392057204900205A0020204D34BC
:1037200032302053004175746F20426564204C652F
:1037300076656C696E673A0A00205A0020590020AD
:10374000204D323036205800486F6D65206F666618
:103750007365743A0A00204A002054002053002068
:10376000204D323035204200204A3C6A756E635F3E
:103770006465763E00416476616E6365643A20421A
:103780003C6D696E5F7365676D656E745F74696DBE
:10379000655F75733E20533C6D696E5F6665656459
:1037A000726174653E20543C6D696E5F747261761F
:1037B000656C5F66656564726174653E00205400E7
:1037C00020520020204D3230342050004163636588
:1037D0006C65726174696F6E2028756E6974732FE1
:1037E0007332293A20503C7072696E745F61636372
:1037F000656C3E20523C726574726163745F6163F4
:1038000063656C3E20543C74726176656C5F6163E5
:1038100063656C3E0A00204500205A0020590020B4
:10382000204D3230312058004D6178696D756D2022
:10383000416363656C65726174696F6E2028756E93
:103840006974732F7332293A0A00204500205A0008
:1038500020590020204D3230332058004D617869C6
:103860006D756D2066656564726174657320287579
:103870006E6974732F73293A0A005374657073204C
:1038800070657220756E69743A0A0020204D3230DE
:10389000302044300A0020204D32303020440020B7
:1038A00044697361626C65640A0046696C616D65A8
:1038B0006E742073657474696E67733A0020286DA6
:1038C0006D29002020473231202020203B20556EDA
:1038D00069747320696E206D6D00486F6D696E6745
:1038E000204661696C6564002E0A006F70656E2069
:1038F0006661696C65642C2046696C653A200070CD
:103900006F7765726F6666004B494C4C45442E20BC
:10391000005072696E7465722068616C7465642E03
:10392000206B696C6C28292063616C6C6564210ACA
:103930000053544F505045442E20005072696E740D
:1039400065722073746F707065642064756520748F
:103950006F206572726F72732E20466978207468CA
:1039600065206572726F7220616E642075736520C8
:103970004D39393920746F20726573746172742EF9
:10398000202854656D706572617475726520697365
:103990002072657365742E205365742069742061EC
:1039A000667465722072657374617274696E6729DA
:1039B0000A006563686F3A004572726F723A00429E
:1039C000696C696E656172204C6576656C696E67BD
:1039D00020477269643A0A00626564002C2073799A
:1039E0007374656D2073746F707065642120486511
:1039F000617465725F49443A2000426564204865FD
:103A00006174696E67204661696C65640048656130
:103A100074696E67206661696C6564004245442084
:103A2000544845524D414C2052554E415741590042
:103A3000546865726D616C2052756E6177617900B2
:103A400045312048656174696E67204661696C651F
:103A5000640048656174696E67206661696C6564BD
:103A600000453120544845524D414C2052554E415D
:103A700057415900546865726D616C2052756E61D2
:103A8000776179002B01010211241FBECFEFD1E233
:103A9000DEBFCDBF00E00CBF18E0A0E0B2E0E0EF79
:103AA000FDE502E00BBF02C007900D92AC3BB107F1
:103AB000D9F72EE1ACEBB8E001C01D92A339B207F3
:103AC000E1F71DE1C3E4DDE100E006C02197010953
:103AD000802FFE010F94212BC234D10780E008070C
:103AE000A9F70F94C9140D94E62E0C9400002F92A0
:103AF0003F924F925F926F927F928F929F92AF927E
:103B0000BF92CF92DF92EF92FF920F931F93CF93CA
:103B1000DF93CDB7DEB7E3970FB6F894DEBF0FBEE5
:103B2000CDBF80910901817091E098272091DB0839
:103B3000921781F19093DB08811116C00E94575EA5
:103B40008091391883FF09C08FEB93E00E94C45322
:103B500061E080E00F94AD0B1DC060E081E00F9448
:103B6000AD0B88ED93E014C00091391803FB0027DA
:103B700000F90E94E65D80913918877F809339189B
:103B8000002341F060E081E00F94AD0B81EF93E002
:103B90000E94C4538091A61481FF11C180912B16FD
:103BA00090912C16891B8F70843008F008C18CE02E
:103BB000E5EAF3E1DE01119601900D928A95E1F7B5
:103BC0008091770290917802A0917902B0917A0267
:103BD00088A799A7AAA7BBA79C01AD016091A513CF
:103BE0007091A6138091A7139091A8130F94292B7D
:103BF0006B017C016093A5137093A6138093A713A8
:103C00009093A81380917B0290917C02A0917D02F9
:103C1000B0917E028CA79DA7AEA7BFA79C01AD0166
:103C20006091A9137091AA138091AB139091AC137A
:103C30000F94292B68A379A38AA39BA36093A9134C
:103C40007093AA138093AB139093AC1380917F026F
:103C500090918002A0918102B091820288AB99ABD1
:103C6000AAABBBAB9C01AD016091AD137091AE13DB
:103C70008091AF139091B0130F94292B4B015C01ED
:103C80006093AD137093AE138093AF139093B01302
:103C9000A7019601C701B6010F949A242B013C019C
:103CA00028A139A14AA15BA1CA01B9010F949A24A4
:103CB0009B01AC01C301B2010F942A2B2B013C01E3
:103CC000A5019401C501B4010F949A249B01AC0194
:103CD000C301B2010F942A2B0F94D82D9B01AC0184
:103CE00060E070E080E89FE30F94242C209165024F
:103CF0003091660240916702509168020F949A24B5
:103D00002DEC3CEC4CEC5DE30F949A2420E030E089
:103D100040E85EE30F949A242B013C0120E030E060
:103D200040E85FE30F94342487FFF1C3A3019201BD
:103D3000C701B6010F949A2428A539A54AA55BA509
:103D40000F942A2B6093A5137093A6138093A71347
:103D50009093A813A301920168A179A18AA19BA1C4
:103D60000F949A242CA53DA54EA55FA50F942A2B50
:103D70006093A9137093AA138093AB139093AC1321
:103D8000A3019201C501B4010F949A2428A939A96D
:103D90004AA95BA90F942A2B6093AD137093AE13BD
:103DA0008093AF139093B0130E941FDB8CE0FE0151
:103DB0003196A5EAB3E101900D928A95E1F78091E1
:103DC000DA0881110C945A398091D8089091D90859
:103DD0009C012F5F3F4F3093D9082093D808883E2D
:103DE000934010F40C945A3981E08093DA081092D1
:103DF000D9081092D8088091B312882309F498C387
:103E00000E94EAC5811194C38091D7088F5F809387
:103E1000D7088091D708853620F01092D7081092E5
:103E2000B312E091B3128E2FEE0F990BAA0BBB0BBE
:103E3000FC013197E730F10508F0A0C08827EE5863
:103E4000FF4F8F4F0D94212B0E94E2C5882309F468
:103E500095C081E080933E0284E094E00E94C453C8
:103E600080E190E09093BE168093BD1685E080932C
:103E7000B11602E80093B41684E190E1A0E0B0E04E
:103E80008093B5169093B616A093B716B093B81654
:103E90000F94D10281E09AE59093BE168093BD16EF
:103EA00086E390E09093C0168093BF1687E08093DE
:103EB000B1160093B41684E890E0A0E0B0E08093DF
:103EC000B5169093B616A093B716B093B8160F9484
:103ED000D10252C00E94E2C5882309F44FC048C0F5
:103EE00082E194E00E94C45381E09AE59093BE166B
:103EF0008093BD1680E490E09093C0168093BF1627
:103F000007E00093B11682E88093B41684E890E04D
:103F1000A0E0B0E08093B5169093B616A093B716C4
:103F2000B093B8160F94D1020093B31227C08091BA
:103F3000D608882319F10E94E2C58823F9F00E946F
:103F4000EAC581111BC0F7C20E94E2C58823B1F007
:103F50000E94EAC5811112C01CC30E94EAC58111EA
:103F60000DC042E060E070E0CB010E9400C604C0DA
:103F70000E94EAC5811102C01092B31280913E02E4
:103F8000882309F4ACC28091AF129091B012892BB2
:103F900009F08FC18091D3089091D408892B09F042
:103FA0001EC184E096E09093BE168093BD1680EA11
:103FB00090E89093C0168093BF1617E01093B11647
:103FC00002E80093B41680EA90E0A0E0B0E08093AD
:103FD000B5169093B616A093B716B093B8160F9473
:103FE000D1028091060290910702A0910802B0913F
:103FF00009020097A105B10511F51092BE161092A5
:10400000BD1615E01093B1160093B4168AE890E13E
:10401000A0E0B0E08093B5169093B616A093B716C3
:10402000B093B8160F94D10289E090E09093BE1639
:104030008093BD161093B1160093B41640C001963C
:10404000A11DB11DF5E0B695A79597958795FA95B1
:10405000D1F70197A109B109009731E0A307B10594
:1040600058F0B093BE16A093BD169093C0168093DF
:10407000BF161093B11607C09093BE168093BD165D
:1040800085E08093B11612E81093B4168AE890E1A7
:10409000A0E0B0E08093B5169093B616A093B71643
:1040A000B093B8160F94D10288E090E09093BE16BA
:1040B0008093BD1685E08093B1161093B4168CE8FA
:1040C00090E1A0E0B0E08093B5169093B616A0936F
:1040D000B716B093B8160F94D10280910602909152
:1040E0000702A0910802B09109020097E1E0AE0733
:1040F000B10550F0B093BE16A093BD169093C016B4
:104100008093BF1687E005C09093BE168093BD16BE
:1041100085E08093B11682E88093B41688E890E138
:10412000A0E0B0E08093B5169093B616A093B716B2
:10413000B093B8160F94D1028091060290910702B5
:10414000A0910802B0910902BA2FA92F982F8827B1
:104150000097F1E0AF07B10550F0B093BE16A09301
:10416000BD169093C0168093BF1687E005C090934C
:10417000BE168093BD1685E08093B11612E81093A9
:10418000B41681EA90E0A0E0B0E08093B516909379
:10419000B616A093B716B093B8160F94D1028091BB
:1041A000B618882319F082E090E002C083E090E026
:1041B0009093BE168093BD1685E08093B116109340
:1041C000B41685E490E1A0E0B0E08093B51690933A
:1041D000B616A093B716B093B8160F94D1020091FB
:1041E000D3081091D408053611057CF41093BE163F
:1041F0000093BD1685E08093B11682E88093B416D3
:1042000080E090E1A0E0B0E011C0C80184569109BF
:104210009093BE168093BD1685E08093B11682E818
:104220008093B41681E090E1A0E0B0E08093B516F1
:104230009093B616A093B716B093B8160F94D10208
:104240000F5F1F4F1093D4080093D308093C11054A
:1042500064F180E294E00E94C45381E090E0909386
:10426000B0128093AF1280933E0281E09AE5909362
:10427000BE168093BD168DE290E09093C016809399
:10428000BF1687E08093B11682E88093B41684E865
:1042900090E0A0E0B0E08093B5169093B616A0939E
:1042A000B716B093B8160F94D1021092DA080C9496
:1042B0005A3980912B1690912C16891B8F7009F01A
:1042C00092C10E9487CF81118EC18091391882FDE1
:1042D0008AC112C384E690E09093BE168093BD1607
:1042E0001093B1160093B4168EE090E1A0E0B0E018
:1042F0008093B5169093B616A093B716B093B816E0
:104300000F94D102C60182539048880F991F909351
:10431000BE168093BD161093B1160093B4168FE0AD
:1043200090E1A0E0B0E08093B5169093B616A0930C
:10433000B716B093B8160F94D1020E9417F590E00B
:104340009093BE168093BD1685E08093B11682E8E7
:104350008093B41686E190E1A0E0B0E08093B516BA
:104360009093B616A093B716B093B8160F94D102D7
:1043700020E030E048EC52E46091C9137091CA1318
:104380008091CB139091CC130F949A240F94962C78
:104390007093BE166093BD1615E01093B11602E837
:1043A0000093B41686E290E1A0E0B0E08093B516E9
:1043B0009093B616A093B716B093B8160F94D10287
:1043C0006091EE0B7091EF0B8091F00B9091F10BDF
:1043D0000F94962C7093BE166093BD161093B11671
:1043E0000093B41686E390E1A0E0B0E08093B516A8
:1043F0009093B616A093B716B093B8160F94D10247
:1044000060918709709188098091890990918A0942
:104410000F94962C7093BE166093BD161093B11630
:104420000093B4168CE390E1A0E0B0E08093B51661
:104430009093B616A093B716B093B8160F94D10206
:104440008091F20B9091F30B9093BE168093BD1662
:104450001093B1160093B41684E390E1A0E0B0E0AD
:104460008093B5169093B616A093B716B093B8166E
:104470000F94D10280918B0990918C099093BE1674
:104480008093BD161093B1160093B4168AE390E1A1
:10449000A0E0B0E08093B5169093B616A093B7163F
:1044A000B093B8160F94D1020091CF0801113CC10E
:1044B0008091D108811138C18091D60881118BC1BA
:1044C0008091651690916616A0916716B091681656
:1044D0008C3420E19207A105B10509F0A1C131E0BA
:1044E000C32E37E1D32E0AE187EA94E10E942F5CC4
:1044F000E090C408F090C508181619060CF085C3A2
:104500008AE1E816F10414F40C941B357EC38CE0A8
:10451000FE013196A5EAB3E101900D928A95E1F78B
:104520000E941FDB8091A6148D7F8093A61447CC38
:104530001092D7086ECC82ED95E00E94C453809112
:10454000D50890E0A0E0B0E0895B9F4FAE4FB54A40
:1045500021E03AE53093BE162093BD169093C01625
:104560008093BF1687E08093B11682E88093B416DB
:1045700084E890E0A0E0B0E08093B5169093B61682
:10458000A093B716B093B8160F94D1021092D60824
:10459000F3CC81E080933E021092B31280EE95E05E
:1045A0000E94C45381E09AE59093BE168093BD1695
:1045B0008EE490E09093C0168093BF1687E08093BE
:1045C000B11682E88093B41684E890E0A0E0B0E0F1
:1045D0008093B5169093B616A093B716B093B816FD
:1045E0000F94D102CBCC8CE090E09093BE168093D8
:1045F000BD1605E00093B11682E88093B41684E1FD
:1046000090E1A0E0B0E08093B5169093B616A09329
:10461000B716B093B8160F94D1020E94F9F320E1B7
:104620003EE040E050E00F948A2A2115310591E0E8
:104630004907510560F05093BE164093BD16309364
:10464000C0162093BF1687E08093B11606C0309342
:10465000BE162093BD160093B11602E80093B4165F
:1046600080E190E1A0E0B0E08093B5169093B6169B
:10467000A093B716B093B8160F94D1020E94F9F325
:1046800020E13EE040E050E00F948A2A2CE330E045
:1046900040E050E00F948A2A3093BE162093BD1656
:1046A00015E01093B1160093B41682E190E1A0E0FA
:1046B000B0E08093B5169093B616A093B716B0935A
:1046C000B8160F94D1020E9417F5882391F00E942A
:1046D00017F58F5F8093D208C82ED12C833308F052
:1046E000F9CDC601880F991F9093BE168093BD1611
:1046F00004C01092BE161092BD161093B11600930E
:10470000B4168EE090E1A0E0B0E08093B5169093EF
:10471000B616A093B716B093B8160F94D1021092A4
:10472000BE161092BD16F7CD20E030E048EC52E402
:104730006091EE0B7091EF0B8091F00B9091F10B6B
:104740000F949A246B017C016091F20B7091F30B32
:10475000072E000C880B990B0F943B249B01AC0196
:10476000C701B6010F94242C0F949D2C643671055B
:1047700010F064E670E07093BE166093BD1645E0DD
:10478000A42EA092B11652E8B52EB092B41684E2CF
:1047900090E1A0E0B0E08093B5169093B616A09398
:1047A000B716B093B8160F94D102C090EE0BD0900C
:1047B000EF0BE090F00BF090F10B20E030E040E2E6
:1047C00053E4C701B6010F948A2D18160CF03AC1B4
:1047D000011188C137C18091C60801E0080F00931C
:1047E000C60890E09093BE168093BD1685E0809336
:1047F000B11682E88093B41682E490E1A0E0B0E0C4
:104800008093B5169093B616A093B716B093B816CA
:104810000F94D1020A3008F453CE1092C60850CE3D
:104820008A349041A105B10509F459CE80E00E9477
:10483000DEC620E030E040E251E40F949A240F9469
:10484000962C7093BE166093BD1615E01093B116AA
:1048500002E80093B41688E490E1A0E0B0E0809311
:10486000B5169093B616A093B716B093B8160F94DA
:10487000D10281E00E94DEC620E030E040E251E457
:104880000F949A240F94962C7093BE166093BD16C5
:104890001093B1160093B4168AE490E1A0E0B0E062
:1048A0008093B5169093B616A093B716B093B8162A
:1048B0000F94D10282E00E94DEC620E030E040E2A8
:1048C00051E40F949A240F94962C7093BE16609323
:1048D000BD161093B1160093B4168CE490E1A0E0DD
:1048E000B0E08093B5169093B616A093B716B09328
:1048F000B8160F94D102F3CD809187099091880961
:10490000A0918909B0918A0988A399A3AAA3BBA3FE
:1049100060918B0970918C09072E000C880B990B04
:104920000F943B246B017C0120E030E040E050E438
:104930000F94292B28A139A14AA15BA10F948A2D9C
:10494000181604F14090EE0B5090EF0B6090F00BB6
:104950007090F10B6091F20B7091F30B072E000C2D
:10496000880B990B0F943B244B015C0120E030E055
:1049700040E251E40F94292BA30192010F948A2D58
:10498000181604F58DE090E09093BE168093BD1646
:1049900085E08093B11682E88093B41684E190E1BB
:1049A000A0E0B0E08093B5169093B616A093B7162A
:1049B000B093B8160F94D1028091B21281113FC00A
:1049C00081E03DC020E030E040E050E4C701B601A6
:1049D0000F942A2B28A139A14AA15BA10F9434245A
:1049E00087FD0EC020E030E040E251E4C501B40193
:1049F0000F942A2BA30192010F94342487FFB8CC83
:104A000084E190E09093BE168093BD1685E080937C
:104A1000B11682E88093B41684E190E1A0E0B0E0A2
:104A20008093B5169093B616A093B716B093B816A8
:104A30000F94D1028091B212811101C082E0809363
:104A4000B21296CC6091F20B7091F30B072E000C12
:104A5000880B990B0F943B249B01AC01C701B60155
:104A60000F948A2D6091D10887FDAEC0662309F4AA
:104A700023CD062E000C770B8BE397E00F94620B8F
:104A80001092D1081092D4081092D30884E090E0DC
:104A90009093BE168093BD1685E08093B11602E810
:104AA0000093B4168EE890E1A0E0B0E08093B516D4
:104AB0009093B616A093B716B093B8160F94D10280
:104AC00081E09AE59093BE168093BD1683E590E051
:104AD0009093C0168093BF1687E08093B116009321
:104AE000B41663C01092CF0820E030E040E251E4F9
:104AF0006091C7087091C8088091C9089091CA0850
:104B00000F949A240F94962C7093BE166093BD1642
:104B1000A092B116B092B41684E590E1A0E0B0E0A6
:104B20008093B5169093B616A093B716B093B816A7
:104B30000F94D10220E030E040E251E46091CB08D4
:104B40007091CC088091CD089091CE080F949A2452
:104B50000F94962C7093BE166093BD16A092B1165A
:104B6000B092B41688E590E1A0E0B0E08093B5166D
:104B70009093B616A093B716B093B8160F94D102BF
:104B80008EEE95E00E94C45381E09AE59093BE16A4
:104B90008093BD1681E490E09093C0168093BF1679
:104BA00087E08093B116B092B41684E890E0A0E05C
:104BB000B0E08093B5169093B616A093B716B09355
:104BC000B8160F94D10278CC662309F475CC809185
:104BD000D3089091D4089C012F5F3F4F3093D408A5
:104BE0002093D30865E070E00F940D2B9093BE16D0
:104BF0008093BD1685E08093B11682E88093B41649
:104C00008EE890E1A0E0B0E0D4CF1E141F040CF0B9
:104C10004CCB9091621680910117981322C090910D
:104C200063168091021798131CC023E0E216F1046A
:104C3000C4F09091031790936116809104178093AC
:104C400064169330D1F4982F9D7F9038B1F49091F1
:104C500005179F3409F059C0909106179B3409F04D
:104C600054C08AE1E1E0F7E1DF011D928A95E9F79E
:104C70001092C5081092C40818CB833809F045C0BB
:104C80008091051790910617982789279827A0E00B
:104C9000B0E08093651690936616A0936716B09364
:104CA0006816C0900717D12CE12CF12CC092691620
:104CB000D0926A16E0926B16F0926C16A8E0B7E1FB
:104CC00040E050E0BA014C155D056E057F0508F027
:104CD0004AC04A015B01B694A79497948794F40163
:104CE0003696EE0FFF1FEF59F94E8C9190E0982FFA
:104CF000882711962C911197822B918380834E5F88
:104D00005F4F6F4F7F4F1296DECF813861F58091F4
:104D1000051790E0A0E0B0E08093651690936616CA
:104D2000A0936716B093681680910617482F50E03D
:104D300060E070E04093691650936A1660936B16BA
:104D400070936C16A7E0B7E1EDE6F6E190E020E0A5
:104D500030E02817390739F04D9150E041935193D5
:104D60002F5F3F4FF6CF8AE1E1E0F7E1DF011D92CF
:104D70008A95E9F71092C5081092C40881E394E07F
:104D80000E94C4536091B312161664F4062E000CF0
:104D9000770B80E397E00F94620B8AE00E94B95290
:104DA0000C940C3560916D1670916E168EE197E043
:104DB0000F94440B8AE00E94B952409165165091BD
:104DC000661660916716709168168FE097E00F94F1
:104DD000330B8AE00E94B952809165169091661655
:104DE000A0916716B0916816EDE8F2E000E010E0DF
:104DF0004191519161917191411551056105710583
:104E0000D1F1481759076A077B0791F5AC01BD013D
:104E100048505041610971094530510561057105DE
:104E200068F1AC01BD01477F423350416105710516
:104E300041F18433F0E19F07A105B10511F1AC0107
:104E4000BD01465450416109710947305105610562
:104E50007105D0F0AC01BD014455504161097109A3
:104E6000453051056105710588F402E110E00EC07E
:104E70000F5F1F4FBDCF0FEF1FEF08C003E010E023
:104E800005C008E010E002C00FE010E08A50904238
:104E9000A109B109833D9105A105B10530F00F3F8E
:104EA0002FEF120721F40C940C3509E110E0F2E524
:104EB000CF2EF4E0DF2EF60181916F01882319F0E7
:104EC0000E94B952F8CFB801012E000C880B990B43
:104ED0000E942D530E94BE5383E097E00E94C4536A
:104EE0000A31110510F00C940835F8018827E758AD
:104EF000FF4F8F4F0D94212B80916D1690916E1660
:104F000081309105E1F410923E028FEF8093151BE2
:104F100060E080E00F94AD0B00E614E0D8018D91C5
:104F20008D01882319F00E94B952F8CF81E09AE5EB
:104F30009093BE168093BD168EE290E0AFC0823093
:104F4000910509F0C5C081E080933E020E9488F57A
:104F50008FEF96E09093C0098093BF098BE090E0BB
:104F60009093BE168093BD1605E00093B11612E82B
:104F70001093B41680E092E1A0E0B0E08093B51603
:104F80009093B616A093B716B093B8160F94D102AB
:104F90001092BE161092BD160093B1161093B4165F
:104FA0008EE090E1A0E0B0E08093B5169093B61645
:104FB000A093B716B093B8160F94D1021092BE16F4
:104FC0001092BD160093B1161093B4168FE090E1C5
:104FD000A0E0B0E08093B5169093B616A093B716F4
:104FE000B093B8160F94D1021092BE161092BD164F
:104FF0000093B1161093B41686E190E1A0E0B0E002
:105000008093B5169093B616A093B716B093B816C2
:105010000F94D10262E070E080E090E00E94F2C65E
:105020001092BE161092BD160093B1161093B416CE
:1050300080E190E1A0E0B0E08093B5169093B616C1
:10504000A093B716B093B8160F94D1021092BE1663
:105050001092BD160093B1161093B41682E190E140
:10506000A0E0B0E08093B5169093B616A093B71663
:10507000B093B8160F94D1020AE814E0F8018191B8
:105080008F01882319F00E94B952F8CF81E09AE588
:105090009093BE168093BD168DE290E09093C0165B
:1050A0008093BF1687E08093B11682E88093B41690
:1050B00084E890E0A0E0B0E08093B5169093B61637
:1050C000A093B716B093B8160F94D1020C940C3578
:1050D0008330910549F581E080933E0204EB14E0B2
:1050E000D8018D918D018823C9F00E94B952F8CF63
:1050F0008091651690916616A0916716B09168161A
:105100008233F0E19F07A105B10509F05BC48091EE
:105110006D1690916E16009709F023C480910502D8
:10512000882309F40DC31DC3049711F00C940C35AA
:1051300010923E020C940C3580916D1690916E1673
:1051400081309105D1F410923E02809105028823AE
:1051500019F082E090E002C083E090E09093BE16E8
:105160008093BD1685E08093B11682E88093B416D3
:105170008EE190E1A0E0B0E09FCF8230910519F57B
:105180000EED14E0F80181918F01882319F00E943F
:10519000B952F8CF81E080933E028091B212843000
:1051A00049F081E09AE59093BE168093BD1685E3A1
:1051B00090E074CF81E09AE59093BE168093BD167F
:1051C00086E390E06BCF8330910509F04CC02091CD
:1051D0000502222319F19093BE168093BD1685E037
:1051E0008093B11682E88093B4168EE190E1A0E03E
:1051F000B0E08093B5169093B616A093B716B0930F
:10520000B8160F94D10240E060E070E088EC92E4C0
:105210000E94EFF5109205020C940C3582E090E0AC
:105220009093BE168093BD1685E08093B11682E8F8
:105230008093B4168EE190E1A0E0B0E08093B516C3
:105240009093B616A093B716B093B8160F94D102E8
:1052500040E060E070E0CB010E94EFF581E08093D8
:1052600005020C940C35049711F00C940C358091C8
:105270009A098823F1F082E090E09093BE16809323
:10528000BD1685E08093B11682E88093B4168FE155
:1052900090E1A0E0B0E08093B5169093B616A0938D
:1052A000B716B093B8160F94D10210929A090C94C5
:1052B0000C3583E090E09093BE168093BD1685E098
:1052C0008093B11682E88093B4168FE190E1A0E05C
:1052D000B0E08093B5169093B616A093B716B0932E
:1052E000B8160F94D10281E080939A090C940C3582
:1052F00060916D1670916E1680E090E00F943924E5
:105300006B017C0120E030E04AEF53E40F94342439
:1053100087FF11C020E030E040E251E4C701B60150
:105320000F948A2D18166CF0C12CD12C70E2E72E48
:1053300071E4F72E06C0C12CD12CEAEFEE2EE3E487
:10534000FE2EC701B6010F94962C709360026093F5
:105350005F020C940C358091651690916616A091B1
:105360006716B09168168830F0E19F07A105B10576
:1053700009F050C081E09AE59093BE168093BD1667
:105380008DE290E09093C0168093BF1687E08093E3
:10539000B11612E81093B41684E890E0A0E0B0E0F3
:1053A0008093B5169093B616A093B716B093B8161F
:1053B0000F94D1021092BE161092BD1605E0009314
:1053C000B1161093B41680E190E1A0E0B0E08093B4
:1053D000B5169093B616A093B716B093B8160F945F
:1053E000D1021092BE161092BD160093B116109302
:1053F000B41682E190E1A0E0B0E08093B5169093FE
:10540000B616A093B716B093B8160F94D1020E94A7
:1054100088F58FC08A3020E19207A105B105E1F53A
:1054200080916D1690916E16813F910511F00C944C
:105430000C3581E09AE59093BE168093BD1686E305
:1054400090E09093C0168093BF1687E08093B116CA
:1054500082E88093B41684E890E0A0E0B0E0809306
:10546000B5169093B616A093B716B093B8160F94CE
:10547000D1024EE755E065E875E084E00E94A28E17
:1054800060E081E795E00E9449F587E695E090931A
:10549000C0098093BF094DC08C309041A105B10572
:1054A00009F047C080916D1690916E16019709F032
:1054B00040C00F940C1E1092B21281E080933E0205
:1054C0008CE090E09093BE168093BD1685E08093AB
:1054D000B11612E81093B41684E190E1A0E0B0E0B8
:1054E0008093B5169093B616A093B716B093B816DE
:1054F0000F94D10281E09AE59093BE168093BD1679
:1055000085E390E09093C0168093BF1687E0809368
:10551000B1161093B41684E890E0A0E0B0E0809358
:10552000B5169093B616A093B716B093B8160F940D
:10553000D1028091651690916616A0916716B09180
:1055400068168C309041A105B10511F00C940C3512
:1055500080916D1690916E16029711F00C940C3597
:105560000F940C1E81E08093D1081092B2128093A8
:105570003E021092D4081092D30881E09AE59093ED
:10558000BE168093BD1682E590E088CD20916D1601
:1055900030916E16B90180E090E037FF09C00F949A
:1055A000392420E030E040E857E40F94292B02C072
:1055B0000F94392420E030E048EC52E40F94242C7E
:1055C0006B017C0120E030E040EA51EC0F948A2D21
:1055D00087FD31C020E030E040EA51E4C701B60168
:1055E0000F94342418163CF1A70196016091C91359
:1055F0007091CA138091CB139091CC130F94292BE7
:1056000020E030E048EC53E40F949A2490580F9433
:10561000962CCB010F94C605C092C913D092CA1321
:10562000E092CB13F092CC138AEF96E09093C009EE
:105630008093BF0928C020E030E048EC52E460913C
:10564000C9137091CA138091CB139091CC130F940E
:105650009A240F94962C7093BE166093BD1685E025
:105660008093B11682E88093B41686E290E1A0E0C0
:10567000B0E08093B5169093B616A093B716B0938A
:10568000B8160F94D1026091C9137091CA1380911A
:10569000CB139091CC138E010B5E1F4F23E041E0A2
:1056A0000F940C1F9F938F938CEE96E09F938F9394
:1056B000045111091F930F930F94CC23C8010E942A
:1056C000CCC70F900F900F900F900F900F900C94ED
:1056D0000C3580916D1690916E16009729F481E03B
:1056E00080933E020C940C3581309105B1F4809189
:1056F0000502882349F081E09AE59093BE168093D5
:10570000BD168CE390E0CACC81E09AE59093BE167A
:105710008093BD168BE390E0C1CC82309105F9F205
:105720008330910539F58091050240E0882389F0A6
:1057300060E070E088EC92E40E94EFF510920502C0
:1057400081E09AE59093BE168093BD1689E390E0C0
:10575000A5CC60E070E0CB010E94EFF581E0809382
:10576000050281E09AE59093BE168093BD168AE308
:1057700090E094CC8530910559F540E060E070E010
:1057800084E393E40E9475C546E060E070E08CE835
:1057900092E40E9475C584EB90E09093BE168093CE
:1057A000BD1605E00093B11612E81093B41684E319
:1057B00090E1A0E0B0E08093B5169093B616A09368
:1057C000B716B093B8160F94D10286E490E02DC0BE
:1057D0008630910599F540E060E070E080E793E461
:1057E0000E9475C546E060E070E08CED92E40E9496
:1057F00075C580EF90E09093BE168093BD1605E0CE
:105800000093B11612E81093B41684E390E1A0E07F
:10581000B0E08093B5169093B616A093B716B093E8
:10582000B8160F94D1028EE690E09093BE16809346
:10583000BD160093B1161093B416BFC0813F9105F9
:1058400011F00C940C3540E060E070E0CB010E9458
:10585000EFF541E060E070E0CB010E94EFF51092BF
:10586000050240E060E070E0CB010E9475C546E0B3
:1058700060E070E0CB010E9475C51092BE161092D8
:10588000BD1605E00093B11612E81093B41684E338
:1058900090E1A0E0B0E08093B5169093B616A09387
:1058A000B716B093B8160F94D10261E070E080E0B3
:1058B00090E00E94F2C61092BE161092BD160093A0
:1058C000B1161093B4168AE390E1A0E0B0E08093A3
:1058D000B5169093B616A093B716B093B8160F945A
:1058E000D10261E070E080E090E00E94F2C684E1C5
:1058F00090E09093BE168093BD160093B11610935E
:10590000B41684E190E1A0E0B0E08093B5169093E6
:10591000B616A093B716B093B8160F94D10281E0D3
:105920009AE59093BE168093BD1689E390E090931C
:10593000C0168093BF1687E08093B1161093B416FB
:1059400084E890E0A0E0B0E08093B5169093B6169E
:10595000A093B716B093B8160F94D10282E00C94BE
:10596000053581309105A9F440E060E070E0CB019D
:105970000E9475C51092BE161092BD1685E08093E8
:10598000B11682E88093B41684E390E1A0E0B0E021
:1059900093CB029711F00C940C3546E060E070E078
:1059A000CB010E9475C51092BE161092BD1685E0FF
:1059B0008093B11682E88093B4168AE390E1A0E068
:1059C000B0E07ACB843320E19207A105B10551F410
:1059D00060916D1670916E1680E090E00F943924FE
:1059E00040E010C08A339041A105B10511F00C943C
:1059F0000C3560916D1670916E1680E090E00F94FA
:105A0000392446E00E9475C50C940C3580916D16C2
:105A100090916E16009709F462CE8130910509F0DD
:105A20004CC08091B618882319F083E090E002C042
:105A300082E090E09093BE168093BD1685E080933F
:105A4000B11682E88093B41685E490E1A0E0B0E05E
:105A50008093B5169093B616A093B716B093B81668
:105A60000F94D1028AE090E09093BE168093BD1609
:105A700085E08093B11682E88093B41680E092E1CD
:105A8000A0E0B0E08093B5169093B616A093B71639
:105A9000B093B8160F94D1020E94E2C5811103C0E1
:105AA0008CED96E002C080ED96E09093C009809363
:105AB000BF0982E08093B31271C18230910509F071
:105AC000A8C081E080933E0288E0E7ECF8E0DF01C7
:105AD0001D928A95E9F780E090E0A0E2B1E480931E
:105AE000C7089093C808A093C908B093CA088093C8
:105AF000CB089093CC08A093CD08B093CE0884E651
:105B000090E09093BE168093BD1605E00093B11609
:105B100012E81093B41684E590E1A0E0B0E0809321
:105B2000B5169093B616A093B716B093B8160F9407
:105B3000D10220E030E040E251E46091CB08709166
:105B4000CC088091CD089091CE080F949A240F94A0
:105B5000962C7093BE166093BD160093B1161093E9
:105B6000B41688E590E1A0E0B0E08093B51690937C
:105B7000B616A093B716B093B8160F94D1026091E1
:105B8000EE0B7091EF0B8091F00B9091F10B0F9455
:105B9000962C7093BE166093BD160093B1161093A9
:105BA000B41686E390E1A0E0B0E08093B516909340
:105BB000B616A093B716B093B8160F94D102809181
:105BC000F20B9091F30B9093BE168093BD16009349
:105BD000B1161093B41684E390E1A0E0B0E0809396
:105BE000B5169093B616A093B716B093B8160F9447
:105BF000D10262E070E080E090E00E94F2C681E0B5
:105C00009AE59093BE168093BD1681E490E00C94C3
:105C100048368330910509F076C01092D50880E0AF
:105C20000E94DEC620E030E040E251E40F949A2466
:105C30000F94962C7093BE166093BD1605E00093EA
:105C4000B11612E81093B41688E490E1A0E0B0E039
:105C50008093B5169093B616A093B716B093B81666
:105C60000F94D10281E00E94DEC620E030E040E2E5
:105C700051E40F949A240F94962C7093BE1660935F
:105C8000BD160093B1161093B4168AE490E1A0E01B
:105C9000B0E08093B5169093B616A093B716B09364
:105CA000B8160F94D10282E00E94DEC620E030E0F8
:105CB00040E251E40F949A240F94962C7093BE16F0
:105CC0006093BD160093B1161093B4168CE490E166
:105CD000A0E0B0E08093B5169093B616A093B716E7
:105CE000B093B8160F94D10262E070E080E090E0CB
:105CF0000E94F2C681E09AE59093BE168093BD168D
:105D000087E490E0C5C78430910509F485C68530E5
:105D1000910549F44EE750E160E070E085E095E0E0
:105D20000F94800279C6069709F076C68CEC96E04F
:105D30009093C0098093BF098BE090E02BC28091C3
:105D40006D1690916E16019711F510923E0281E04A
:105D50009AE59093BE168093BD168FE390E09093E2
:105D6000C0168093BF1687E08093B11682E88093B7
:105D7000B41684E890E0A0E0B0E08093B51690936C
:105D8000B616A093B716B093B8160F94D1028091AF
:105D90006D1690916E16029709F03EC681E09AE565
:105DA0009093BE168093BD1680E490E077C9E09191
:105DB0006D16F0916E163197EB30F10508F0E4C1E5
:105DC0008827ED56FF4F8F4F0D94212B8091A514FE
:105DD00080FF5CC6869580FD5CC658C62DEC3CEC09
:105DE0004CEC5DE36091C9137091CA138091CB13A1
:105DF0009091CC130F942A2B6B017C0120E030E0B2
:105E000040EA51EC0F948A2D87FDC2C120E030E0BA
:105E100040EA51E4C701B6010F94342418160CF07F
:105E20003FC6B6C12DEC3CEC4CEC5DE36091C91370
:105E30007091CA138091CB139091CC130F94292B9E
:105E40006B017C0120E030E040EA51EC0F948A2D98
:105E500087FD9EC120E030E040EA51E4C701B60171
:105E60000F94342418160CF092C692C180E00F945F
:105E700013080E94E2C5811103C083E796E002C0C7
:105E800085E696E09093C0098093BF0982E08093F5
:105E9000B31281E09AE59093BE168093BD1684E517
:105EA00090E09093C0168093BF1687E08093B11660
:105EB00082E88093B41684E890E0A0E0B0E080939C
:105EC000B5169093B616A093B716B093B8160F9464
:105ED000D1025EC183E08093B31283E090E090939F
:105EE000BE168093BD1685E08093B11682E880933C
:105EF000B4168DE890E1A0E0B0E08093B5169093E1
:105F0000B616A093B716B093B8160F94D102E12C31
:105F1000F12C00E0DD24D394AA24A39445E0942E30
:105F200055E0852E62E8762EDD2031F0CC24C39436
:105F300035E0B32E10E005C0CC24CA94BB24BA943B
:105F400014E0DA24B116D1F1802F90E04897A4F53F
:105F50000F5FF701919EE00DF11D1124EE0FFF1F61
:105F6000EE0FFF1FE75CFB4E20E030E04AE754E411
:105F700060817181828193810F949A240F94962C71
:105F80007093BE166093BD168092B1167092B416CF
:105F9000802F90E08158974F880F991F092E000C91
:105FA000AA0BBB0B8093B5169093B616A093B716A9
:105FB000B093B8160F94D1021C0DC4CFBFEFEB1AEB
:105FC000FB0AE5E0EE16F10409F0AECF81E09AE5B8
:105FD0009093BE168093BD1685E590E09093C01611
:105FE0008093BF1687E08093B11682E88093B41641
:105FF00084E890E0A0E0B0E08093B5169093B616E8
:10600000A093B716B093B8160F94D10287E096E02C
:106010009093C0098093BF09BBC042E060E070E08C
:1060200080E890E40E9400C640E060E070E084E315
:1060300093E40E9400C641E060E070E084E393E4F2
:1060400013C042E060E070E080E890E40E9400C687
:1060500040E060E070E080E292E40E9400C641E02F
:1060600060E070E080E292E40E9400C686E08093E7
:10607000B3128EC042E060E070E080E890E40E94DD
:1060800000C640E060E070E080EA93E4E6CF42E0E2
:1060900060E070E080E890E40E9400C640E060E0CC
:1060A00070E080EA93E40CC042E060E070E080E8D9
:1060B00090E40E9400C640E060E070E080E292E47C
:1060C0000E9400C641E060E070E080EA93E4CCCF3B
:1060D0008091B61881111CC083E090E09093BE16A9
:1060E0008093BD1685E08093B11682E88093B41644
:1060F00085E490E1A0E0B0E08093B5169093B616E9
:10610000A093B716B093B8160F94D10281E01BC0CC
:1061100082E090E09093BE168093BD1685E0809358
:10612000B11682E88093B41685E490E1A0E0B0E077
:106130008093B5169093B616A093B716B093B81681
:106140000F94D10280E00F94130820E030E048EC77
:1061500052E46091C9137091CA138091CB1390914E
:10616000CC130F949A240F94962C7093BE166093C0
:10617000BD1685E08093B11682E88093B41686E25E
:1061800090E1A0E0B0E09BCE8BEE95E00E94C4537E
:106190008AE090E09093BE168093BD1685E08093D0
:1061A000B11682E88093B4164BC184E08093B31299
:1061B0008091651690916616A0916716B091681649
:1061C00060916D1670916E168834F0E19F07A105FD
:1061D000B10509F453C08A3420E19207A105B10545
:1061E00009F456C08C3430E19307A105B10509F4D8
:1061F0005AC086349041A105B10509F05EC06330F4
:106200007105B9F58AED95E09093C0098093BF09B7
:1062100081E08093D60880933E021092C60881E008
:106220009AE59093BE168093BD168AE490E0909311
:10623000C0168093BF1687E08093B11612E81093C2
:10624000B41684E890E0A0E0B0E08093B516909397
:10625000B616A093B716B093B8160F94D1028AE081
:1062600090E09093BE168093BD1685E08093B116A2
:10627000E5C06093D5081092B312CEC380E090E0E1
:10628000A4EBB3E48CA39DA3AEA3BFA3312C15C094
:1062900080E090E0A4EBB3E48CA39DA3AEA3BFA3E6
:1062A000332433940AC080E090E0A8ECB3E48CA3DC
:1062B0009DA3AEA3BFA382E0382E80E090E00F94B0
:1062C000392420E030E040E251E40F94242C6B01AB
:1062D0007C0120E030E0A9010F94342487FF09C03D
:1062E0001092C0081092C1081092C2081092C30800
:1062F0001FC02CA13DA14EA15FA1C701B6010F9403
:106300008A2D18164CF0C092C008D092C108E092B5
:10631000C208F092C3080CC08CA19DA1AEA1BFA180
:106320008093C0089093C108A093C208B093C3089B
:106330006091C0087091C1088091C2089091C30813
:10634000432D0E9400C661E070E080E090E00E9472
:10635000F2C680E00E94DEC620E030E040E251E478
:106360000F949A240F94962C7093BE166093BD16CA
:1063700005E00093B11612E81093B41688E490E19A
:10638000A0E0B0E08093B5169093B616A093B71630
:10639000B093B8160F94D10281E00E94DEC620E0CF
:1063A00030E040E251E40F949A240F94962C7093BD
:1063B000BE166093BD160093B1161093B4168AE40E
:1063C00090E1A0E0B0E08093B5169093B616A0934C
:1063D000B716B093B8160F94D10282E00E94DEC6C1
:1063E00020E030E040E251E40F949A240F94962C80
:1063F0007093BE166093BD160093B1161093B41639
:106400008CE490E1A0E0B0E08093B5169093B616CE
:10641000A093B716B093B8160F94D10261E070E064
:1064200080E090E00E94F2C61092B3128AE090E001
:106430009093BE168093BD160093B1161093B416B8
:1064400080E092E1A0E0B0E00C945C2880916516B9
:1064500090916616A0916716B09168168635E0E1B6
:106460009E07A105B10509F041C020E030E040E2FF
:1064700053E46091EE0B7091EF0B8091F00B9091D3
:10648000F10B0F94342420916D1630916E1687FF16
:106490000AC42530310508F006C480EA90E09093E4
:1064A000BE168093BD1685E08093B11612E8109356
:1064B000B41680E290E1A0E0B0E08093B51690932E
:1064C000B616A093B716B093B8160F94D10265E034
:1064D00070E080E090E00E94F2C681E09AE590933F
:1064E000BE168093BD1682E490E0D2C38435F0E1FD
:1064F0009F07A105B105B9F460916D1670916E16F4
:1065000080E090E00F94392420E030E040E251E454
:106510000F94242C6093C7087093C8088093C9080F
:106520009093CA0879C288359041A105B10509F058
:1065300073C260916D1670916E1680E090E00F94BA
:10654000392420E030E040E251E40F94242C6093A1
:10655000CB087093CC088093CD089093CE085CC292
:1065600060916D1670916E1684EC95E00F94440B5B
:1065700080916D1690916E1682309105A1F038F4DD
:10658000009771F00197E1F48EE295E043C2843008
:10659000910579F058F0059799F489E995E00BC0D9
:1065A00088E195E037C286EB95E005C08CEA95E07E
:1065B00002C087EA95E09093C0098093BF092CC27E
:1065C00082E495E027C281E595E00E94C453809162
:1065D0006D1690916E168130910519F46499C3C4BB
:1065E0001BC2892B09F018C28FE595E00E94C453A5
:1065F0008091BC08813039F585E795E00E94C4534D
:1066000081E09AE59093BE168093BD168EE290E0ED
:106610009093C0168093BF1687E08093B11682E8EE
:106620008093B41684E890E0A0E0B0E08093B516C3
:106630009093B616A093B716B093B8160F94D102E4
:106640001092B11235C0823069F489E895E00E9459
:10665000C45381E09AE59093BE168093BD1686E3FD
:1066600090E00EC0833031F58DE995E00E94C4536F
:1066700081E09AE59093BE168093BD1681E490E088
:106680009093C0168093BF1687E08093B11682E87E
:106690008093B41684E890E0A0E0B0E08093B51653
:1066A0009093B616A093B716B093B8160F94D10274
:1066B000109214141092BC080E9488F5ADC180910C
:1066C0006D1690916E168F3F910531F028F08FEF87
:1066D00090E0A0E0B0E002C0A0E0B0E0809306024D
:1066E00090930702A0930802B093090280910602DA
:1066F00090910702A0910802B09109020097A105AC
:10670000B10509F51092BE161092BD1605E0009372
:10671000B11612E81093B4168AE890E1A0E0B0E058
:106720008093B5169093B616A093B716B093B8168B
:106730000F94D10289E090E09093BE168093BD162D
:106740000093B1163DC00196A11DB11D05E0B6959F
:10675000A795979587950A95D1F70197A109B10952
:10676000009731E0A307B10550F0B093BE16A09397
:10677000BD169093C0168093BF1687E005C0909316
:10678000BE168093BD1685E08093B11612E8109373
:10679000B4168AE890E1A0E0B0E08093B51690933B
:1067A000B616A093B716B093B8160F94D10288E02E
:1067B00090E09093BE168093BD1685E08093B1164D
:1067C0001093B4168CE890E1A0E0B0E08093B51689
:1067D0009093B616A093B716B093B8160F94D10243
:1067E0008091060290910702A0910802B0910902DF
:1067F000BA2FA92F982F88270097E1E0AE07B1059F
:1068000050F0B093BE16A093BD169093C01680931F
:10681000BF1687E005C09093BE168093BD1685E035
:106820008093B11682E88093B41681EA90E0A0E0EC
:10683000B0E00C945C2881EB95E00E94C4530E9468
:1068400069C5409165165091661660916716709102
:106850006816882339F0433DF0E25F076105710552
:1068600009F4C7C3423D50426105710509F0D4C027
:1068700080916D1690916E16019709F00CC50E94DB
:1068800069C5882309F407C58091151B87FDC4C01D
:10689000A2E18A02C00111248053934E0E94FF5D41
:1068A000C12C90E2D92EE12CF12C05E012E81092D7
:1068B000BE161092BD160093B1161093B416C09276
:1068C000B516D092B616E092B716F092B8160F949D
:1068D000D102BFEFCB1ADB0AEB0AFB0AEAE0CE16C5
:1068E000E0E2DE06E104F10411F70091151BF2E18C
:1068F0000F02800111240859144EF8010190002064
:10690000E9F7C8018E1B9F0B439697FD01967C010A
:10691000F594E7941E141F040CF0C6C49E012F5F6B
:106920003F4F690184E1D9011D928A95E9F7A701DA
:1069300062EC75E0C9010F949D2EB801C6018E0D61
:106940009F1D0F94882E40E050E260E070E0C60189
:106950000F94800262E070E080E090E00E94F2C656
:1069600040E060E070E08FE793E40E94EFF541E0E3
:1069700060E070E08FE793E40E94EFF5109205026B
:106980008DE090E09093BE168093BD1685E08093D5
:10699000B11612E81093B41684E190E1A0E0B0E0E3
:1069A0008093B5169093B616A093B716B093B81609
:1069B0000F94D10262E070E080E090E00E94F2C6A5
:1069C00081E09AE59093BE168093BD1685E390E032
:1069D0009093C0168093BF1687E08093B1161093F2
:1069E000B41684E890E0A0E0B0E08093B5169093F0
:1069F000B616A093B716B093B8160F94D10281E0E3
:106A000080933E028093B11283E08093B21204C05F
:106A10008EE895E00E94C45380E5E1E6F6E1DF01EF
:106A20001D928A95E9F78AE58093621685EA80933C
:106A300063160C94552187EA94E10E940D5CF701DE
:106A4000EF5FF84E8083809101178A3581F01E1424
:106A50001F0414F00C947422D601E02F1D92EA95C5
:106A6000E9F71092C5081092C4080C94742262E0F1
:106A700070E080E090E00E94F2C6FFEFEF1AFF0A9C
:106A8000F092C508E092C4080C9474228CEB96E056
:106A900002C08BEA96E09093C0098093BF0955CB62
:106AA00088E290E00F94C6052DEC3CEC4CEC5DE3E5
:106AB0006091C9137091CA138091CB139091CC133C
:106AC0000F942A2B6B017C0120E030E040EA51EC6E
:106AD0000F948A2D87FD12C020E030E040EA51E497
:106AE000C701B6010F943424181644F0C092C9139C
:106AF000D092CA13E092CB13F092CC1320E030E096
:106B000048EC52E46091C9137091CA138091CB1381
:106B10009091CC130F949A240F94962C7093BE16D8
:106B20006093BD1685E08093B11682E88093B41619
:106B300086E290E1A0E0B0E08093B5169093B6169F
:106B4000A093B716B093B8160F94D1026091C913F1
:106B50007091CA138091CB139091CC138E010B5E70
:106B60001F4F23E041E00F940C1F9F938F938DE9FB
:106B700096E09F938F93045111091F930F930F94E5
:106B8000CC23C8010E94CCC788E996E076C088ED86
:106B90009FEF0F94C6052DEC3CEC4CEC5DE360914F
:106BA000C9137091CA138091CB139091CC130F9499
:106BB000292B6B017C0120E030E040EA51EC0F947E
:106BC0008A2D87FD12C020E030E040EA51E4C70181
:106BD000B6010F943424181644F0C092C913D09211
:106BE000CA13E092CB13F092CC1320E030E048ECD3
:106BF00052E46091C9137091CA138091CB139091A4
:106C0000CC130F949A240F94962C7093BE16609315
:106C1000BD1685E08093B11682E88093B41686E2B3
:106C200090E1A0E0B0E08093B5169093B616A093E3
:106C3000B716B093B8160F94D1026091C913709132
:106C4000CA138091CB139091CC138E010B5E1F4F12
:106C500023E041E00F940C1F9F938F938AE896E006
:106C60009F938F93045111091F930F930F94CC237B
:106C7000C8010E94CCC785E896E09093C009809334
:106C8000BF090F900F900F900F900F900F9080CA38
:106C90009093C0168093BF1687E08093B11610932F
:106CA000B4160C9458282430310589F481E00F94EF
:106CB000F61D2091CB083091CC084091CD08509121
:106CC000CE080F942A2B41E00F94CD1DB2C0253081
:106CD000310508F4F4C02630310509F431C108F05B
:106CE00023C181E08093CF0840E060E070E08EE354
:106CF00093E40E9475C520E030E048EC52E46091D6
:106D0000EE0B7091EF0B8091F00B9091F10B0F94C3
:106D10009A246B017C016091F20B7091F30B072EAA
:106D2000000C880B990B0F943B249B01AC01C7010D
:106D3000B6010F94242C0F949D2C6436710510F02D
:106D400064E670E07093BE166093BD1605E0009394
:106D5000B11612E81093B41684E290E1A0E0B0E01E
:106D60008093B5169093B616A093B716B093B81645
:106D70000F94D1026091EE0B7091EF0B8091F00BAC
:106D80009091F10B0F94962C7093BE166093BD16E4
:106D90000093B1161093B41686E390E1A0E0B0E042
:106DA0008093B5169093B616A093B716B093B81605
:106DB0000F94D1028091F20B9091F30B9093BE1639
:106DC0008093BD160093B1161093B41684E390E13E
:106DD000A0E0B0E08093B5169093B616A093B716D6
:106DE000B093B8160F94D10265E070E080E090E0B7
:106DF0000E94F2C681E09AE59093BE168093BD167C
:106E000084E490E09093C0168093BF1687E080934F
:106E1000B1161093B41684E890E0A0E0B0E080933F
:106E2000B5169093B616A093B716B093B8160F94F4
:106E3000D10220E030E040E251E46091C708709157
:106E4000C8088091C9089091CA080F949A240F9499
:106E5000962C7093BE166093BD1605E00093B11694
:106E600012E81093B41684E590E1A0E0B0E08093BE
:106E7000B5169093B616A093B716B093B8160F94A4
:106E8000D10220E030E040E251E46091CB08709103
:106E9000CC088091CD089091CE080F949A240F943D
:106EA000962C7093BE166093BD160093B116109386
:106EB000B41688E590E1A0E0B0E00C945C282230A4
:106EC000310579F480E00F94F61D2091C7083091C8
:106ED000C8084091C9085091CA080F942A2B40E075
:106EE000F3CE2330310570F081E00F94F61D209130
:106EF000CB083091CC084091CD085091CE080F942A
:106F0000292BE1CE2130310509F093CF80E00F9499
:106F1000F61D2091C7083091C8084091C9085091CA
:106F2000CA080F94292BDBCF213F310509F081CF0F
:106F30001092CF0861E070E080E090E00E94F2C61D
:106F400081E09AE59093BE168093BD1681E490E0AF
:106F50009093C0168093BF1687E08093B11682E8A5
:106F60008093B41658CF8FE096E00E94C45381E01E
:106F70000E948B8D8DE090E09093BE168093BD169D
:106F800085E08093B11612E81093B41684E190E185
:106F9000A0E0B0E08093B5169093B616A093B71614
:106FA000B093B8160F94D10283E08093B21281E0BF
:106FB0009AE59093BE168093BD1685E390E090937A
:106FC000C0168093BF1687E08093B1161093B41655
:106FD00084E890E0A0E0B0E08093B5169093B616F8
:106FE000A093B716B093B8160F94D1021092BC08B4
:106FF00013CD87E296E00E94C4538091161B9091B6
:10700000171B992720916D1630916E1682179307E2
:1070100008F402CD8AEB95E00E94C45380916D166E
:1070200081508093151BA4ED8A2EA0E29A2EA12CEC
:10703000B12C05E012E81092BE161092BD16009316
:10704000B1161093B4168092B5169092B616A0920F
:10705000B716B092B8160F94D1022FEF821A920A87
:10706000A20AB20A3EED831630E29306A104B104EF
:1070700011F78091151BA2E18A02C0011124FC01C5
:10708000E859F44E7F0101900020E9F7C7018E1BFB
:107090009F0B439697FD01968C0115950795101649
:1070A0001106FCF49E012F5F3F4F690184E1D90175
:1070B0001D928A95E9F7A80162EC75E0C9010F9469
:1070C0009D2EB701C601800F911F0F94882E44EDAD
:1070D00050E260E070E0C6010F94800205E012E823
:1070E00006C044ED50E260E070E0C701F5CF1092B9
:1070F000BE161092BD160093B1161093B41680926E
:10710000B5169092B616A092B716B092B8160F9414
:10711000D102BFEF8B1A9B0AAB0ABB0AE6EE8E16B2
:10712000E0E29E06A104B10411F78E010F5F1F4F2C
:1071300084E1D8011D928A95E9F78091171B8F93FE
:107140008091161B8F9380916E168F9380916D1690
:107150008F938CEC95E09F938F931F930F930F94D5
:10716000B72E4EED50E260E070E0C8010F9480024F
:1071700062E070E080E090E00E94F2C60FB6F89402
:10718000DEBF0FBECDBF31E2C32E32E1D32EE12CE4
:10719000F12C43E1442E40E6542E612C712C8824BE
:1071A0008394912CAA24AA94BA2C75E0272EE2E8A5
:1071B0003E2E0AE010E08091161B9091171B881557
:1071C000990594F1B092BE16A092BD162092B11608
:1071D0003092B4164092B5165092B6166092B71619
:1071E0007092B8160F94D1021093BE160093BD167C
:1071F0002092B1163092B416C092B516D092B6163F
:10720000E092B716F092B8160F94D102FFEF8F1AE2
:107210009F0A20E1420E511C611C711C3FEFC31AF2
:10722000D30AE30AF30AC7CF80916D1690916E16C8
:1072300024E0880F991F2A95E1F78D5F9F49A0E010
:10724000B0E020EF37E83093BE162093BD1605E07E
:107250000093B11612E81093B4168093B51690936C
:10726000B616A093B716B093B8160F94D1028091BA
:107270006D1690916E16805E9D4EA0E0B0E026E007
:1072800030E03093BE162093BD160093B1161093D4
:10729000B4160C945C2880916D1690916E16892B13
:1072A00011F40C946F2BB8CB40E050E260E070E03A
:1072B000C8014ECBE3960FB6F894DEBF0FBECDBF2C
:1072C000DF91CF911F910F91FF90EF90DF90CF90C2
:1072D000BF90AF909F908F907F906F905F904F90F6
:1072E0003F902F9008952F923F924F925F926F920E
:1072F0007F928F929F92AF92BF92CF92DF92EF9246
:10730000FF920F931F93CF93DF93CDB7DEB7C15496
:10731000D1090FB6F894DEBF0FBECDBF22968FAF56
:10732000229720916F122CAF21E020936F12809151
:1073300090128D3409F4B3C4843511F40C94A44B29
:10734000873411F00C94AB4B80918E1290918F1278
:107350008B31910509F420C2B4F48430910534F4E2
:1073600082309105E4F597FF2EC095C485319105D3
:1073700011F40C94AD4B8A31910509F409C20497BC
:1073800009F089C4C6C18A32910509F4B5C34CF429
:107390008D319105B1F00CF429C24E9709F465C204
:1073A0007AC48B35910509F425C38C35910509F410
:1073B00025C38A35910509F06EC41092EF080C942C
:1073C000AD4B14E03FC280918702882311F40C94E6
:1073D000AD4B0E9456E10E941FDB0C94AD4B2091F7
:1073E0008702222311F40C94AD4B11E0029709F0AF
:1073F00010E00E9456E119821A821B821C821D82B3
:107400001E821F82188682E50E940D8D882309F452
:1074100038C10E948D8C4B015C0120E030E0A90155
:107420000F943424882309F442C18091770290910B
:107430007802A0917902B0917A028CA39DA3AEA3A9
:10744000BFA380917B0290917C02A0917D02B091BC
:107450007E0288A799A7AAA7BBA78091A5139091A0
:10746000A613A091A713B091A8138CA79DA7AEA7B0
:10747000BFA78091A9139091AA13A091AB13B091CB
:10748000AC1388AB99ABAAABBBAB2CA53DA54EA565
:107490005FA56CA17DA18EA19FA10F9434248111C1
:1074A0000DC028A939A94AA95BA968A579A58AA50B
:1074B0009BA50F943424882309F4F9C020E030E020
:1074C000A901C501B4010F943424881F8827881F9F
:1074D000181729F080E090E0A0E8BFEB04C080E03E
:1074E00090E0A0E8BFE388AF99AFAAAFBBAF2CA1F3
:1074F0003DA14EA15FA16CA57DA58EA59FA50F9472
:10750000292B6CAB7DAB8EAB9FAB28A539A54AA5CB
:107510005BA568A979A98AA99BA90F94292B6B015E
:107520007C012CA93DA94EA95FA9CA01B9010F94FC
:107530009A242B013C01A7019601C701B6010F94C3
:107540009A249B01AC01C301B2010F942A2B0F9422
:10755000D82D2B013C019B01AC0160E070E080E87C
:107560009FE30F94242C21966CAF7DAF8EAF9FAF1D
:10757000219720E030E040E05FE3C301B2010F94C7
:107580009A242B013C01A5019401C501B4010F947B
:107590009A244B015C01A3019201C301B2010F9433
:1075A0009A249B01AC01C501B4010F94292B0F94BF
:1075B000D82D28AD39AD4AAD5BAD0F949A244B015F
:1075C0005C01C701B601905821962CAD3DAD4EAD82
:1075D0005FAD21970F949A24A50194010F949A24EA
:1075E0006B017C012CA53DA54EA55FA56CA17DA1DD
:1075F0008EA19FA10F942A2B20E030E040E05FE3B2
:107600000F949A249B01AC01C701B6010F942A2B59
:107610002CA13DA14EA15FA10F94292B69837A83F0
:107620008B839C8328A939A94AA95BA968A579A558
:107630008AA59BA50F942A2B20E030E040E05FE371
:107640000F949A246B017C0121962CAD3DAD4EAD7B
:107650005FAD21976CA97DA98EA99FA90F949A244B
:10766000A50194010F949A249B01AC01C701B601B6
:107670000F942A2B28A539A54AA55BA50F94292B81
:1076800012C089E40E940D8D882331F00E948D8CF8
:1076900069837A838B839C838AE40E940D8D88237F
:1076A00031F00E948D8C6D837E838F83988720E0DC
:1076B00030E0A90169817A818B819C810F94342407
:1076C00081110BC020E030E0A9016D817E818F81A6
:1076D00098850F9434248823A1F0412FBE016F5F59
:1076E0007F4F85EA93E10E949DB50E94F1EE609381
:1076F0009D1470939E1480939F149093A0140C94E7
:10770000AD4B0F94820B8CE797E00F949D0A0C947D
:10771000AD4B80E50E940D8D882329F00E94B5A411
:107720006B017C0103C0C12CD12C760183E50E9442
:107730000D8D882361F00E948D8C20E030E04AE7B7
:1077400054E40F949A240F949D2C6B017C010E94A9
:107750001CBF8091CE13811105C060E082E997E0E3
:107760000E9449F50E94F1EEC60ED71EE81EF91ED2
:107770000E94F1EEDC01CB018C199D09AE09BF0915
:10778000B7FD02C00C94AD4B80E00E94E553F0CFF2
:107790000E94BBA90C94AD4B0E9497E881110C94F8
:1077A000AD4B80E090E0A8E4B2E489839A83AB8398
:1077B000BC8380E090E0A0E2B1E48D839E83AF8340
:1077C000B88789879A87AB87BC8780E50E940D8D33
:1077D000882321F00E94558C862F01C080E0BE01D5
:1077E0006F5F7F4F0E9481F40C94AD4B8091CD135D
:1077F0008770873011F00C94D14B60E08FE40E94C9
:107800001A8D81110C94AD4B0C94D14B8091B6180C
:1078100081111DC00E941B848823F9F0115011F4BE
:107820000C94BB4D40E050E060E078E085E00E94C1
:10783000E98D61E083EF97E00E942F8D8BED97E05B
:107840000E9480BB0E9497E8882301F306C060E095
:107850008FE40E941A8D8823E9F20E94538D8EE9ED
:1078600098E00E9480BB0C94AD4B2091C1133091E5
:10787000C2134091C3135091C41360917702709169
:1078800078028091790290917A020F942A2BAB01B1
:10789000BC0188E50E943BC86C8F7D8F8E8F9F8FC7
:1078A0002091C5133091C6134091C7135091C8134E
:1078B00060917B0270917C0280917D0290917E02AA
:1078C0000F942A2BAB01BC0189E50E943BC8698358
:1078D0007A838B839C83BE016F5F7F4FCE014C9672
:1078E0000E94ACA5882311F40C94AD4B80E00F945A
:1078F00013080E9403DE61E085E40E941A8D182FB0
:1079000021E0482FBE016F5F7F4FCE014C960E9451
:1079100046E96B017C019B01AC010F941C2E811187
:107920005FC08C8C9D8CAE8CBF8C20E030E0A901B8
:10793000C501B4010F94342487FF05C027E137EB5C
:1079400041E558EB04C027E137EB41E558E3C501B9
:10795000B4010F942A2BAB01BC0180EC98E00F948A
:10796000510B89809A80AB80BC8020E030E0A90177
:10797000C501B4010F94342487FF05C027E137EB1C
:1079800041E558EB04C027E137EB41E558E3C50179
:10799000B4010F942A2BAB01BC018BEB98E00F9440
:1079A000510B20E030E0A901C701B6010F94342447
:1079B00087FF05C027E137EB41E558EB04C027E11D
:1079C00037EB41E558E3C701B6010F942A2BAB0111
:1079D000BC0186EB98E00F94510B8AE00E94B952EB
:1079E0000E94EADD113011F40E94B39C0E94B0DFC6
:1079F0000C94AD4B2093EF080C94AD4B95E0292EE1
:107A000093E0392E21E9E22E22E1F22E27E732E03F
:107A10003DA32CA335EBC32E33E1D32E00E010E0C1
:107A2000D1018D911D010E940D8D882309F44BC059
:107A30000E948D8C2B013C01133049F0F60120810E
:107A40003181428153810F94292B2B013C01ACA140
:107A5000BDA12D913D914D915C91C301B2010F9457
:107A6000292B4B015C012DEB37E346E855EB0F94D6
:107A70008A2D87FD0AC02DEB37E346E855E3C501A3
:107A8000B4010F9434241816F4F4133051F44092D6
:107A9000830250928402609285027092860201E015
:107AA00012C0A5019401F7016081718182819381E7
:107AB0000F942A2BD7016D937D938D939C931397ED
:107AC000812F0E9449C51F5FB4E0EB0EF11CECA1B1
:107AD000FDA13496FDA3ECA3F4E0CF0ED11C14302D
:107AE00009F09ECF002321F083E892E00E942DBF91
:107AF0000E94B0DF0C94AD4B80918702882311F473
:107B00000C94AD4B89E40E940D8D082F882321F041
:107B10000E94898CE82E01C0E12C8AE40E940D8D20
:107B2000182F882321F00E94898CF82E01C0F12C97
:107B3000002319F024E02E1528F0112349F034E039
:107B40003F1530F488EC98E00F949D0A0C94AD4BEF
:107B50000E944B8C0023F1F020912D1430912E14B3
:107B60004E2D4203B001439F700D112480912314C8
:107B700090912414680F791F072E000C880B990B25
:107B80000F943B246093A5137093A6138093A713BF
:107B90009093A8131123F1F020912F1430913014F9
:107BA0004F2D4203B001439F700D11248091251485
:107BB00090912614680F791F072E000C880B990BE3
:107BC0000F943B246093A9137093AA138093AB1373
:107BD0009093AC1360E080E50E941A8D8823C1F178
:107BE0000023D1F02091C1133091C2134091C313EF
:107BF0005091C4136091A5137091A6138091A7139F
:107C00009091A8130F94292B6093A5137093A6133A
:107C10008093A7139093A8131123D1F02091C5133B
:107C20003091C6134091C7135091C8136091A913A6
:107C30007091AA138091AB139091AC130F94292BE0
:107C40006093A9137093AA138093AB139093AC1312
:107C500040E050E0BA0186E40E943BC86B017C0121
:107C600020E030E0A9010F948A2D181684F420E05A
:107C700030E040E752E4C701B6010F94242C609332
:107C800065027093660280936702909368020E9477
:107C90001FDB0C94AD4B0E94737F0C94AD4B809115
:107CA0008E1290918F128537910509F4B6C70CF0AA
:107CB00053C18934910509F494C40CF06CC08A3125
:107CC000910509F419C3B4F58431910509F48EC204
:107CD00094F48131910509F468C244F4029710F0DC
:107CE0000C94A14B0E9463B90C94AD4B429709F4DC
:107CF000C2C60C94A14B8731910509F4A1C28CF442
:107D00008531910509F498C2469711F00C94A14B66
:107D10000E94E65D80913918877F809339180C9412
:107D2000AD4B8831910509F4A3C2499709F4D9C232
:107D30000C94A14B8F31910509F40CC47CF48C3167
:107D4000910509F451C30CF4E5C28D31910509F494
:107D500055C34E9709F459C30C94A14B8A3291052F
:107D600009F418C464F48032910509F4ADC3819715
:107D700011F00C94A14B0E94AACE0C94AD4B8B3207
:107D8000910509F42AC4C09711F00C94A14B0E94EC
:107D9000817F0C94AD4B8836910509F4CBC4D4F5A2
:107DA0008135910509F44FC6C4F48C34910509F46A
:107DB00027C44CF48B34910511F00C94A14B0E9414
:107DC000E7BC0C94AD4B8D34910509F41DC48E3481
:107DD000910509F41DC40C94A14B8435910509F457
:107DE0004AC674F48235910509F442C6833591057B
:107DF00011F00C94A14B81E08093E9080C94AD4BF9
:107E00008535910509F463C68C35910509F478C66A
:107E10000C94A14B8E36910509F40BC5D4F48B3626
:107E2000910509F400C654F48936910509F49DC5FD
:107E30008A36910509F4CFC50C94A14B8C36910577
:107E400011F40C94AD4B8D36910509F497C40C9444
:107E5000A14B8137910509F442C55CF48F36910539
:107E600009F4F8C48037910511F40C94AD4B0C94CF
:107E7000A14B8237910509F4CDC68337910511F0E6
:107E80000C94A14B8AE49BE00F949D0A60E08AE386
:107E90009BE00E94F4B960E085E29BE00E94F4B9A7
:107EA00061E08EE19BE00E94F4B961E083E19BE038
:107EB0000E94F4B961E083E09BE00E94F4B960E0C5
:107EC0008AEF9AE00E94F4B961E080EF9AE00E94A4
:107ED000F4B961E086EE9AE00E94F4B961E08EEDBB
:107EE0009AE00E94F4B961E080ED9AE00E94F4B952
:107EF00061E082EC9AE00E94F4B960E083EB9AE0E2
:107F00000E94F4B960E085EA9AE00E94F4B960E06A
:107F10008FE89AE00E94F4B961E08EE79AE00E944F
:107F2000F4B961E08FE69AE00E94F4B961E08AE575
:107F30009AE00E94F4B961E087E49AE00E94F4B903
:107F400060E08AE39AE00E94F4B960E086E29AE099
:107F50000E94F4B90C94AD4B8F32A1E09A0711F452
:107F60000C94A5490CF079C08B3C910509F41EC70F
:107F7000ACF58D37910509F463C5BCF487379105DD
:107F800009F496C60CF45AC68837910509F493C6CD
:107F90008937910511F00C94A14B1092AF09109202
:107FA000AE090E943DE10C94AD4B8E3B910509F466
:107FB000CAC454F48C38910509F4B3C48B399105C3
:107FC00009F4E3C40C94A14B883C910509F47BC6E9
:107FD000893C910509F4C4C60C94A14B8D3D9105D3
:107FE00009F438C7E4F48E3C910509F401C76CF438
:107FF0008C3C910509F4F9C68D3C910511F00C9467
:10800000A14B0E94C5A40C94AD4B833D910509F48E
:1080100011C78C3D910509F410C70C94A14B823215
:10802000E1E09E0711F40C94634854F4823E9105FC
:1080300009F466C78831914009F4AEC70C94A14B8E
:108040008D3231E0930711F40C946E488E329140DA
:1080500011F40C9461490C94A14B853FA1E09A075F
:1080600011F40C94BC4A0CF04EC08A39E1E09E0732
:1080700011F40C94AD4B14F5803921E0920711F402
:108080000C94A8493CF48033914011F40C94EE48D0
:108090000C94A14B8139A1E09A0711F40C94AB49DF
:1080A0008239914011F00C94A14B80E00E94FB9C1E
:1080B0000E94B39C0E94B0DF0C94AD4B853AE1E086
:1080C0009E0711F40C94BC497CF48C3921E0920792
:1080D00011F40C94B149843A914011F00C94A14BE5
:1080E0000E94FCA60C94AD4B8C3A41E0940711F42D
:1080F0000C942C4A843F914011F00C94A14B0E94A7
:10810000FDEE0C94AD4B8B35B2E09B0711F40C9453
:10811000DE4A5CF5883FF1E09F0711F40C94C24AF7
:10812000ACF4863F31E0930711F40C94BF4A873FCB
:10813000914011F00C94A14B61E083E50E941A8DEF
:1081400091E089270E9434FE0C94AD4B8C30A2E064
:108150009A0711F40C94D34A8835924011F00C948C
:10816000A14B0E942EE20C94AD4B8438E3E09E07B5
:1081700011F40C94574B6CF4833523E0920711F4FF
:108180000C94DB4A8C36934011F40C94AD4B0C9458
:10819000A14B803A43E0940709F4CCC1873E934059
:1081A00011F40C94934B0C94A14B80918A1284FF90
:1081B00002C00C94CD4D80918C1287FF02C00C94AC
:1081C000CD4D80918D12837011F00C94CD4D60E0F7
:1081D00087EE98E00E9449F55F988A98809108019F
:1081E00081708093060112980C94AD4B8FEF98E04C
:1081F0000F949D0A1092B30B8DE995E10E948C6655
:108200008BE1EDE9F5E1DE01119601900D928A9581
:10821000E1F740E050E0BE016F5F7F4F80E090E00B
:108220000E946C5FCE0101960E94C26780EF98E0C9
:108230000F949D0A0C94AD4B0E94575E0C94AD4B6D
:10824000E0914513F09146138081882329F0803214
:1082500009F410823196F8CF40E061E08091451337
:10826000909146130E944261109215140C94AD4BEC
:108270008091450B8823E9F080E090E0A0EAB1E42A
:1082800088A399A3AAA3BBA31C8E1D8E1E8E1F8E2E
:1082900019821A821B821C8220E0AE01405E5F4F71
:1082A000BE01645E7F4FCE0101960E94A98E0C94A0
:1082B000AD4B0E9487CF882321F00E94F75D0E947A
:1082C000E7BC40E050E060E179E085E00E94A28EEA
:1082D00061E089EC94E30E942F8D0E94CDF50C940F
:1082E000AD4B8091391882FF03C08B7F8093391882
:1082F0000E9435E30C94AD4B8091391883FD02C088
:108300000C94AD4B83E50E940D8D81110C94E94DC9
:108310000C94AD4B83E40E94C48C8823D9F184E291
:1083200099E00F949D0A80914715882351F1BE0171
:108330006F5F7F4F84E495E10E9453658E010F5F6C
:108340001F4FF80181918F01882319F00E94B952C3
:10835000F8CFBE016F5F7F4F80E090E00E940A611E
:108360008091C61A882389F080E20E94B95206ECF7
:108370001AE1D8018D918D01882339F00E94B952FC
:10838000F8CF8AE199E00F949D0A8AE00E94B952E1
:108390000C94AD4B83E50E940D8D882309F10E945A
:1083A000658C182F90E0CD970CF01CE31093E0083B
:1083B0000E94F1EE6B017C01212F30E0A8EEB3E0CA
:1083C0000F94DE2AC60ED71EE81EF91EC092DC08E6
:1083D000D092DD08E092DE08F092DF080C94AD4BFD
:1083E0000E94BF5D0C94AD4B40E060E0809145136E
:1083F000909146130E9442610C94AD4B80913918C4
:108400008E7F809339180C94AD4B8091391883FD81
:1084100002C00C94AD4B0E942BEB8091391883FD68
:1084200002C00C94AD4B6091451370914613CE0180
:108430004C960F94DE048C01009711F40C94AD4B14
:108440006C8D7D8D19821C8222E0AC01CE010196DB
:108450000E94A56B811102C0F12C14C0CE010196BF
:108460000F944C048823C1F361E0CE0101960E9471
:108470003765009789F325EEFC0120831C820E945A
:108480004667F82ECE0101960E94C267B801FF2010
:1084900089F08EE499E00F946F0B8AE00E94B95244
:1084A000109235181092361810923718109238180A
:1084B0000C94AD4B86E399E00F946F0B83E399E046
:1084C0000F949D0A0C94AD4B8091391882FD0E9447
:1084D0001CBF8091391883FD02C00C94AD4B60E045
:1084E00080E50E941A8D182F482F61E08091451376
:1084F000909146130E94426183E50E940D8D88236E
:1085000081F00E94558CAB01BC014093351850930B
:108510003618609337187093381884E495E10E94F8
:108520004D640E94F75D11110C94AD4B0E94E7BCA5
:108530000C94AD4B2091451330914613909139180E
:1085400092609093391840E060E0C9010E94426156
:108550000C94AD4B0E94F9F36C8F7D8F8E8F9F8FA3
:10856000BE016F5F7F4FCE014C960E94CECD60E082
:10857000CE0101960E94A4F50F94860BBE016F5F99
:108580007F4F8CE599E00F946F0B8AE00E94B952FF
:108590000C94AD4B83E50E940D8D882311F40C944F
:1085A000AD4B0E94658CF82E6DE070E080E50E9476
:1085B000E1A68C0197FF02C00C94AD4BE82E60E061
:1085C00089E40E941A8D81110C94FA4D802F0E942B
:1085D0002A508111B2C40C94FA4D0E94F3E40C9419
:1085E000AD4B80E50E94C48C882311F40C94AD4BF4
:1085F0008091391882FF02C00C94AD4B0C94134E3D
:108600000E9448F40C94AD4B0E9497BD0C94AD4B66
:1086100060E070E083E50E94E1A68E34910531F4BC
:108620000E9452BE0E94CDF50C94AD4B87EC99E0B0
:108630000F949D0A60919E0970919F098EEB99E0BD
:108640000F94440B6091A0097091A10981EB99E00E
:108650000F94440B60919E0970919F098091A0092D
:108660009091A109681B790B8091B812815021E08B
:1086700030E0823010F020E030E0621B730B86EABD
:1086800099E00F94440B8AE00E94B9528EE999E078
:108690000F949D0A8091A2099091A309A091A40929
:1086A000B091A5098C8F9D8FAE8FBF8FBE016F5F7C
:1086B0007F4FCE014C960E94CECDBE016F5F7F4FA3
:1086C00081E999E00F946F0B8091A6099091A70919
:1086D000A091A809B091A9098C8F9D8FAE8FBF8FF3
:1086E000BE016F5F7F4FCE014C960E94CECDBE0182
:1086F0006F5F7F4F81E899E00F946F0B20E030E0CF
:108700004AE754E46091AA097091AB098091AC09E1
:108710009091AD090F94242CAB01BC0189E699E03E
:108720000F94510B8DE60E94B9528AE00E94B95213
:108730000C94AD4B8091371183FF02C00C94AD4B6C
:108740000E9405E287FF02C00C94AD4B83E50E94B6
:108750000D8D882379F00E948D8C0F94962C8B01BF
:10876000CB010E94ECD70135110524F40E9497BD7E
:108770000E94CDF50F949D1D0C94AD4B8091371147
:1087800083FF02C00C94AD4B0E9405E2F82E87FFD8
:1087900002C00C94AD4B83E50E940D8D082F811112
:1087A00006C082E50E940D8D182F8823C1F10E941A
:1087B0008D8C0F94962CCB010E94ECD70E948D8C4F
:1087C00020E030E040EA52E40F943424181614F408
:1087D0000C941E4E0E9497BD0E94CDF56091F20B45
:1087E0007091F30B072E000C880B990B0F943B2410
:1087F0004B015C014090EE0B5090EF0B6090F00B42
:108800007090F10BA30192010F948A2D181614F4A5
:108810000C94314E002311F40C94224E11E00F946D
:108820009D1D112309F499C7602F8F2D0E94FBD144
:1088300094C78EE40E940D8D882309F48EC70E9490
:10884000558C60934113709342138093431390931C
:10885000441383C783E50E94C48C882331F060E011
:1088600083E50E94F0A6809337110F94860B87EF63
:1088700099E00F949D0A80913711882369F18DEE5C
:10888000E82E89E0F82E00E010E020E0809137111A
:1088900090E0A0E0B0E0002E04C0B695A7959795B3
:1088A00087950A94D2F780FF0EC0DD24D394D20EB0
:1088B000222319F08CE20E94B952F701859194911C
:1088C0000F949D0A2D2D0F5F1F4FF2E0EF0EF11C4C
:1088D00005301105D9F659CD89EE99E054CD83E5DF
:1088E0000E940D8D882371F00E94658C282F30E046
:1088F0002D3331051CF4809300022FC78CE3809345
:1089000000022BC70F94860B4091000250E060E0FC
:1089100070E08EEF99E00F94330B8AE00E94B95219
:108920001CC78091371183FD18C783E50E940D8D08
:10893000882309F412C70E948D8C0F94962CCB01CA
:108940000E943D8C0AC78091371183FD06C783E5DD
:108950000E940D8D182F81110C94344E82E50E94D7
:108960000D8D81110C94344EF8C60E9405E2182F2B
:1089700087FDFAC683E29AE00F949D0A812F0E9438
:108980000BD08AE00E94B952EFC683E50E940D8D9C
:10899000882309F4E2C60E94658C182F90E0CD97D9
:1089A0000CF01CE31093E5080E94F1EE6B017C01D2
:1089B000212F30E0A8EEB3E00F94DE2AC60ED71EBA
:1089C000E81EF91EC092E108D092E208E092E308A6
:1089D000F092E408C2C660E080E50E94F0A6F82E9E
:1089E00031E0381708F4B9C681E40E94C48C8823AA
:1089F00021F06091D70B062F02C00FEF10E083E546
:108A00000E940D8D882349F00E94558C8B016F3F89
:108A1000710519F010F00FEF10E0EF2DF0E0E952C2
:108A2000F44F00839AC660E080E50E94F0A6823091
:108A300008F093C6E82FF0E0E952F44F10828DC69B
:108A40000E9435E38AC60E94FDD70E9497BD0E940E
:108A5000B0C00E946C501092121410921114109217
:108A6000101468EE73E080E090E00F946E0A75C613
:108A70001092E90872C683E50E940D8D882399F053
:108A80000E948D8C20E030E04AE754E40F949A2451
:108A90000F949D2C60930102709302028093030255
:108AA000909304025AC680918A1284FF02C00C94EB
:108AB000694E80918C1287FF02C00C94694E8091A0
:108AC0008D12837011F00C94694E0C949A4E83E5CC
:108AD0000E94C48C882309F440C60E948D8C20E03B
:108AE00030E04AE754E40F949A240F949D2C60934D
:108AF000EA087093EB088093EC089093ED082DC67C
:108B00000E9405E287FD29C690918A1294FD04C057
:108B100090918C1297FF0AC015E0C12E13E0D12E60
:108B200008E3E02E01E1F02E10E009C090918D12D3
:108B3000937091F7682F81E00E94B8E40EC6D601C9
:108B40008D916D010E940D8D882309F459C0133059
:108B500009F04FC00E948D8C4B015C0120E030E099
:108B600040EA51E40F94342487FF3AC0A5019401F0
:108B7000609158117091591180915A1190915B1127
:108B80000F94242C2B013C019B01AC0160916811D6
:108B90007091691180916A1190916B110F949A24D0
:108BA000609368117093691180936A1190936B11AF
:108BB0006091CB0B7091CC0B8091CD0B9091CE0B33
:108BC0000F943924A30192010F949A240F949D2CA1
:108BD0006093CB0B7093CC0B8093CD0B9093CE0B0B
:108BE0008092581190925911A0925A11B0925B1133
:108BF00007C00E948D8CF701648B758B868B978BD9
:108C00001F5FF4E0EF0EF11C143009F098CF0E94C2
:108C1000F8BEA3C50E940EBAA0C5809145139091DD
:108C20004613009741F0DC012C91222321F060E0F3
:108C30000E94A4F592C50E94CDF58FC50091451301
:108C40001091461394E0F12C40E0915021F1F8018D
:108C50008081282F2B7F213421F421812133D9F4E5
:108C600007C08035C1F4818180538A3048F013C039
:108C7000813421F0853421F441E002C0FF24F394D3
:108C800098012E5F3F4F89012F5F3F4FF801808190
:108C90008032C9F3DACF41110F94860BFF2021F007
:108CA00087E39CE00F949D0AC8010E94C45355C5F8
:108CB0000E94E6E052C581E08093AF098093AE093F
:108CC0000E943DE14AC50E9405E2182F87FD45C577
:108CD00084E40E94C48C882309F43FC00E948D8CD8
:108CE0006B017C0101E020E030E0A9010F94342405
:108CF000811101C000E000939D1220E030E0A90145
:108D0000C701B6010F943424882339F10E948D8C59
:108D100024E01202F0011124EE55FD4E60837183B0
:108D20008283938320E030E0A9016091A2127091C8
:108D3000A3128091A4129091A5120F943424811152
:108D40000CC080E090E0A0EEBFE38093A21290936D
:108D5000A312A093A412B093A5120E94DAC1FDC47D
:108D60000E9405E287FDF9C4A5E0EA2EA3E0FA2EF1
:108D700008E311E1B8E4CB2EB1E1DB2ED7018D91F0
:108D80007D010E94C48C882349F00E948D8C0F9431
:108D90009D2CF80160837183828393830C5F1F4F46
:108DA000C016D10659F70E9481BED7C40E9405E2C1
:108DB00087FDD3C4F5E0EF2EF3E0FF2E08E311E1C9
:108DC000D7018D917D010E94C48C882339F00E94C7
:108DD0008D8CF80164A375A386A397A30C5F1F4F26
:108DE000F1E108341F0761F7B8C40E943FA4B5C47D
:108DF00075E0C72E73E0D72EE2EBEE2EE9E0FE2EF3
:108E000010E0D6018D916D010E94C48C882351F031
:108E10000E948D8CF7016083718382839383812FFD
:108E20000E9449C51F5FF4E0EF0EF11C133049F7B3
:108E30000C94783D0E9403E490C483E50E940D8D5C
:108E4000882309F48AC40E94898C909360028093DD
:108E50005F0283C40E9405E2F82E87FD7EC483E58D
:108E60000E940D8D0F2D0F2C000C110B882369F122
:108E70000E94898CF801EE0FFF1FE05DFD4F91838A
:108E80008083000F111F000F111F98012B5E3D4FB3
:108E90007901BC01990F880B990B0F943B242AE0B0
:108EA00037ED43E25CE30F949A24F801E256FD4E5D
:108EB00020813181428153810F949A24D7016D938F
:108EC0007D938D939C93139748C40F94860B85E4F0
:108ED0000E94B95280E38F0D0E94B952000F111FFA
:108EE000F801E05DFD4F608171818BE39CE00F94A0
:108EF000620B85E20E94B9528AE00E94B9522DC4E9
:108F000080E50E94C48C882309F427C460E070E0E7
:108F100080E50E94E1A6F82E6FEF7FEF83E50E94C7
:108F2000E1A68C010196039708F017C4F7FC15C45D
:108F30008F2D0E942A50882339F00F94820B83E4EE
:108F40009CE00F949D0A09C40E941CBF60E08F2D15
:108F50000E9493ED0F3FBFEF1B0731F00130110569
:108F600071F000E010E00DC08F2D0E943BED31E06C
:108F700020E0892B09F030E0032F122F02C001E01E
:108F800010E08F2D0E943BED8017910709F4E5C397
:108F900080E00E94E553F5CF80E50E94C48C8823D1
:108FA00009F4DBC30E94898C8C01892B09F07FC0F6
:108FB00083E50E94C48C882389F00E94898C8F3FAE
:108FC000EFEF9E0729F485E296E10E947150C5C338
:108FD000BC0185E296E10E944151BFC30F94860B0C
:108FE00060E070E08BE69CE00F94620B80912716A6
:108FF00028E532E06901C81AD10887FDD394CC0C6A
:10900000DD1CCC0CDD1C0D2C000CEE08FF08809143
:10901000261628E830E04901881A910887FD9394C4
:10902000880C991C880C991C092C000CAA08BB08F8
:10903000809125168F3FC1F090E0FC01EE0FFF1FDD
:109040008E0F9F1FFC01E854FA4E2181328183E08C
:10905000220F331F8A95E1F794E0369527959A956C
:10906000E1F72E5F3F4F02C020E030E02F5F3F4F1F
:10907000C901330FAA0BBB0B9C01AD01281939099B
:109080004A095B09A4EBB0E00F94CB2AA701960133
:10909000281939094A095B090F94AC2AB90188E6F5
:1090A0009CE00F94620B8AE00E94B95256C30F9461
:1090B000820BB80181E69CE00F94620B82E59CE094
:1090C0000F949D0A4AC38AE50E940D8D811135C611
:1090D00083E50E940D8D811130C63FC360E085E4B9
:1090E0000E94F0A6811173C080E50E94C48C882381
:1090F00051F00E948D8C6093F50B7093F60B80936A
:10910000F70B9093F80B89E40E94C48C882381F0BC
:109110000E948D8C2CEA35EC47E25EE30F949A2492
:109120006093F90B7093FA0B8093FB0B9093FC0BFD
:1091300084E40E94C48C882381F00E948D8C2CEAE8
:1091400035EC47E25EE30F94242C6093FD0B7093A3
:10915000FE0B8093FF0B9093000C0F94860B4091B5
:10916000F50B5091F60B6091F70B7091F80B8EE9AF
:109170009CE00F94510B2CEA35EC47E25EE36091E2
:10918000F90B7091FA0B8091FB0B9091FC0B0F94F3
:10919000242CAB01BC018AE99CE00F94510B2CEA12
:1091A00035EC47E25EE36091FD0B7091FE0B809120
:1091B000FF0B9091000C0F949A24AB01BC0186E93F
:1091C0009CE00F94510B8AE00E94B952C6C20F94E2
:1091D000820B84E89CE00F949D0ABFC280E50E9448
:1091E000C48C882351F00E948D8C60938E097093FB
:1091F0008F09809390099093910989E40E94C48C0F
:10920000882381F00E948D8C2CEA35EC47E25EE3E6
:109210000F949A2460939209709393098093940910
:109220009093950984E40E94C48C882381F00E9465
:109230008D8C2CEA35EC47E25EE30F94242C60938E
:1092400096097093970980939809909399090F94C0
:10925000860B40918E0950918F0960919009709111
:1092600091098AEA9CE00F94510B2CEA35EC47E215
:109270005EE36091920970919309809194099091B5
:1092800095090F94242CAB01BC0186EA9CE00F9455
:10929000510B2CEA35EC47E25EE360919609709140
:1092A000970980919809909199090F949A24AB019C
:1092B000BC0182EA9CE00F94510B8AE00E94B952F3
:1092C0004CC283E50E94C48C182F882371F00E9441
:1092D0008D8C0F94962C70931A026093190221E0E2
:1092E000672B09F020E02093E90B80E50E94C48CF5
:1092F000882359F02091190230911A02232B11F082
:109300000E94798C8093E90B28C2111126C20F9418
:10931000860B8AEC9CE00F949D0A8091E90B8823D0
:1093200019F082EB9CE002C08EEA9CE00F949D0A4B
:109330006091190270911A0289EB9CE00F94620B04
:1093400085EB9CE00F949D0A08C20E9452C805C29A
:109350000E941CBF02C281E00E94FB9C0E94B0DF01
:10936000FCC180918A12887809F04CC580918C12DA
:10937000867009F047C576C56FEF7FEF89E40E94DC
:10938000E1A6F82E6FEF7FEF8AE40E94E1A6E82EB7
:109390008AE50E94C48C182F811105C081E50E94C6
:1093A000C48CB82E01C0B12CF7FC06C0E7FC04C089
:1093B000111109C0B11007C00F94820B84E39DE026
:1093C0000F949D0ACAC1F4E0FF1510F0FE1538F4A1
:1093D0000F94820B85E19DE00F949D0ABEC1CF2CB6
:1093E0000F2C000CDD080E2D0E2C000C110B0E9412
:1093F0008D8CBB2099F025E02C9DF0012D9DF00D6A
:109400001124E00FF11FEE0FFF1FEE0FFF1FE75CAF
:10941000FB4E208131814281538103C020E030E046
:10942000A9010F942A2B9B01AC0185E08C9DF001D2
:109430008D9DF00D1124E00FF11FEE0FFF1FEE0FB9
:10944000FF1FE75CFB4E20833183428353836E2DE5
:109450008F2D0E940DC781C10E9497E881117DC1A7
:1094600007ED19E227E732E03DA32CA3CE010196D8
:109470005C014CE2842E4AE2942E1C01F8016591B5
:10948000759185919491ACA1BDA1CD90DD90ED90A9
:10949000FD90BDA3ACA3A70196010F94292B2B012E
:1094A0003C01F101608371838283938320E030E08B
:1094B00040EA51EC0F948A2D87FD0AC020E030E08D
:1094C00040EA51E4C301B2010F94342418162CF47D
:1094D000F401849118160CF4E9C4D101CD90DD900B
:1094E000ED90FD901D0120E030E040EA51ECC70115
:1094F000B6010F948A2D87FD0AC020E030E040EAD3
:1095000051E4C701B6010F943424181664F40F9483
:10951000820B82E79DE00F949D0A61E084E69DE066
:109520000E9449F51AC10C5F1F4FBFEF8B1A9B0AAF
:10953000E9E2033E1E0709F0A1CF32EBE32E39E04A
:10954000F32E10E0F50181919191A191B1915F010C
:10955000F70181939193A193B1937F01812F0E9491
:1095600049C51F5F133071F70E94B0DF60E084E5EA
:109570009DE00E9449F5F1C00F945601EEC00E9493
:10958000E7FCEBC081E0809328140E9442F6109221
:109590002814882309F4E1C00F94860B80E99DE02C
:1095A0000F949D0ADAC08091391882FFD6C080627C
:1095B00080933918D2C00E9479B3CFC00E9405E2CF
:1095C000082F87FDCAC085E50E94C48C8823B1F1AD
:1095D000E02E002E000CFF080E948D8C4B015C01D8
:1095E00020E030E0A9010F948A2D87FF04C0B7FA6C
:1095F000B094B7F8B094C70123E0880F991F2A955B
:10960000E1F79C012F5C3B4E7901D9018D929D922F
:10961000AD92BC92139720E030E04AEF53E4C501CD
:10962000B4010F948A2D18164CF480E090E0AAEF54
:10963000B3E4F70180839183A283B3838CE40E9417
:10964000C48C882309F489C0002E000C110B0E94E1
:109650008D8C6B017C0120E030E0A9010F948A2DF4
:1096600087FF04C0F7FAF094F7F8F09420E030E0B8
:109670004AEF53E4C701B6010F948A2D980193E095
:10968000220F331F9A95E1F7F901EF5CFB4E181694
:109690002CF0C482D582E682F7825FC080E090E041
:1096A000AAEFB3E484839583A683B78356C08BE483
:1096B0000E940D8D882329F10E948D8C6B017C0105
:1096C00020E030E0A9010F948A2D87FD15C020E02D
:1096D00030E040E251E4C701B6010F94342418167B
:1096E0005CF00E941CBFC092010CD092020CE09270
:1096F000030CF092040C31C08BE99DE00F949D0A9D
:109700002CC00F94860B4091010C5091020C60917B
:10971000030C7091040C8AEB9DE00F94510B8AE0CE
:109720000E94B9521AC081E08093870210920E14F1
:1097300060E083E50E941A8D81110FC00E9495CFD1
:109740000CC00E94737F09C080918E12882329F07B
:109750000E94966C02C00E94737F2296FFAD2297F2
:10976000F11102C00E9482B22CAD20936F12CF5B28
:10977000DF4F0FB6F894DEBF0FBECDBFDF91CF91A4
:109780001F910F91FF90EF90DF90CF90BF90AF901F
:109790009F908F907F906F905F904F903F902F9011
:1097A00008950E941CBF3091B6183CAB80E00F9426
:1097B00013080E9403DE81E08093AF090E943DE11F
:1097C00088E50E94C48C182F89E50E94C48C082F5C
:1097D0008AE50E94C48C1013C0C1181711F0012F24
:1097E000BCC101E011E091E09CA70E944B8C82E596
:1097F0000E940D8D882361F00E948D8C6B017C018D
:1098000020E030E0A9010F943424882369F106C0D8
:10981000C12CD12C40E8E42E40E4F42E111103C0F9
:10982000002309F4FCC0C092AD13D092AE13E092B5
:10983000AF13F092B013A701960160917F0270916F
:10984000800280918102909182020F94342487FFDC
:109850000BC019821A821B821C82BE016F5F7F4F70
:109860008DEA93E10E9405DF112309F4D3C00023A0
:1098700009F4CDC010927B0210927C0210927D02FE
:1098800010927E0210927702109278021092790262
:1098900010927A020E94AEDFECE2FAE2A491A8AF45
:1098A000E0E2FAE2C590D590E590F490E4E2FAE2C5
:1098B00085909590A590B490A5019401C701B6013B
:1098C0000F948A2D18162CF4A7019601C501B40136
:1098D00004C0A5019401C701B6010F94242C2B01EB
:1098E0003C01E7EEF9E285919591A591B4918CA3A5
:1098F0009DA3AEA3BFA3E3EEF9E285919591A59157
:10990000B49188A799A7AAA7BBA79C01AD016CA198
:109910007DA18EA19FA10F948A2D181634F428A43E
:1099200039A49AA598AB1BA505C02CA03DA0AEA15B
:10993000A8AB1FA1A3019201C301B2010F949A2405
:1099400020E030E040E85FE30F942A2B0F94D82DFD
:10995000910148A9512F0F949A2468A379A38AA34F
:109960009BA3EDE2FAE2149120E030E040EC5FE3EB
:10997000C501B4010F949A244B015C01612F110FB2
:10998000770B880B990B0F943B249B01AC01C5010D
:10999000B4010F949A2469837A838B839C8320E09B
:1099A00030E040EC5FE3C701B6010F949A246B01ED
:1099B0007C01B8AD6B2FBB0F770B880B990B0F9405
:1099C0003B249B01AC01C701B6010F949A246C8F14
:1099D0007D8F8E8F9F8FAE01405E5F4FBE016F5FA8
:1099E0007F4FCE014C960E94E3DE0E94DCFC109279
:1099F0007B0210927C0210927D0210927E021092E5
:109A00007702109278021092790210927A0280E026
:109A10000E9416C4002319F081E00E9416C4ECA530
:109A2000EE2309F48CC080E00E9444928091A5143A
:109A30008370833051F060E08DEC97E00E9449F52F
:109A40000F94860B8EEB97E093C00E94AEDF80915F
:109A50007F0290918002A0918102B0918202809356
:109A6000AD139093AE13A093AF13B093B0132091A6
:109A7000C1133091C2134091C3135091C41360E0DD
:109A800070E088E492E40F94292B6B017C016093D1
:109A9000A5137093A6138093A7139093A8132091F6
:109AA000C5133091C6134091C7135091C81360E09D
:109AB00070E088E492E40F94292B4B015C016093E1
:109AC000A9137093AA138093AB139093AC1327E15F
:109AD00037EB41ED58EB0F948A2D87FD40C023E012
:109AE00030E044EB53E4C501B4010F94342418165C
:109AF000B4F127E137EB41ED58EBC701B6010F9404
:109B00008A2D87FD2CC023E030E044EB53E4C701ED
:109B1000B6010F943424181614F119821A821B828C
:109B20001C82AE014F5F5F4F69EA73E185EA93E102
:109B30000E94E3DE82E00E9416C40E94B39C0E9451
:109B4000AEDF8091AE098093AF098CA90F94130802
:109B50000E94EADD0E94B0DF00CE8CA746CE60E016
:109B60008DEA97E00E9449F50F94860B8BE997E008
:109B70000F949D0AE2CF61E081E998E00E942F8D69
:109B80008CE198E00E9480BB61E08BEA94E30E9444
:109B90002F8D8DE098E00F94770388E50E94C48CA8
:109BA00081115F9889E50E94C48C81118A988AE5A9
:109BB0000E94C48C882329F08091080181708093D1
:109BC000060185E40E94C48C882309F4C6CD12984E
:109BD000C4CD0E94558CAB01BC0140933518509305
:109BE0003618609337187093381884E495E10E9412
:109BF0004D64B3CD61E0802F0E9493ED6F2D802FD7
:109C00000E9464ED6F2D70E0802F0E94CFED47E041
:109C1000E41203C0F092D80BA0CD89E0E8129DCDEC
:109C2000F092D70B9ACD0E94658C90E08536910515
:109C300014F084E690E0809315148FCD0E94E7BC69
:109C40000C94EE43A3019201C501B4010F948A2D37
:109C500018163CF08FEC99E060E00E9449F50C94F6
:109C60000E448CED99E0F8CF0E948D8C0F94962CC9
:109C7000CB010E943D8C0E948D8C20E030E040EAB8
:109C800050E40F948A2D181614F40E94E7BC6091DA
:109C90008B0970918C09072E000C880B990B0F947F
:109CA0003B2420918709309188094091890950917E
:109CB0008A090F948A2D18161CF484E19AE002C0D8
:109CC00085E09AE060E00E9449F5812F0E947DD0F6
:109CD00044CD0E941CBF88E50E94C48C882331F0CB
:109CE0005F9A8091A5148E7F8093A51489E50E94C8
:109CF000C48C882331F08A9A8091A5148D7F80933B
:109D0000A5148AE50E94C48C882359F0809108012B
:109D100080958170809306018091A5148B7F80933C
:109D2000A51485E40E94C48C882309F416CD0E94F2
:109D3000285013CD0E94B0C010CD0E948D8C20E021
:109D400030E040E050EC0F94342487FD15C00E94B1
:109D50008D8C20E030E040E050E40F948A2D1816FE
:109D60002CF00E948D8C6B017C010BC0C12CD12C7E
:109D7000E12C10E4F12E05C0C12CD12CE12CB0EC6B
:109D8000FB2E209154113091551140915611509154
:109D90005711C701B6010F949A240F94962CCB014A
:109DA0000F94C60580E50E94C48C882329F00E9488
:109DB000798C882309F4D1CCA70196016091C9134D
:109DC0007091CA138091CB139091CC130F942A2BCE
:109DD0006093C9137093CA138093CB139093CC13E1
:109DE0000F94860B4091C9135091CA136091CB1305
:109DF0007091CC1383E79CE00F94510B8AE00E9492
:109E0000B952ABCC88E40E94C48C882321F00E9414
:109E1000798C8093EE0882E50E94C48C082F83E53C
:109E20000E94C48C182F011102C0882351F0109297
:109E300081090E944F50112321F00E94798C809358
:109E40001B0284E40E94C48C882309F486CC0E94FF
:109E50008D8C6093690270936A0280936B02909379
:109E60006C027BCC0F94860B84E09DE00F949D0ADE
:109E700080911B02811117C08DED9CE00F949D0A0B
:109E80008AE00E94B9524091690250916A02609141
:109E90006B0270916C0284EE9CE00F94510B8AE08F
:109EA0000E94B9525ACC81EE9CE0E8CFF7FAF094C8
:109EB000F7F8F094D101CD92DD92ED92FC921397D8
:109EC0000CCBCF92DF92EF92FF920F931F93CF9321
:109ED000DF936C018B017A01EC01CB50D74F888165
:109EE00087FF04C0FB011182108224C02CE02C9D4E
:109EF000C0012D9D900D11242881AC01420F511DF0
:109F000027FD5A952091241630E04217530794F408
:109F10002881AC01420F511D27FD5A959A01FA0183
:109F2000EE0FFF1F2E0F3F1FF901E854FA4E20815C
:109F300027FD19C088818F5F88832CE02C9DC0018C
:109F40002D9D900D11242881AC01420F511D27FD3C
:109F50005A952091241630E042175307BCF428810B
:109F60002C3044F113C02881820F911D27FD9A9552
:109F7000FC01EE0FFF1F8E0F9F1FFC01E854FA4EED
:109F8000808160E08F770E9464EDD4CFF8018081FA
:109F90009181049680349C4918F480E49CE904C0C3
:109FA000F801808191810496F701918380838FEF7E
:109FB000888345C0F801408151812881BC01620F2E
:109FC000711D27FD7A959B01FB01EE0FFF1F2E0FE0
:109FD0003F1FF901E854FA4E21813281240F351FC9
:109FE000F701318320832881AC01420F511D27FDE9
:109FF0005A959A01FA01EE0FFF1F2E0F3F1FF9012C
:10A00000E854FA4E208127FF1AC02881820F911D43
:10A0100027FD9A95FC01EE0FFF1F8E0F9F1FFC017D
:10A02000E854FA4E808161E08F77DF91CF911F91E4
:10A030000F91FF90EF90DF90CF900C9464EDDF9143
:10A04000CF911F910F91FF90EF90DF90CF900895E7
:10A05000129A0895FF920F931F93CF93DF931F924D
:10A06000CDB7DEB7F82E0FED1DE041E050E0B801AE
:10A07000CE0101960F946E2389818F1102C081E079
:10A0800007C00F5F1F4F8DE0083F180771F780E092
:10A090000F90DF91CF911F910F91FF9008958091C4
:10A0A000690290916A02A0916B02B0916C02809358
:10A0B000A2119093A311A093A411B093A511089598
:10A0C0008091F808811107C00F945601882319F078
:10A0D00081E08093F8080895E7EDFBE0108211829B
:10A0E0000895DC01EC91F0E0CF01880F991FE80F93
:10A0F000F91FE854FA4E80818F77808308958F92FC
:10A100009F92AF92BF92CF92DF92EF92FF920F9306
:10A11000CF93DF931F92CDB7DEB75C016B017A015D
:10A120004901F501808191810F94642A898300237C
:10A1300011F0F6018083BE016F5F7F4FC4010F9461
:10A140006802F50180819181019691838083FFEF00
:10A15000CF1ADF0A81E0E81AF10819F780E00F90C2
:10A16000DF91CF910F91FF90EF90DF90CF90BF9054
:10A17000AF909F908F9008957F928F929F92AF9211
:10A18000BF92CF92DF92EF92FF920F931F93CF93E4
:10A19000DF931F92CDB7DEB77C0159018B016B01B4
:10A1A000C40ED51E0C151D0559F1F7018080918054
:10A1B000F80171908F017982C4010F94642A781696
:10A1C00091F0672DC4010F946C2AC4010F94642A86
:10A1D0009981891741F00F94860B85EC9DE00F94CF
:10A1E0009D0A81E00EC0BE016F5F7F4FC5010F94D5
:10A1F0006802F70180819181019691838083D2CF9B
:10A2000080E00F90DF91CF911F910F91FF90EF9021
:10A21000DF90CF90BF90AF909F908F907F900895E8
:10A22000009781F41092900082E080939100109248
:10A23000950010929400C19A809171008260809381
:10A24000710008958130910569F41092A00082E0B8
:10A250008093A1001092A5001092A40089BB809366
:10A2600072000895029761F41092200182E08093B9
:10A27000210110922501109224018ABB8093730062
:10A2800008957F928F929F92AF92BF92CF92DF926A
:10A29000EF92FF920F931F93CF93DF93FC01908176
:10A2A000943208F0CEC06B017F01892F90E0FC0151
:10A2B000EE0FFF1F8E0F9F1FFC01E854FA4E8081A6
:10A2C00061E08F770E9493EDF70111821282808105
:10A2D0006CE00F94ED2AFCE08F9FB001112440E068
:10A2E00050E09B01240F351FF901EE0FFF1F2E0FC9
:10A2F0003F1FF901E854FA4E908197FD08C04F5F67
:10A300005F4F4C30510569F790E00E941051F70102
:10A310007080C72DD0E08E01000F111FF801EC0FE7
:10A32000FD1FE854FA4E80818068808377FC89C0E5
:10A33000F0E2CF16F2E0DF060CF041C0F7018281B7
:10A3400028E532E0281B310987FD3395220F331FA2
:10A35000220F331F032E000C440B550B818168E83C
:10A3600070E04B01881A910887FD9394880C991C22
:10A37000880C991C092C000CAA08BB08D7FC0BC040
:10A38000B601653B710514F064EB70E0072E000C1C
:10A39000880B990B03C060E070E0CB0128193909E4
:10A3A0004A095B090F947A2A24EB30E040E050E040
:10A3B0000F94AC2A820E931EA41EB51E01C0460146
:10A3C000F3E2F71558F1F701218188E890E0821B4C
:10A3D000910927FD9395880F991F880F991F88165B
:10A3E000990684F0F701228188E592E0821B9109A9
:10A3F00027FD9395880F991F880F991F8816990636
:10A400000CF4C40102972FB7F894C00FD11FC854A1
:10A41000DA4E880F991F9A8389832FBF62E370E019
:10A4200080E090E0DF91CF911F910F91FF90EF902E
:10A43000DF90CF90BF90AF909F908F907F900D94C2
:10A440006E0ADF91CF911F910F91FF90EF90DF90F7
:10A45000CF90BF90AF909F908F907F9008951F9264
:10A460000F920FB60F9211240BB60F922F933F93BA
:10A470004F935F936F937F938F939F93AF93BF930C
:10A48000EF93FF9348E251E064E271E082E090E0F4
:10A490000E94614FFF91EF91BF91AF919F918F917A
:10A4A0007F916F915F914F913F912F910F900BBED4
:10A4B0000F900FBE0F901F9018951F920F920FB61E
:10A4C0000F9211240BB60F922F933F934F935F93EC
:10A4D0006F937F938F939F93AF93BF93EF93FF936C
:10A4E00048EA50E064EA70E081E090E00E94614F49
:10A4F000FF91EF91BF91AF919F918F917F916F915C
:10A500005F914F913F912F910F900BBE0F900FBE17
:10A510000F901F9018951F920F920FB60F92112453
:10A520000BB60F922F933F934F935F936F937F934D
:10A530008F939F93AF93BF93EF93FF9348E950E0BE
:10A5400064E970E080E090E00E94614FFF91EF913C
:10A55000BF91AF919F918F917F916F915F914F913B
:10A560003F912F910F900BBE0F900FBE0F901F9039
:10A5700018959091C00095FFFCCF8093C600089578
:10A580008F929F92AF92BF92EF92FF920F931F9381
:10A59000CF93DF93CDB7DEB7A0970FB6F894DEBFA9
:10A5A0000FBECDBF611571058105910591F100E0E8
:10A5B000842E912CA12CB12C102FEE24E394F12C9D
:10A5C000EC0EFD1EE00EF11C07FDFA94A5019401AE
:10A5D0000F948A2AF7016083B901CA010F5F6115E0
:10A5E00071058105910541F71F3F31F1E1E0F0E090
:10A5F000EC0FFD1FE10FF11D17FDFA9580818A30E8
:10A6000010F097E301C090E3890F0E94B9521150F6
:10A61000EBCF80E3A0960FB6F894DEBF0FBECDBFA0
:10A62000DF91CF911F910F91FF90EF90BF90AF906E
:10A630009F908F900C94B952A0960FB6F894DEBFFD
:10A640000FBECDBFDF91CF911F910F91FF90EF9083
:10A65000BF90AF909F908F900895CF92DF92EF922E
:10A66000FF926B017C0197FF0BC08DE20E94B952F3
:10A67000F094E094D094C094C11CD11CE11CF11C56
:10A680004AE0C701B601FF90EF90DF90CF900C94A5
:10A69000C0528F929F92AF92BF92CF92DF92EF9271
:10A6A000FF92CF936B017C01B42E20E030E0A90132
:10A6B0000F94342487FF07C08DE20E94B952F7FA45
:10A6C000F094F7F8F094C0E060E070E080E09FE381
:10A6D000CB1541F02DEC3CEC4CEC5DE30F949A244F
:10A6E000CF5FF6CF9B01AC01C701B6010F942A2BB7
:10A6F0006B017C010F949D2C4B015C014AE00E9490
:10A70000C052CC2389F1C501B4010F9439249B01B7
:10A71000AC01C701B6010F94292B6B017C018EE2BD
:10A720000E94B95220E030E040E251E4C701B60196
:10A730000F949A244B015C010F94962C6B01770FB8
:10A74000EE08FF08C701B6010E942D53C701B601EC
:10A750000F943B249B01AC01C501B4010F94292B3C
:10A760006B017C01C150F1F6CF91FF90EF90DF902B
:10A77000CF90BF90AF909F908F9008958DE00E94F2
:10A78000B9528AE00C94B952CF93DF93EC018991CE
:10A79000882319F00E94B952FACFDF91CF910C941F
:10A7A000BE538091BD129091BE12981759F0E92FB7
:10A7B000F0E0E354FD4E82819F5F9F779093BE123D
:10A7C00090E008958FEF9FEF08952F923F924F9260
:10A7D0005F926F927F928F929F92AF92BF92CF9231
:10A7E000DF92EF92FF920F931F93CF93DF93CDB73A
:10A7F000DEB728970FB6F894DEBF0FBECDBFE82EA8
:10A800000E94771D0E94F1EE4B015C0180910002D5
:10A81000882359F180916F12882339F14091F9080A
:10A820005091FA086091FB087091FC089501840131
:10A83000041B150B260B370B37FD2AC0833079F02C
:10A840003CF4813094F00F94860B87E29EE00BC0BD
:10A85000843059F40F94860B88EF9DE004C00F9468
:10A86000860B80E19EE00F949D0A2091000230E06B
:10A87000A8EEB3E00F94DE2A860E971EA81EB91E1E
:10A880008092F9089092FA08A092FB08B092FC0816
:10A8900080911B02882319F18091810981111FC0C9
:10A8A0008091391882FD08C08091B812813021F062
:10A8B0008091450B882399F0F894649919C66091AA
:10A8C000A2117091A3118091A4119091A511789477
:10A8D00020E030E0A9010F94342487FD99C58091D0
:10A8E000420B843008F07EC20E94F1EE4B015C0105
:10A8F0008091420B81111DC08091BD129091BE12BA
:10A90000891B8F77B1F48091620990916309A091BE
:10A910006409B0916509A5019401281B390B4A0B04
:10A920005B0BDA01C901885E9340A109B109B7FF49
:10A93000F0C570E6F72E8091420B843008F035C1E7
:10A940008091BD129091BE12891B8F7709F42DC1A1
:10A950000E94D153AC0197FDEECF20913F1330916F
:10A9600040138A3019F08D3009F0ECC01092610963
:10A970002115310519F40F941F10DDCFF901EF5F98
:10A98000F64F10821092401310923F1301E019E02D
:10A99000F8018191803211F48F01FACF8E3409F0E1
:10A9A0007AC00115110509F476C069EA7FE0C80193
:10A9B0000F94B2236C01892B41F06EE470E0C80162
:10A9C00004960F947D2E009709F4C8014AE050E0E8
:10A9D00060E070E001960F942A216093FD08709367
:10A9E000FE088093FF089093000940904113509017
:10A9F000421360904313709044133FEF431A530A7D
:10AA0000630A730A641575058605970531F0CD282C
:10AA100021F460E086E79FE051C06AE270E0C8017F
:10AA20000F94AC2E9C01009709F1982F901BD12C0C
:10AA3000992339F09150F801E90FF11D8081D82652
:10AA4000F7CF4AE050E060E070E0C90101960F9452
:10AA50002A214D2C512C612C712C6415750586050D
:10AA6000970541F060E087E59FE028C060E08DE257
:10AA70009FE024C08091FD089091FE08A091FF08FE
:10AA8000B09100098093411390934213A093431314
:10AA9000B093441316C08091391880FF12C065E24C
:10AAA00071E1C8010F94B223009729F0FC01838162
:10AAB00080538A3030F460E083E09FE00E94B1CFA1
:10AAC00074C08091870281111CC067E470E0C801E6
:10AAD0000F947D2E0097A9F04AE050E060E070E00E
:10AAE00001960F942A21643071058105910548F47F
:10AAF0008CE89EE00F949D0A60E082E89EE00E9450
:10AB000049F58092620990926309A0926409B0921B
:10AB10006509809101098B3309F40DCF8091420BB7
:10AB2000843008F008CF8091BE09F89EC00111243E
:10AB300061E079E08F53964F0F94882E81E00E9458
:10AB4000D7B2F9CE2F3531050CF0F5CE8C35C1F4E6
:10AB50000E94D15397FDEFCE209161092111EBCED8
:10AB600020913F1330914013A9014F5F5F4F5093E5
:10AB7000401340933F13F901EF5FF64F8083DBCE24
:10AB80008B3321F481E080936109D5CE80916109F6
:10AB90008111D1CEC90101969093401380933F1348
:10ABA000F901EF5FF64F4083C6CE8091391882FFDE
:10ABB00019C18091420B811102C010926709DD24F6
:10ABC000D394409135185091361860913718709190
:10ABD00038188091311890913218A0913318B091A3
:10ABE0003418481759076A077B0708F4D12C00E08E
:10ABF00010E0CC24C39440E6B42E54E6A52E69E6BA
:10AC0000962E8091420B843008F0ECC0D110EAC03F
:10AC1000809167098111E6C080914C1590914D1586
:10AC2000A0914E15B0914F1580933518909336181A
:10AC3000A0933718B093381841E050E0BE016F5F21
:10AC40007F4F84E495E10E943268019719F489816D
:10AC500090E002C08FEF9FEFF82E40903518509093
:10AC6000361860903718709038184091311850910C
:10AC700032186091331870913418DD24D39444163F
:10AC800055066606770608F4D12C44165506660666
:10AC90007706B0F4019609F461C02AE0F21609F4CF
:10ACA0006EC03DE0F31609F46AC043E2F41619F0F1
:10ACB0005AE3F5127CC080916609811178C054C0B6
:10ACC0000E941CBF84E495E10E94B967809130180E
:10ACD000882339F1815080933018989EC001112447
:10ACE00041E061E0865B944F0E944261E091301840
:10ACF00064E0E69FF0011124EA5BF44F408151814A
:10AD000062817381409335185093361860933718D9
:10AD10007093381884E495E10E944D640E94F75DB9
:10AD200016C00E94E65D0E94B0C00E9497BD0E94BE
:10AD3000F9F36D3371058105910518F484EB9FE0FB
:10AD400002C089EB9FE00E941EB3A092151480916F
:10AD5000391882FD0DC08CEC9FE004C00F94820B6B
:10AD60008DEB9FE00F949D0A73E2F71208C005C0B7
:10AD700053E2F512DBC300E010E0C09267091092C5
:10AD800066090115110519F40F941F100DC080916B
:10AD9000BE09B89E000D111D1124F801EF53F64FA6
:10ADA000108280E00E94D7B200E010E02ACF0F3579
:10ADB000110508F026CF8BE3F81203C0C092660994
:10ADC00020CF8091660981111CCF8091BE09F801C6
:10ADD000B89EE00DF11D1124EF53F64FF0820F5F86
:10ADE0001F4F0FCF0E94F1EE4B015C014091EA082A
:10ADF0005091EB086091EC087091ED0841155105F8
:10AE00006105710529F180919D1490919E14A09186
:10AE10009F14B091A014840F951FA61FB71F950112
:10AE20008401081B190B2A0B3B0B37FD11C00F9433
:10AE3000820B6091B90B7091BA0B80EE9FE00F947A
:10AE40006F0B8AE00E94B95280E090E00F94770384
:10AE5000409101025091020260910302709104023C
:10AE6000411551056105710509F44EC090912B16ED
:10AE700080912C16981759F00E94F1EE60939D1462
:10AE800070939E1480939F149093A0143DC0809162
:10AE9000450B811137C0E11035C080919D14909110
:10AEA0009E14A0919F14B091A014840F951FA61F0B
:10AEB000B71FA5019401281B390B4A0B5B0B57FDEB
:10AEC00021C08091780981111FC081E080937809A9
:10AED0005F9A8091A5148E7F8093A5148A9A8091A1
:10AEE000A5148D7F8093A5148091080180958170B1
:10AEF000809306018091A5148B7F8093A5140E94F6
:10AF0000285002C0109278098091740990917509B7
:10AF1000A0917609B0917709B501A401481B590B9E
:10AF20006A0B7B0B77FDBCC120912B1690912C16E0
:10AF300080913F0210914002291317C06091D70BF6
:10AF4000869FB0011124660F672F661F770B7195DE
:10AF5000062F8091D80B189FB0011124660F672F20
:10AF6000661F770B7195162F29C020912C1653E57B
:10AF7000259F900111242B5F334FF901EF5AFF4FAA
:10AF80006081869FB0011124660F672F661F770BC3
:10AF90007195062F31968081819FB0011124660F33
:10AFA000672F661F770B7195162F80912C16909145
:10AFB0002B16981719F08F5F8F70F9CF002331F19E
:10AFC0000E94F1EEC0906C09D0906D09E0906E097E
:10AFD000F0906F09DC01CB01C114D104E104F1044C
:10AFE00069F48C599F4FAF4FBF4F80936C0990937A
:10AFF0006D09A0936E09B0936F0906C08C199D0965
:10B00000AE09BF09B7FF0AC00FEF08C010926C0964
:10B0100010926D0910926E0910926F09602F70E006
:10B0200089E00E94CFED112331F10E94F1EEC09032
:10B030007009D0907109E0907209F0907309DC01F9
:10B04000CB01C114D104E104F10469F48C599F4F80
:10B05000AF4FBF4F8093700990937109A09372090D
:10B06000B093730906C08C199D09AE09BF09B7FFDB
:10B070000AC01FEF08C01092700910927109109257
:10B08000720910927309612F70E087E00E94CFED82
:10B0900080915D13882309F4F6C0E0903602F090A9
:10B0A000370200913802109139026091F20B7091D1
:10B0B000F30B6E5F7F4F072E000C880B990B0F94DC
:10B0C0003B249701A8010F94342487FDDCC0309005
:10B0D0002C16212C1A821B821C8280912B16831520
:10B0E00009F467C0832D90E063E5689FF001699FD4
:10B0F000F00D1124EB5FF34F458956896789708DF8
:10B10000452B462B472B89F4418D528D638D748DD1
:10B11000452B462B472B49F4458D568D678D70A1E5
:10B12000452B462B472B09F43FC073E5789F9001D0
:10B13000799F300D1124C9018B5F934F6C01FC0185
:10B1400061817281838194810F94D82D2B013C0100
:10B15000F60161A172A183A194A10F9439246D839A
:10B160007E838F839887F60165A176A187A190A53C
:10B170000F9439249B01AC016D817E818F8198856C
:10B180000F94242CA30192010F949A243B016C018B
:10B19000222D3A814B815C810F948A2D181624F45C
:10B1A000262C7A82CB82DC8281E0830D8F70382E50
:10B1B00094CF20913A0230913B0240913C02509151
:10B1C0003D02622D7A818B819C810F949A24970194
:10B1D000A8010F942A2B3B016C0120903202309081
:10B1E000330240903402509035029B01AC01B7010C
:10B1F000C8010F948A2D18166CF09101A201B301B9
:10B20000C6010F948A2D18161CF47101820102C028
:10B2100073018601409068095090690960906A093D
:10B2200070906B099701A801C301B2010F948A2D98
:10B230001816C4F420E037ED43EA5CE3B701C80117
:10B240000F949A246B017C0128E431EE4AE75FE316
:10B25000C301B2010F949A24A70196010F942A2BDF
:10B260007B018C01C701D80180936809909369091B
:10B27000A0936A09B0936B09B701C8010F94962C8B
:10B28000CB010E94ECD7F4E68F0E911CA11CB11CDF
:10B290008092740990927509A0927609B09277090C
:10B2A0000F941F108091B812813009F06EC00E9477
:10B2B000F1EE6B017C0180917D0990917E09A09156
:10B2C0007F09B091800997018601081B190B2A0B91
:10B2D0003B0B37FD3AC08090B9129090BA12A09003
:10B2E000BB12B090BC120E94F9F36093B912709334
:10B2F000BA128093BB129093BC120091A2091091D4
:10B30000A3092091A4093091A509081919092A094E
:10B310003B09DC01CB01800F911FA21FB31F80935B
:10B32000A2099093A309A093A409B093A509D701FA
:10B33000C601805F984DAF4FBF4F80937D099093BA
:10B340007E09A0937F09B09380098091790990913B
:10B350007A09A0917B09B0917C09A7019601281B6D
:10B36000390B4A0B5B0B57FD10C030E8C30E3EEEA5
:10B37000D31EE11CF11CC0927909D0927A09E092A7
:10B380007B09F0927C090E9471BD8091E5088823B9
:10B3900091F00E94F1EE0091E1081091E2082091F5
:10B3A000E3083091E408DC01CB01801B910BA20B78
:10B3B000B30BB7FFBEC00E94F1EE6B017C01209180
:10B3C000E008222309F4D3C08091DC089091DD08C5
:10B3D000A091DE08B091DF08B701A601481B590B08
:10B3E0006A0B7B0B77FDC3C030E0A8EEB3E00F948F
:10B3F000DE2AC60ED71EE81EF91EC092DC08D092C7
:10B40000DD08E092DE08F092DF080E94BF5DAFC069
:10B4100011E0109381098091450B811166C086E38C
:10B4200096E00E94C45384E08093B21282E080933D
:10B43000BC0881E09AE59093BE168093BD168EE419
:10B4400090E09093C0168093BF1687E08093B1166A
:10B4500082E88093B41684E890E0A0E0B0E08093A6
:10B46000B5169093B616A093B716B093B8160F946E
:10B47000D102109391110E94538D40E061E77EE06C
:10B4800087E597E10E945F8D80E30E94B9528AE0D0
:10B490000E94B9520E94478D8091EE0860E0182703
:10B4A00019F087E396E10DC08FE59EE00E942F8D95
:10B4B00080E30E94B9528AE00E94B95260E089E3B9
:10B4C0009EE00E942F8D8DE49EE00F949D0A80E304
:10B4D0000E94B9528AE00E94B952112331F08FE3E1
:10B4E0009EE09093C0098093BF090E941CBFF7C9DA
:10B4F0008091690290916A02A0916B02B0916C02F6
:10B500008093A2119093A311A093A411B093A511BD
:10B51000D6C98EEA9FE00F949D0A809262099092AC
:10B520006309A0926409B092650903CA1092660982
:10B530002BCC0E94F1EE6B017C012091E50830E0FC
:10B54000A8EEB3E00F94DE2AC60ED71EE81EF91E41
:10B55000C092E108D092E208E092E308F092E40899
:10B5600080E00E940BD08AE00E94B95224CF289636
:10B570000FB6F894DEBF0FBECDBFDF91CF911F9104
:10B580000F91FF90EF90DF90CF90BF90AF909F9082
:10B590008F907F906F905F904F903F902F90089585
:10B5A0001F920F920FB60F9211240F900FBE0F90A3
:10B5B0001F9018951F920F920FB60F9211240BB681
:10B5C0000F920F931F932F933F934F935F936F931C
:10B5D0007F938F939F93AF93BF93CF93DF93EF931B
:10B5E000FF930091BE12D091BD1211E01D0F1F7785
:10B5F000C091C6009091F408492F092E000C550BFC
:10B60000660B770B4131510508F064C0FA018827B9
:10B61000E256FF4F8F4F0D94212BCD3449F0CE349D
:10B62000B9F481E006C0CA3338F0CD3409F043C024
:10B6300082E08093F40876C0C03308F073C0C03253
:10B6400009F470C0CD32B9F56DC0C13351F018F4B2
:10B65000C03289F567C0C43331F0C83361F58BE07F
:10B66000E8CF83E0E6CF88E0E4CFC03321F0C133F8
:10B6700011F586E0DECF84E0DCCFC833E1F485E06D
:10B68000D8CFC233C1F487E0D4CFC133A1F489E06D
:10B69000D0CFC03381F48AE0CCCFC73361F48CE0E3
:10B6A000C8CFC63341F48DE0C4CFC032D9F1C33521
:10B6B00011F48EE0BECF80E1BCCF80ED8C0F8A30DC
:10B6C00088F59FE09093F4088093F3082BC0CA306C
:10B6D00049F526C0CA3031F580911F17882301F142
:10B6E000973089F03CF49530D9F4109214021092FE
:10B6F000141416C09A3059F09F3091F48091F308D9
:10B700000E948B8D0DC081E08093571E09C00E945E
:10B7100006C10E941CBF8EEF0E9440DF0E94AEDF78
:10B720001092F408011731F0ED2FF0E0E354FD4ED4
:10B73000C283D12FD093BD12FF91EF91DF91CF91B2
:10B74000BF91AF919F918F917F916F915F914F9139
:10B750003F912F911F910F910F900BBE0F900FBE35
:10B760000F901F9018958EBD0DB407FEFDCF089564
:10B770008FEF8EBD0DB407FEFDCF8EB5089590916D
:10B7800064009B7F90936400982F906A96959CBD6F
:10B7900080FD03C091E0863009F490E09DBD0895DE
:10B7A000CF92DF92EF92FF920F931F93CF93DF938D
:10B7B0006C017A018B01C0E0D0E0CE15DF0581F08D
:10B7C000D8016D918D01D601ED91FC910190F08130
:10B7D000E02DC6011995892B11F02196EECF7E013F
:10B7E000C701DF91CF911F910F91FF90EF90DF90F4
:10B7F000CF900895089580E090E00895FC01538D66
:10B80000448D252F30E0842F90E0821B930B54173A
:10B8100010F0CF96089501970895FC01918D828DC7
:10B82000981761F0828DDF01A80FB11D5D968C9194
:10B83000928D9F5F9F73928F90E008958FEF9FEF9F
:10B840000895FC01918D828D981731F0828DE80F5B
:10B85000F11D858D90E008958FEF9FEF0895FC0115
:10B86000918D228D892F90E0805C9F4F821B9109E2
:10B870008F739927089587EA94E10E942F5C21E055
:10B88000892B09F420E0822F0895FC01848DDF01CB
:10B89000A80FB11DA35ABF4F2C91848D90E0019643
:10B8A0008F739927848FA689B7892C93A089B18932
:10B8B0008C91837080648C93938D848D981306C0D3
:10B8C0000288F389E02D80818F7D80830895EF9237
:10B8D000FF920F931F93CF93DF93EC0181E0888F4A
:10B8E0009B8D8C8D981305C0E889F989808185FD31
:10B8F00026C0F62E0B8D10E00F5F1F4F0F73112720
:10B90000E02E8C8DE8120CC00FB607FCFACFE88948
:10B91000F989808185FFF5CFCE010E94455CF1CF8A
:10B920008B8DFE01E80FF11DE35AFF4FF0829FB7A8
:10B93000F8940B8FEA89FB89808180620AC09FB7E7
:10B94000F894EE89FF896083E889F98980818370A2
:10B95000806480839FBF81E090E0DF91CF911F9151
:10B960000F91FF90EF900895CF93DF93EC01888DB6
:10B970008823C9F0EA89FB89808185FD05C0A889F3
:10B98000B9898C9186FD0FC00FB607FCF5CF808179
:10B9900085FFF2CFA889B9898C9185FFEDCFCE01C3
:10B9A0000E94455CE7CFDF91CF91089580E090E061
:10B9B000892B41F080E090E0892B21F00E9400006B
:10B9C000811121C080E090E0892B41F080E090E07F
:10B9D000892B21F00E940000811118C080E090E0C6
:10B9E000892B21F00E943B5C811113C080E090E024
:10B9F000892BA1F080E090E0892B81F00E9400006B
:10BA000081110AC008950E940000DCCF0E9400004E
:10BA1000E5CF0E940000EACF0C9400000895FC01DD
:10BA200020E03EE2DB014C91403241F0283011F43D
:10BA300030833196DB014C91408331962F5F6F5FED
:10BA40007F4F2B3079F7108208950F943C2E0F937F
:10BA50001F93CF93DF938B01EA01DB016D917C9102
:10BA60000E945365D801ED91FC91119790818881D6
:10BA7000992349F0893638F43196ED93FC93888107
:10BA80008F5F8883EFCF893658F48FE28083F80187
:10BA90008081918101969183808388818F5F8883E3
:10BAA000DF91CF911F910F9108951F920F920FB6C2
:10BAB0000F9211240BB60F922F933F934F935F93E6
:10BAC0006F937F938F939F93AF93BF93EF93FF9366
:10BAD00087EA94E10E94455CFF91EF91BF91AF919D
:10BAE0009F918F917F916F915F914F913F912F9196
:10BAF0000F900BBE0F900FBE0F901F9018951F92C6
:10BB00000F920FB60F9211240BB60F922F938F93B3
:10BB10009F93EF93FF93E091B714F091B814808155
:10BB2000E091BD14F091BE1482FD12C0908180910D
:10BB3000C0148F5F8F732091C114821751F0E09170
:10BB4000C014F0E0E955FB4E958F8093C01401C0FE
:10BB50008081FF91EF919F918F912F910F900BBE5C
:10BB60000F900FBE0F901F9018958BE1EDE9F5E156
:10BB7000A2E8B5E101900D928A95E1F708958091D0
:10BB8000391882FF1FC085EA92E10F949D0A6091E7
:10BB900035187091361880913718909138184AE00E
:10BBA0000E94C0528FE20E94B95260913118709188
:10BBB000321880913318909134184AE00E94C05294
:10BBC0000C94BE5387EB92E10D949D0A1092450BA5
:10BBD000809139188F7D8B7F809339180E9487CF91
:10BBE000882321F084E495E10C94B967089580914D
:10BBF000391883FF03C08460809339180895CF9269
:10BC0000DF92EF92FF920F931F93CF93DF93CDB705
:10BC1000DEB7EDB6FEB6DC010D900020E9F79D0120
:10BC2000281B390B2C5F3F4F4DB75EB7421B530BA0
:10BC30000FB6F8945EBF0FBE4DBF0DB71EB70F5FB6
:10BC40001F4F9F938F9381EA91E19F938F931F934F
:10BC50000F930F94CC23680154E0C50ED11C0F90B4
:10BC60000F900F900F900F900F90F6018081882316
:10BC700049F0082E000C990B0F94412EF601819388
:10BC80006F01F3CFC8010E94ECB28DE991E10E94EF
:10BC90001EB30FB6F894FEBE0FBEEDBEDF91CF917E
:10BCA0001F910F91FF90EF90DF90CF9008958F92AA
:10BCB0009F92AF92BF92CF92DF92EF92FF92CF937B
:10BCC00080913918877F809339188091A015882337
:10BCD00021F08DE995E10E94B967109281151092CB
:10BCE0007E1585E380937D150E94F1EE6B017C014A
:10BCF00020EDC20E27E0D21EE11CF11CA89561E0E8
:10BD000080917D150E9464ED61E080917D150E9417
:10BD100093ED209A289A219A2398229A81E00E94F2
:10BD2000BF5B85E080937F150E94BF5BCAE08FEF09
:10BD30000E94B35BC150D9F7A89520E030E0A9017B
:10BD400060E08DE795E10E949966809380158130CF
:10BD500061F00E94F1EEDC01CB018C199D09AE0966
:10BD6000BF09B7FDEACF81E062C0A8952AEA31E0B9
:10BD700040E050E068E08DE795E10E9499668530EB
:10BD800011F481E00AC0C4E00E94B85B8093801582
:10BD9000C150D1F78A3A61F482E080938115A89569
:10BDA00080918115823081F0812C912C540111C039
:10BDB0000E94F1EEDC01CB018C199D09AE09BF098F
:10BDC000B7FDD4CF82E033C0812C912CA12C80E42C
:10BDD000B82E20E030E0A90167E38DE795E10E94ED
:10BDE0009966A501940169E28DE795E10E94996643
:10BDF00080938015882361F00E94F1EEDC01CB0175
:10BE00008C199D09AE09BF09B7FDE3CF8AE00FC0C9
:10BE100080918115823021F520E030E0A9016AE3AC
:10BE20008DE795E10E949966882361F088E0809310
:10BE30007E158DE795E10E9491660F94860B8FE841
:10BE400091E122C00E94B85B807C803C19F483E0C1
:10BE5000809381150E94B85B0E94B85B0E94B85B1A
:10BE60008DE795E10E94916610927F1581E00F9415
:10BE7000B90D81110CC080E00F94B90D811107C07C
:10BE80000F94820B8BE791E10F949D0A1AC06FE526
:10BE900075E18DE995E10E94E464811105C00F947C
:10BEA000820B8AE691E1F0CF809139188860809307
:10BEB00039180F94860B8EE591E10F949D0A0E942C
:10BEC0006050CF91FF90EF90DF90CF90BF90AF90F8
:10BED0009F908F900C94B55D2F923F925F926F92DE
:10BEE0007F928F929F92AF92BF92CF92DF92EF920A
:10BEF000FF920F931F93CF93DF93CDB7DEB7C35657
:10BF0000D1090FB6F894DEBF0FBECDBF8C016B0117
:10BF10004A012DB63EB6512C7E0187E5E80EF11C94
:10BF2000F6018381823008F41FC180859185A28546
:10BF3000B3858F719927AA27BB27892B8A2B8B2B37
:10BF400009F012C11092C61A46EC5AE1BE016F5FA9
:10BF50007F4FC6010E944E6918160CF005C18C85F2
:10BF6000982F9871903129F42091B30B21502230F1
:10BF700078F42981222309F4F7C0253E89F22E3274
:10BF800079F22091C61A2E3259F28A7049F67CC095
:10BF90006DB67EB6BE016F5F7F4FC7010E940F5D19
:10BFA0000115110521F0F8018081811163C021E0A4
:10BFB00081E090E0F70101900020E9F73197EE1958
:10BFC000FF09E80FF91F32968DB79EB78E1B9F0BA6
:10BFD0000FB6F8949EBF0FBE8DBFEDB7FEB731967A
:10BFE0005F01211102C0B80102C062E976E0C5011B
:10BFF0000F94882EB701C5010F94722E62E976E086
:10C00000C5010F94722E19A21CA221E0A701B6014E
:10C01000CE0181960E94A56B81110DC08091B30B5A
:10C02000811109C00F94860B8AE491E10F949D0A57
:10C03000C7010E94C4538BE1FE01B196DE01DC967C
:10C0400001900D928A95E1F740E050E0BE01645CFA
:10C050007F4FC5010E946C5FCE01CC960E94C267E3
:10C06000CE0181960E94C2670FB6F8947EBE0FBEC5
:10C070006DBE56CFF80101900020E9F73197CF014E
:10C08000801B910B20E096CF21E0903109F020E059
:10C090008091391820FB84F980933918903141F050
:10C0A0008985873409F03CCF8A858E3709F438CFEB
:10C0B0008091B30B813021F068F08230C1F130CF34
:10C0C0008091B60B9091B70B01969093B70B80932C
:10C0D000B60B26CFBE016F5F7F4F88E09BE10E94C9
:10C0E0000F5D0115110529F488E0A82E8BE1B82E0B
:10C0F00009C05801F50181915F018823A9F30E94CD
:10C10000B952F8CFF50181915F01882319F00E949F
:10C11000B952F8CF80E20E94B9526D8D7E8D8F8D1D
:10C1200098A14AE00E94C0520E94BE53F9CEBE01BF
:10C130006F5F7F4F88E09BE10E940F5D8114910447
:10C1400041F068E07BE1C4010F945F2E892B51F42C
:10C150000BC0852D90E02091B40B3091B50B821768
:10C16000930711F05394DCCE0FB6F8943EBE0FBE89
:10C170002DBECD59DF4F0FB6F894DEBF0FBECDBF39
:10C18000DF91CF911F910F91FF90EF90DF90CF90B3
:10C19000BF90AF909F908F907F906F905F903F90F7
:10C1A0002F900895CF93DF93CDB7DEB76B970FB67F
:10C1B000F894DEBF0FBECDBF81E08093B30B109229
:10C1C000B70B1092B60B82E895E10E948C668BE16A
:10C1D000E2E8F5E1DE01119601900D928A95E1F712
:10C1E00040E050E0BE016F5F7F4F80E090E00E9432
:10C1F0006C5FCE0101960E94C2678091B60B909150
:10C20000B70B6B960FB6F894DEBF0FBECDBFDF91B4
:10C21000CF9108950F931F93CF93DF93CDB7DEB7E0
:10C220006B970FB6F894DEBF0FBECDBF8B0122E037
:10C230002093B30B9093B50B8093B40B82E895E1F8
:10C240000E948C668BE1E2E8F5E1DE011196019037
:10C250000D928A95E1F7A801BE016F5F7F4F80E0E4
:10C2600090E00E946C5FCE0101960E94C2676B96BF
:10C270000FB6F894DEBF0FBECDBFDF91CF911F91F7
:10C280000F910895DF92EF92FF920F931F93CF9338
:10C29000DF9300D01F92CDB7DEB72091391823FF6E
:10C2A0003DC1F42EE62E8C010E9487CF882309F42D
:10C2B00081C0FF2009F48CC080913018882351F090
:10C2C0000F94820B80E692E10F949D0A80E090E04B
:10C2D0000F9477038BE49BE09A8389838FE28093AA
:10C2E0004A0B81E08B83F12C9BE1D92E80912F1892
:10C2F000F81678F4DF9CC0011124AE014D5F5F4F4A
:10C30000BE016F5F7F4F8F5D984E0E94275DF39453
:10C31000EDCF8B818B3578F4AE014D5F5F4FBE0161
:10C320006F5F7F4F84E495E10E94275D89819A8148
:10C3300001979A838983E981FA811082E09130180C
:10C3400084E0E89FF0011124EA5BF44F80913518F6
:10C3500090913618A0913718B09138188083918346
:10C36000A283B3830F94860BB80187E492E10F9404
:10C370006F0B6091301889E6689FB0011124665BED
:10C38000744F8CE392E10F946F0B409135185091EC
:10C390003618609137187091381886E392E10F943F
:10C3A000330B8AE00E94B952809130188F5F8093DE
:10C3B000301826C0FF2039F00F94860B86E292E1F8
:10C3C0000F949D0A1DC01092301882E0F82E02C012
:10C3D000FF24F3940F94860B81E292E10F949D0A5F
:10C3E00081E0F81609F497C08DE092E10F949D0A60
:10C3F000B80189E192E10F946F0B8AE00E94B95273
:10C400000E94E65DB801CE0103960F94DE048C0114
:10C41000009709F483C06B817C81EE2009F450C041
:10C4200021E0AC0184E495E10E94A56B882309F426
:10C430003FC08091551590915615A0915715B09118
:10C4400058158093311890933218A0933318B093F5
:10C45000341810923518109236181092371810921E
:10C460003818B8018FEF91E10F946F0B409131189C
:10C4700050913218609133187091341887EF91E120
:10C480000F94330B8AE00E94B95288EE91E10F9429
:10C490009D0AB80180E090E00E940A618091C61A6E
:10C4A000811102C0C80102C086EC9AE160E030C090
:10C4B000B80184ED91E10F946F0B81ED91E10FC014
:10C4C00026E5AC0184E495E10E94A56B81110AC0C8
:10C4D000B8018DEB91E10F946F0B8AEB91E10F9412
:10C4E0009D0A1CC080913918816080933918B80169
:10C4F00080E090E00E940A6110921F17B80188EA5C
:10C5000091E10F946F0B8AE00E94B95260E0C8017C
:10C510000E94A4F503C083E192E168CF0F900F90D1
:10C520000F900F90DF91CF911F910F91FF90EF909F
:10C53000DF900895CF92DF92EF92FF92CF936B013D
:10C540007C01C42F8091BB1A9091BC1AA091BD1A96
:10C55000B091BE1A8C159D05AE05BF05D1F00E94A5
:10C560004667811102C080E018C02BEB38E1B701AB
:10C57000A6018091C41A9091C51A0E94C8678823A9
:10C5800091F3C092BB1AD092BC1AE092BD1AF092FD
:10C59000BE1A81E0C1118093C31ACF91FF90EF9032
:10C5A000DF90CF9008954F925F926F927F928F921B
:10C5B0009F92AF92BF92CF92DF92EF92FF920F9332
:10C5C0001F93CF93DF93EC01423051056105710554
:10C5D00010F480E069C089859A85AB85BC85019699
:10C5E000A11DB11D84179507A607B70790F38F8982
:10C5F000803149F4852E962EA72EBB248B899C89E9
:10C60000AD89BE890FC0803221F78B889C88AD88A8
:10C61000BE88DB01CA01E7E0B695A7959795879597
:10C62000EA95D1F7880E991EAA1EBB1E2801390172
:10C630006A017B0141E0C501B4010E949A6288232E
:10C6400041F29F89903161F4DD24EE24FF249601AC
:10C65000220F331FF901E554F74E5182408211C079
:10C66000E894C7F8DD24EE24FF249601220F331F3F
:10C67000220F331FF901E554F74E40825182628246
:10C6800073829A89923080F04D815E816F817885C6
:10C69000840E951EA61EB71E8092BF1A9092C01AD5
:10C6A000A092C11AB092C21ADF91CF911F910F913F
:10C6B000FF90EF90DF90CF90BF90AF909F908F90C2
:10C6C0007F906F905F904F900895CF92DF92EF929E
:10C6D000FF920F931F93CF93DF93FC018185928587
:10C6E000A385B4850196A11DB11D84179507A607E2
:10C6F000B70710F480E061C08789803149F4BB2717
:10C70000A72F962F852FC388D488E588F6880FC079
:10C71000803281F783899489A589B6896A017B0172
:10C72000C7E0F694E794D794C794CA95D1F78C0DD7
:10C730009D1DAE1DBF1DE9016A017B018F01409166
:10C74000BB1A5091BC1A6091BD1A7091BE1A841721
:10C750009507A607B70739F040E0BC01CD010E945C
:10C760009A62882339F2F8018789803179F4B70118
:10C77000A601552766277727440F551FFA01E55470
:10C78000F74E80819181A0E0B0E012C0B701A60110
:10C790004F77552766277727440F551F440F551F9E
:10C7A000FA01E554F74E80819181A281B381BF7077
:10C7B00088839983AA83BB8381E0DF91CF911F9106
:10C7C0000F91FF90EF90DF90CF9008954F925F927E
:10C7D0006F927F92AF92BF92CF92DF92EF92FF92D1
:10C7E0000F931F93CF93DF9300D01F92CDB7DEB787
:10C7F0008C0149835A836B837C835901C12CD12CD2
:10C800007601412C82E0582E612C712C49815A818D
:10C810006B817C819E012F5F3F4FC8010E94656341
:10C82000882341F1D301C201F801058404C0880FB7
:10C83000991FAA1FBB1F0A94D2F7C80ED91EEA1E61
:10C84000FB1E49815A816B817C818789803139F453
:10C8500081E0483F5F4F6105710538F4D7CF81E033
:10C86000483F5F4F6F4F7F4088F2F501C082D18211
:10C87000E282F3820F900F900F900F90DF91CF9193
:10C880001F910F91FF90EF90DF90CF90BF90AF90EE
:10C890007F906F905F904F9008958F929F92AF928C
:10C8A000BF92CF92DF92EF92FF920F931F93CF939D
:10C8B000DF93EC018B81811102C080E078C009898F
:10C8C0001A892B893C890417150726073707A8F30F
:10C8D0006A017B01823029F4C886D986EA86FB8604
:10C8E0000DC0C114D104E104F10451F41886198675
:10C8F0001A861B861C821D821E821F8281E057C001
:10C9000088849984AA84BB84E98DFA8D258530E0DA
:10C91000275F3F4FB501A4014150510961097109D9
:10C92000022E04C076956795579547950A94D2F7DD
:10C93000D701C6010197A109B10904C0B695A79511
:10C94000979587952A95D2F784179507A607B70775
:10C9500020F089288A288B2871F44D895E896F8997
:10C96000788D4C835D836E837F834C015D018E01E6
:10C970000C5F1F4F16C0841B950BA60BB70BF5CF92
:10C980004C815D816E817F819801898D9A8D0E9495
:10C99000656391E0891A9108A108B108882309F418
:10C9A0008CCF81149104A104B10451F795CFDF918C
:10C9B000CF911F910F91FF90EF90DF90CF90BF909C
:10C9C000AF909F908F9008950F931F93CF93DF9315
:10C9D000FC012381222311F080E044C08B01EC0193
:10C9E000FB018789803139F18032B1F783E08B8395
:10C9F000F801428D538D648D758D4D8B5E8B6F8BE1
:10CA0000788F9E012F5E3F4FC8010E94E663882306
:10CA100019F31A8F098F81E08983188619861A867F
:10CA20001B861C821D821E821F82188A1C861D8600
:10CA30001E861F8617C082E08B831D8A1E8A1F8A6E
:10CA4000188EFB01808D918DA0E0B0E025E0880F6D
:10CA5000991FAA1FBB1F2A95D1F7898B9A8BAB8B85
:10CA6000BC8BD7CFDF91CF911F910F910895CF93BA
:10CA7000DF93EC0141E0611101C040E06C857D85F0
:10CA80008E859F850E949A62882341F0888920E2E2
:10CA9000829FC00111248554974E02C080E090E02F
:10CAA000DF91CF910895CF93DF93EB01FC012381B8
:10CAB000211102C080E028C02250223020F48FE2F1
:10CAC0008883198220C060E00E943765009791F347
:10CAD000FC0190E080E02EE23081303269F0883055
:10CAE00029F4DE01A90FB11D2C939F5FDE01A90F70
:10CAF000B11D30813C939F5F8F5F31968B3061F722
:10CB0000C90FD11D188281E0DF91CF9108953F9226
:10CB10004F925F926F927F928F929F92AF92BF924D
:10CB2000CF92DF92EF92FF920F931F93CF93DF93F9
:10CB3000CDB7DEB72C970FB6F894DEBF0FBECDBFD2
:10CB40005C01DC0159968D909C905A97F401818587
:10CB50009285A385B4859C01AD012F5F3F4F4F4F58
:10CB60005F4F29873A874B875C87D5011496CD9014
:10CB7000DD90ED90FC901797C114D104E104F1040D
:10CB800039F0BFEFCB1ADB0AEB0AFB0A312C07C0E6
:10CB9000F401C080D180E280F380332433942601F5
:10CBA00037011D821E821F821886F40181859285BD
:10CBB000A385B4852D813E814F815885281739077B
:10CBC0004A075B0708F064C089859A85AB85BC85F8
:10CBD0008C159D05AE05BF0550F482E0C82ED12C02
:10CBE000E12CF12C92E0492E512C612C712C9E01EC
:10CBF0002F5F3F4FB701A601C4010E9465638823E0
:10CC000009F446C089819A81AB81BC81892B8A2B2A
:10CC10008B2B41F0260137019FEF491A590A690A07
:10CC2000790A05C0C414D504E604F70491F02D81F7
:10CC30003E814F8158852F5F3F4F4F4F5F4F2D8370
:10CC40003E834F8358873FEFC31AD30AE30AF30AA0
:10CC5000ACCF0FEF1FEF2FEF3FE0B301A201C401F4
:10CC60000E94D362F82E882399F0D50114964D9135
:10CC70005D916D917C911797411551056105710585
:10CC800049F093018201C4010E94D362811102C064
:10CC9000F12C29C0D50114964D925D926D927C9233
:10CCA0001797332051F0D301C2010196A11DB11D88
:10CCB000F40180839183A283B383F50185899689EA
:10CCC000A789B08D892B8A2B8B2B69F4D5015596BA
:10CCD0004D925D926D927C92589711968C9111971E
:10CCE000806811968C938F2D2C960FB6F894DEBF2A
:10CCF0000FBECDBFDF91CF911F910F91FF90EF90AD
:10CD0000DF90CF90BF90AF909F908F907F906F906B
:10CD10005F904F903F90089540E050E0BA010C942E
:10CD20004D6461E0FC0180810E9464ED8FEF0C9402
:10CD3000B35BEF92FF921F93CF93DF9300D01F92CC
:10CD4000CDB7DEB77C01162F29833A834B835C83F2
:10CD5000FC0182810E94BF5B60E0F70180810E943C
:10CD600064ED0F942804812F80640E94B35B8C8152
:10CD70000E94B35B8B810E94B35B8A810E94B35B8C
:10CD800089810E94B35B112311F087E801C085E916
:10CD90000E94B35B1C3011F40E94B85B10E00E944B
:10CDA000B85BF701838387FF04C01F3F11F01F5F4B
:10CDB000F6CF0F900F900F900F90DF91CF911F91B2
:10CDC000FF90EF9008950F931F93CF93DF93EC01A3
:10CDD00089018C81833039F089E0440F551F661F2B
:10CDE000771F8A95D1F79A01AB0168E1CE010E94C5
:10CDF0009966811128C08EEF8EBDF801C8019E5F33
:10CE00000DB407FEFDCF20812EBD0DB407FEFDCF72
:10CE100021812EBD32968E179F0791F70DB407FE24
:10CE2000FDCF8FEF0E94B35B8FEF0E94B35B0E9438
:10CE3000B85B8B838F71853041F083E18983CE01AC
:10CE40000E94916619C086E016C00F9428048823BA
:10CE500079F020E030E0A9016DE0CE010E949966F2
:10CE6000811108C00E94B85B811104C011E005C0A7
:10CE700087E101C086E1898310E0CE010E949166BE
:10CE8000812FDF91CF911F910F910895CF938091C2
:10CE9000C31A8823B9F14091BB1A5091BC1A609112
:10CEA000BD1A7091BE1A2BEB38E18091C41A909193
:10CEB000C51A0E94E366C82F811102C0C0E023C0DA
:10CEC0004091BF1A5091C01A6091C11A7091C21A54
:10CED000411551056105710591F02BEB38E1809109
:10CEE000C41A9091C51A0E94E366882339F3109200
:10CEF000BF1A1092C01A1092C11A1092C21A109240
:10CF0000C31A01C0C1E08C2FCF910895CF93DF9356
:10CF1000EC018B81882339F1898187FF20C061E092
:10CF2000CE010E943765FC01892BE9F08081853EA6
:10CF3000D1F08B81823040F489899A89AB89BC8990
:10CF4000848F958FA68FB78F8D899E89AF89B88D75
:10CF5000938F828FB58BA48B89818F778983DF91A3
:10CF6000CF910C94466781E0888380E0DF91CF9178
:10CF70000895CF93DF93EC010E9486671B82DF91B7
:10CF8000CF910895FC01238121110C94B967089574
:10CF9000CF92DF92EF92FF920F931F93CF93DF9385
:10CFA000EC0189018C81833039F089E0440F551FF1
:10CFB000661F771F8A95D1F79A01AB0161E1CE0117
:10CFC0000E949966882339F084E08983CE010E940B
:10CFD000916680E03EC00E94F1EE6B017C012CE284
:10CFE000C20E21E0D21EE11CF11C0E94B85B8B83B3
:10CFF0008F3F61F40E94F1EEDC01CB018C199D0999
:10D00000AE09BF09B7FDF1CF81E11DC08E3FD1F45C
:10D010008FEF8EBDF801D801A150BE4F0DB407FEB1
:10D02000FDCF9EB591938EBDEA17FB07B9F70DB4FE
:10D0300007FEFDCF8EB58C930E94B85B0E94B85B53
:10D0400011E003C08FE0898310E0CE010E94916659
:10D05000812FDF91CF911F910F91FF90EF90DF9083
:10D06000CF9008952F923F924F925F926F927F924E
:10D070008F929F92AF92BF92CF92DF92EF92FF92E8
:10D080000F931F93CF93DF9300D01F92CDB7DEB7DE
:10D090009C838B834B015A01DC0113968C91811187
:10D0A00003C08FEF9FEFE3C0EB81FC81818180FFA4
:10D0B000F8CFEB81FC8181899289A389B48940856D
:10D0C000518562857385841B950BA60BB70BA50153
:10D0D00060E070E084179507A607B70708F45C01C5
:10D0E00075018B819C8104969A838983612C42E02F
:10D0F000742EE114F10409F48BC0AB81BC81189645
:10D100004D915D916D917C911B976A01B1E0DB229D
:10D11000EB81FC812381818D928D1A012B0139E0F5
:10D1200056944794379427943A95D1F7223061F476
:10D13000FC01828D938DA48DB58DBC01CD01620D56
:10D14000731D841D951D4AC0DC0114961C9111505D
:10D150001221C114D10401F511111EC0452B462B1B
:10D16000472B59F4EB81FC8185899689A789B08D7D
:10D1700084839583A683B7830FC0AB81BC8114964B
:10D180004D915D916D917C91179729813A810E9413
:10D190006563882309F485CFEB81FC81218D328D75
:10D1A00084819581A681B7810297A109B109F9010E
:10D1B000058404C0880F991FAA1FBB1F0A94D2F7C9
:10D1C0004685578560897189840F951FA61FB71FF3
:10D1D000BC01CD01610F711D811D911D93012C19A1
:10D1E0003D0987012E153F0508F489010115F2E07C
:10D1F0001F0779F52091BB1A3091BC1A4091BD1AD6
:10D200005091BE1A621773078407950719F421C05D
:10D21000C5012DC09401AB01BC018091C41A90914D
:10D22000C51A0E94C867882309F43BCF800E911E5F
:10D23000EB81FC8180859185A285B385800F911F4C
:10D24000A11DB11D80879187A287B387E01AF10ADB
:10D2500050CF40E00E949A62882309F422CFB601A1
:10D260006554774EA801C4010F94562EDFCF0F905E
:10D270000F900F900F90DF91CF911F910F91FF9022
:10D28000EF90DF90CF90BF90AF909F908F907F9066
:10D290006F905F904F903F902F900895DF92EF92A4
:10D2A000FF920F931F93CF93DF938C01EB017A01D1
:10D2B0008DE0D82E40E250E0BE01C8010E943268E5
:10D2C0008032910539F021E0892B09F420E0822F8A
:10D2D000819544C028812223C9F1253E11F02E32C8
:10D2E00031F4E114F10431F3F7011082E3CFE114DA
:10D2F000F10441F13B853F733F3021F54A8D5B8D51
:10D30000452B01F52F713FEF320F3530D8F430E067
:10D3100021503109D29EC001D39E900D1124D70116
:10D32000A80FB91FFE0120E0AD01253088F431813E
:10D330003D932F5F32962D30C1F7288126FF02C022
:10D34000FA0115862B8523FDB5CF08C080E006C005
:10D350002B3010F43481ECCF3681EACFDF91CF91BE
:10D360001F910F91FF90EF90DF9008954F925F9281
:10D370006F927F929F92AF92BF92CF92DF92EF9285
:10D38000FF920F931F93CF93DF931F92CDB7DEB71A
:10D390008C017B015A01C22EDB0159968D919C9123
:10D3A0005A97F801928F818FCB010E948C66912C45
:10D3B000F70180859185A285B3854189528963896A
:10D3C000748984179507A607B70708F060C025E0A1
:10D3D000B695A795979587952A95D1F7F82FFF7061
:10D3E000DF2ED70113968C91823008F460C041E0A3
:10D3F00050E0BE016F5F7F4FC7010E943268019706
:10D4000019F4898190E002C08FEF9FEF019609F433
:10D410004EC0F70180859185A285B3854F96A11DE9
:10D42000B11D80879187A287B387F0E2DF9EB001AC
:10D4300011246554774E61157105C9F1DB018C919A
:10D44000882319F0853EC1F46CC191100EC0809103
:10D45000BB1A9091BC1AA091BD1AB091BE1AF801E6
:10D4600084879587A687B787D08ADB018C9188232C
:10D4700061F0992493949CCF4BE050E0C5010F9448
:10D48000492E892B09F094CF14C0992493948C2DA4
:10D490008274823461F4992009F48BC0F801D08839
:10D4A00061E0C8010E943765009709F00DC180E076
:10D4B0003BC1C7FCFCCFF0E2DF9EA00111249A0122
:10D4C0002554374ED9011B968C91817121F08C2DFA
:10D4D000827109F06AC08091BB1A9091BC1AA09128
:10D4E000BD1AB091BE1AF80184879587A687B787C1
:10D4F000D08ACA018554974E7C01DC0154964D9127
:10D500005C91559760E070E0DA0199278827858B58
:10D51000968BA78BB08FF701428D538D60E070E042
:10D52000482B592B6A2B7B2BD80155964D935D9335
:10D530006D937C935897F9018385887161F4F701A5
:10D54000848D958DA68DB78DF801818B928BA38BE1
:10D55000B48B81E010C0803141F598012F5E3F4FC0
:10D56000D80159968D919C915A970E94E663882321
:10D57000E1F084E0F80183838C2D8F70D80111963F
:10D580008C931197F80114821582168217821896CF
:10D590001D921D921D921C921B97C4FEB5C0C8011E
:10D5A0000F944C048111B0C082CFD80113961C9205
:10D5B0007ECFD70113968C911397823009F477CFE1
:10D5C00051968D919D910D90BC91A02D803E9F4FC5
:10D5D000AF41B10508F06BCFC7010E948765882372
:10D5E00009F465CF0E944667882309F460CFD7010C
:10D5F00059962D913C915A9714968D919D910D902D
:10D60000BC91A02D0297A109B109F901058404C0BC
:10D61000880F991FAA1FBB1F0A94D2F7468457840C
:10D6200060887188480E591E6A1E7B1E81E08093B7
:10D63000C31A4092BB1A5092BC1A6092BD1A7092E3
:10D64000BE1A80E092E0EBEBF8E1DF019C011D9255
:10D6500021503040E1F7DD24D394D7015996ED9164
:10D66000FC915A978481D81698F42BEB38E1B301DA
:10D67000A2014D0D511D611D711D8091C41A909123
:10D68000C51A0E94E366882309F411CFD394E5CF2D
:10D6900080E092E0A0E0B0E0058404C0880F991F0C
:10D6A000AA1FBB1F0A94D2F7F701418952896389E7
:10D6B0007489840F951FA61FB71F818B928BA38B34
:10D6C000B48B8BEB98E1D12C20E2DC011D922A95E2
:10D6D000E9F72BE0F501DC0101900D922A95E1F7C5
:10D6E00021E238E2FC01318B208B40E058E0578783
:10D6F0004687338B228B318F208F578B468B0E942E
:10D7000046678111D8CED3CEC5FE09C0F801418944
:10D71000528963897489C8010E944D6405C081E003
:10D7200003C09110A6CE93CE0F90DF91CF911F91A1
:10D730000F91FF90EF90DF90CF90BF90AF909F90B0
:10D740007F906F905F904F9008952F923F924F92ED
:10D750005F926F927F928F929F92AF92BF92CF9281
:10D76000DF92EF92FF920F931F93CF93DF93CDB78A
:10D77000DEB7C254D1090FB6F894DEBF0FBECDBFDD
:10D780004C015B016A01322E19821C821C8E1F8E95
:10D790006115710511F410E0A6C0FC0183818111AF
:10D7A000FACFFA0180818F3209F09BC0F5018381A5
:10D7B0008250823010F485010CC0F501618D728DAC
:10D7C000CE014C960E94E464882329F38E01045E06
:10D7D0001F4FC6016C010196F60120812F32D1F353
:10D7E000CE0101967C013C012E019CE1490E511CA9
:10D7F0002396EFAE23972F2C9BE09150E7E3F0E0C8
:10D80000EC0FFD1FE90FF11D80E280839111F5CF30
:10D81000960147E0D9018D91882369F18F3259F142
:10D820008E3239F44A3009F4B6CF98E04AE09D01CF
:10D83000F1CFEAEDF2E12491222321F03196821317
:10D84000FACFA9CF491708F4A6CF813208F4A3CFA5
:10D850008F3709F4A0CF21E0290FE7E3F0E0EC0FC8
:10D86000FD1FE90FF11D9FE9980F9A3108F48052CE
:10D870008083922FDCCF8FA9803209F48CCF69018D
:10D88000F90180812F5F3F4F8F32C9F38823F9F070
:10D8900021E0AE01495C5F4FB801C7010E94B66943
:10D8A000882309F478CF0A151B0519F0C8010E94D6
:10D8B000B9676E147F0441F023969FAD2397822DA4
:10D8C0008701E92EF82E98CF942D852DF9CF232DA1
:10D8D000AE01495C5F4FB801C4010E94B669182FC0
:10D8E00002C08B017DCFCE014C960E94C267CE0153
:10D8F00001960E94C267812FCE5BDF4F0FB6F8946E
:10D90000DEBF0FBECDBFDF91CF911F910F91FF9072
:10D91000EF90DF90CF90BF90AF909F908F907F90CF
:10D920006F905F904F903F902F900895CF93C82FA6
:10D930000F94860B84E50E94B9526C2F70E080E052
:10D9400090E00E942D5380E20E94B95288EC92E14F
:10D95000CF910D949D0A2F923F924F925F926F92BA
:10D960007F928F929F92AF92BF92CF92DF92EF926F
:10D97000FF920F931F93CF93DF93CDB7DEB7CD59AF
:10D98000D1090FB6F894DEBF0FBECDBF4B015A01CF
:10D990006901ED96FFAEEEAEED97DC012D913D9164
:10D9A0004D915C91E3962CAF3DAF4EAF5FAFE397E7
:10D9B00020914C1130914D1140914E1150914F11C9
:10D9C000E3966CAD7DAD8EAD9FADE3970F949A2439
:10D9D0000F94972DA7966CAF7DAF8EAF9FAFA79793
:10D9E00065966CAF7DAF8EAF9FAF6597D4012D91DB
:10D9F0003D914D915C91AF962CAF3DAF4EAF5FAF77
:10DA0000AF97209150113091511140915211509186
:10DA10005311AF966CAD7DAD8EAD9FADAF970F94AA
:10DA20009A240F94972D2B013C0169966CAF7DAF22
:10DA30008EAF9FAF6997D5012D913D914D915C912E
:10DA4000E7962CAF3DAF4EAF5FAFE79720915411F3
:10DA5000309155114091561150915711E7966CAD88
:10DA60007DAD8EAD9FADE7970F949A240F94972DBF
:10DA70004B015C016D966CAF7DAF8EAF9FAF6D9724
:10DA8000D6012D913D914D915C91AB962CAF3DAF60
:10DA90004EAF5FAFAB972091581130915911409123
:10DAA0005A1150915B11AB966CAD7DAD8EAD9FADB3
:10DAB000AB970F949A240F94972D6B017C01A1963C
:10DAC0006CAF7DAF8EAF9FAFA197E3962CAD3DAD10
:10DAD0004EAD5FADE39725962CAF3DAF4EAF5FAF38
:10DAE0002597AF968CAD9DADAEADBFADAF972996E6
:10DAF0008CAF9DAFAEAFBFAF2997E7962CAD3DADD4
:10DB00004EAD5FADE7972D962CAF3DAF4EAF5FAFFB
:10DB10002D97AB968CAD9DADAEADBFADAB9761967D
:10DB20008CAF9DAFAEAFBFAF61978091371183FFD0
:10DB300016C0C0925D16D0925E16E0925F16F0920B
:10DB40006016AB962CAD3DAD4EAD5FADAB9720935F
:10DB50004D1630934E1640934F16509350168091A9
:10DB6000351190913611892B11F00C94817DD801DB
:10DB7000BC91C158DF4FB883CF57D040F801F18135
:10DB8000CD57DF4FF883C358D040D8011296BC91CF
:10DB9000C957DF4FB883C758D040F801038180913F
:10DBA0002B1690912C16891B8F708F3021F480E0FA
:10DBB0000E94E553F4CFF0912B16C556DF4FF88342
:10DBC000CB59D04080912B16282E312C80915116A4
:10DBD00090915216A0915316B0915416A7962CAD61
:10DBE0003DAD4EAD5FADA797281B390B4A0B5B0BC4
:10DBF000A7962CAF3DAF4EAF5FAFA797809155165C
:10DC000090915616A0915716B0915816481A590A75
:10DC10006A0A7B0A8091591690915A16A0915B1658
:10DC2000B0915C16A5019401281B390B4A0B5B0BC4
:10DC3000AF962CAF3DAF4EAF5FAFAF9780915D1603
:10DC400090915E16A0915F16B0916016A7019601A3
:10DC5000281B390B4A0B5B0BE3962CAF3DAF4EAF45
:10DC60005FAFE397232B242B252B09F48CC08091E5
:10DC7000E90B811133C06091EE0B7091EF0B809135
:10DC8000F00B9091F10B0F94962C2091190230918A
:10DC90001A026217730714F5C0925D16D0925E16D1
:10DCA000E0925F16F0926016AB968CAD9DADAEAD76
:10DCB000BFADAB9780934D1690934E16A0934F1621
:10DCC000B09350160F94860B8FE193E10F949D0A49
:10DCD000E3961CAE1DAE1EAE1FAEE397E3966CAD91
:10DCE0007DAD8EAD9FADE3970F943B24209115023F
:10DCF0003091160240911702509118020F949A2405
:10DD00004B015C0120E030E0A9010F948A2D87FFD0
:10DD100004C0B7FAB094B7F8B09420E030E04AEF0E
:10DD200053E4609158117091591180915A1190915A
:10DD30005B110F949A24A50194010F94342487FF5A
:10DD400022C0C0925D16D0925E16E0925F16F092ED
:10DD50006016AB962CAD3DAD4EAD5FADAB9720934D
:10DD60004D1630934E1640934F16509350160F9405
:10DD7000860B80E093E10F949D0AE3961CAE1DAEE6
:10DD80001EAE1FAEE397A7968CAD9DADAEADBFADF9
:10DD9000A7978827B7FD83959927AA27BB27182F10
:10DDA00077FC1260AF968CAD9DADAEADBFADAF97B9
:10DDB000B7FD1460E3962CAD3DAD4EAD5FADE3977E
:10DDC00057FD1860E3966CAD7DAD8EAD9FADE397CA
:10DDD0000F943B24209115023091160240911702B6
:10DDE000509118020F949A246B017C0120E030E0DE
:10DDF000A9010F948A2D87FF04C0C701B60190586E
:10DE000002C0C701B60120E030E040E05FE30F94BC
:10DE10002A2B0F949D2CEB966CAF7DAF8EAF9FAFEE
:10DE2000EB9783E5829DF001839DF00D1124EB5F5C
:10DE3000F34F108215ABA7968CAC9DACAEACBFACCB
:10DE4000A797B7FE08C0B094A09490948094811CCA
:10DE5000911CA11CB11C83E5829DF001839DF00DF6
:10DE60001124EB5FF34F858A968AA78AB08EAB9612
:10DE70004CAE5DAE6EAE7FAEAB9777FE0DC0882721
:10DE80009927DC0184199509A609B709AB968CAFCF
:10DE90009DAFAEAFBFAFAB9783E5829DF001839D91
:10DEA000F00D1124EB5FF34FAB962CAD3DAD4EADB5
:10DEB0005FADAB97218F328F438F548FAF968CAD70
:10DEC0009DADAEADBFADAF97E7968CAF9DAFAEAF9A
:10DED000BFAFE797B7FF0DC0B095A095909581951E
:10DEE0009F4FAF4FBF4FE7968CAF9DAFAEAFBFAF69
:10DEF000E79783E5829DF001839DF00D1124EB5F90
:10DF0000F34FE7962CAD3DAD4EAD5FADE797258F56
:10DF1000368F478F50A3A7966CAD7DAD8EAD9FAD6C
:10DF2000A7970F943B242091D90B3091DA0B4091A5
:10DF3000DB0B5091DC0B0F949A24A7966CAF7DAF4E
:10DF40008EAF9FAFA79769AB7AAB8BAB9CABC3018E
:10DF5000B2010F943B242091DD0B3091DE0B4091F8
:10DF6000DF0B5091E00B0F949A242B013C016DAB19
:10DF70007EAB8FAB98AFAF966CAD7DAD8EAD9FADE8
:10DF8000AF970F943B242091E10B3091E20B40912D
:10DF9000E30B5091E40B0F949A24AF966CAF7DAFD6
:10DFA0008EAF9FAFAF9769AF7AAF8BAF9CAF209129
:10DFB000E50B3091E60B4091E70B5091E80BC70160
:10DFC000B6010F949A246B017C0121966CAF7DAF52
:10DFD0008EAF9FAF219736E083169104A104B10460
:10DFE0001CF5AB968CAD9DADAEADBFADAB970697B6
:10DFF000A105B105CCF4E7962CAD3DAD4EAD5FADBE
:10E00000E797263031054105510574F420E030E0F2
:10E01000A901C701B6010F948A2D87FF16C0F7FA30
:10E02000F094F7F8F09411C0ED96AEADBFADED975A
:10E03000CD90DD90ED90FC9020E030E0A901C7018B
:10E04000B6010F943424882369F083E5829DF001A2
:10E05000839DF00D1124EB5FF34FC586D686E786CE
:10E06000F08A38C0A7962CAD3DAD4EAD5FADA797F9
:10E07000CA01B9010F949A246B017C01A30192019A
:10E08000C301B2010F949A249B01AC01C701B601F0
:10E090000F942A2B6B017C01AF962CAD3DAD4EAD9C
:10E0A0005FADAF97CA01B9010F949A249B01AC01EF
:10E0B000C701B6010F942A2B0F94D82D23E5229D7A
:10E0C000F001239DF00D1124EB5FF34F65877687F8
:10E0D0008787908B83E5829DF001839DF00D11244D
:10E0E000EB5FF34FEB962CAD3DAD4EAD5FADEB97D7
:10E0F00021A332A343A354A3582D492D3A2D2B2DF0
:10E10000AB968CAD9DADAEADBFADAB978816990605
:10E11000AA06BB0660F4A8965FADA897A9964FAD76
:10E12000A997AA963FADAA97AB962FADAB97852F2F
:10E13000942FA32FB22FE7962CAD3DAD4EAD5FAD22
:10E14000E79782179307A407B50710F4DA01C9010E
:10E15000EB962CAD3DAD4EAD5FADEB9782179307BF
:10E16000A407B50710F4DA01C90123E5229DF001E7
:10E17000239DF00D1124EB5FF34F85A396A3A7A376
:10E18000B0A70697A105B10510F40C941C7EDF0121
:10E19000AF5ABF4F8091D70B8C93EE5AFF4F8091AF
:10E1A000D80B808389288A288B2809F05F9883E51B
:10E1B000829DF001839DF00D1124EB5FF34F818D63
:10E1C000928DA38DB48D892B8A2B8B2B09F08A9885
:10E1D00083E5829DF001839DF00D1124EB5FF34FE9
:10E1E000858D968DA78DB0A1892B8A2B8B2B29F03D
:10E1F00080910801817080930601EB968CAD9DADF6
:10E20000AEADBFADEB97892B8A2B8B2B11F40C9401
:10E21000837D80919011882319F081508093901113
:10E22000129880E280939011D0907811E09079114B
:10E23000F0907A1110917B112D2D3E2D4F2D512FE5
:10E24000C158DF4F6881CF57D040CD57DF4F78811D
:10E25000C358D040C957DF4F8881C758D040902F4E
:10E260000F94342487FF10C0C158DF4FD882CF5796
:10E27000D040CD57DF4FE882C358D040C957DF4F59
:10E28000F882C758D040012F83E5829DF001839D1D
:10E29000F00D1124EB5FF34F45845684678470883A
:10E2A000A301920160E070E080E89FE30F94242CCA
:10E2B000EF966CAF7DAF8EAF9FAFEF97C158DF4F3A
:10E2C0002881CF57D040CD57DF4F3881C358D04039
:10E2D000C957DF4F4881C758D040502F0F949A2418
:10E2E0004B015C0180912B1690912916891B8F7030
:10E2F000C557DF4F8883CB58D040A501940160E01B
:10E3000074E284E799E40F94242C0F94972D6B0109
:10E310007C01C557DF4F8881CB58D0408250863072
:10E32000D0F58091481190914911A0914A11B09176
:10E330004B11C816D906EA06FB0668F58C199D092B
:10E34000AE09BF09BC01CD01660F771F881F991F59
:10E35000C557DF4FA881CB58D0400A2F10E020E0EE
:10E3600030E0A90198010F948A2ACA01B9010F94DB
:10E3700039240F94972D6C0D7D1D8E1D9F1D0F94BC
:10E3800039249B01AC0160E074E284E799E40F94C6
:10E39000242C4B015C01A5019401C301B2010F942F
:10E3A0009A249B01AC010F949A24C157DF4F6883D4
:10E3B00079838A839B83CF58D04083E5829D8001F7
:10E3C000839D100D11240B5F134FC157DF4F288120
:10E3D00039814A815B81CF58D040D80111962D9365
:10E3E0003D934D935C93149795962D913D914D914E
:10E3F0005C919897C158DF4F288339834A835B83A8
:10E40000CF57D040CA01B9010F943924CD57DF4FFF
:10E41000688379838A839B83C358D0409B01AC0176
:10E42000C501B4010F949A240F94082C0F949D2CCD
:10E43000CD56DF4F688379838A839B83C359D0404D
:10E44000F801EF5BFF4F60837183828393838E01BA
:10E450000F5C1F4FFE01B196C957DF4FF983E88368
:10E46000C758D0402CE531E1C756DF4F39832883A8
:10E47000C959D040A801405F5F4FC456DF4F598350
:10E480004883CC59D040C956DF4FF983E883C75938
:10E49000D040A4961FAEA497A8961FAEA89750E8A8
:10E4A000AC965FAFAC978FE3E4968FAFE497D8015B
:10E4B0002D913D914D915D918D01C501B4010F9458
:10E4C0009A246B017C01C956DF4FE881F981C75955
:10E4D000D0406193719381939193C956DF4FF98333
:10E4E000E883C759D04020E030E0A9010F948A2D7D
:10E4F00087FF04C0F7FAF094F7F8F094C756DF4F9F
:10E50000A881B981C959D0404D905D906D907D90A2
:10E51000C756DF4FB983A883C959D040A7019601D8
:10E52000C301B2010F94342487FF24C0A7019601D0
:10E53000C301B2010F94242C7B016C01A4962FAD72
:10E54000A497A8963FADA897AC964FADAC97E4962C
:10E550005FADE4970F94342487FF0CC0A496EFAE10
:10E56000A497A896FFAEA897AC96CFAEAC97E496CA
:10E57000DFAEE497C456DF4FE881F981CC59D04033
:10E58000E017F10709F093CF20E030E040E85FE3C7
:10E59000A4966FADA497A8967FADA897AC968FADC3
:10E5A000AC97E4969FADE4970F94342487FF84C022
:10E5B0008E010F5C1F4FA4962FADA497A8963FAD78
:10E5C000A897AC964FADAC97E4965FADE497C9576A
:10E5D000DF4FA881B981C758D0406D917D918D9151
:10E5E0009C910F949A24C957DF4FE881F981C7584D
:10E5F000D0406193719381939193C957DF4FF98311
:10E60000E883C758D0400E171F07A9F623E5229DBF
:10E61000C001239D900D11249C012B5F334F790184
:10E6200089010F5B1F4FCD56DF4F688179818A8149
:10E630009B81C359D0400F943924A4962FADA49741
:10E64000A8963FADA897AC964FADAC97E4965FAD5A
:10E65000E4970F949A240F949D2CD8016D937D9389
:10E660008D939C931397A4962FADA497A8963FAD36
:10E67000A897AC964FADAC97E4965FADE497A4969F
:10E680006FADA497A8967FADA897AC968FADAC97C9
:10E69000E4969FADE4970F949A24C157DF4F2881E9
:10E6A00039814A815B81CF58D0400F949A24F70179
:10E6B0006183728383839483CD57DF4F28813981AF
:10E6C0004A815B81C358D040EF966CAD7DAD8EAD75
:10E6D0009FADEF970F949A24A7966CAF7DAF8EAF46
:10E6E0009FAFA79783E5829D8001839D100D112424
:10E6F0000B5F134FD80155968D909D90AD90BC90B7
:10E70000589781149104A104B10469F559968D912B
:10E710009D910D90BC91A02D892B8A2B8B2B19F5E7
:10E72000F801858D968DA78DB0A1892B8A2B8B2B17
:10E73000D1F420917011309171114091721150916A
:10E740007311A7966CAD7DAD8EAD9FADA7970F945D
:10E750009A240F94082C0F949D2C2B013C01D80176
:10E76000D6961C923FC3EB962CAD3DAD4EAD5FAD42
:10E77000EB97232B242B252B49F020916C11309102
:10E780006D1140916E1150916F1108C0209174115C
:10E79000309175114091761150917711A7966CAD1B
:10E7A0007DAD8EAD9FADA7970F949A240F94082C42
:10E7B0000F949D2C2B013C01EB968CAD9DADAEAD25
:10E7C000BFADEB97892B8A2B8B2BD9F020E030E063
:10E7D000A9016091010C7091020C8091030C909141
:10E7E000040C0F943424882361F081E0E3962CAD6F
:10E7F0003DAD4EAD5FADE397121613061406150638
:10E800000CF080E093E5929D8001939D100D112402
:10E810000B5F134FD801D6968C93882309F4CCC094
:10E820002091411630914216409143165091441662
:10E8300025966CAD7DAD8EAD9FAD25970F94292BA0
:10E84000AB966CAF7DAF8EAF9FAFAB972091451667
:10E8500030914616409147165091481629966CAD56
:10E860007DAD8EAD9FAD29970F94292BE3966CAFAC
:10E870007DAF8EAF9FAFE3972091491630914A1636
:10E8800040914B1650914C162D966CAD7DAD8EADD2
:10E890009FAD2D970F94292B6B017C01AB962CAD6E
:10E8A0003DAD4EAD5FADAB97CA01B9010F949A244F
:10E8B000AB966CAF7DAF8EAF9FAFAB97E3962CADB1
:10E8C0003DAD4EAD5FADE397CA01B9010F949A24F7
:10E8D0009B01AC01AB966CAD7DAD8EAD9FADAB97A2
:10E8E0000F942A2BAB966CAF7DAF8EAF9FAFAB97DB
:10E8F000A7019601C701B6010F949A249B01AC01B0
:10E90000AB966CAD7DAD8EAD9FADAB970F942A2BC2
:10E910000F94D82D6B017C0120914D1630914E162D
:10E9200040914F165091501661966CAD7DAD8EADF5
:10E930009FAD61970F94292BA70196010F94242C6A
:10E940006B017C01F801FD96608371838283938360
:10E9500020E030E040E450E40F948A2D18161CF4B7
:10E96000F80116AA29C02091010C3091020C4091A7
:10E97000030C5091040CC701B6010F949A249B011B
:10E98000AC016091D30B7091D40B8091D50B909119
:10E99000D60B0F94242CA7962CAD3DAD4EAD5FAD9C
:10E9A000A7970F949A240F949D2C641575058605DE
:10E9B000970510F42B013C018091CF0B9091D00B67
:10E9C000A091D10BB091D20BC158DF4F2881398172
:10E9D0004A815B81CF57D04082179307A407B507C0
:10E9E00008F4DCC081149104A104B10411F1609118
:10E9F000BF0B7091C00B8091C10B9091C20B64153D
:10EA0000750586059705A8F40F947A2A6B017C0199
:10EA1000A5019401C301B2010F947A2AC616D70644
:10EA2000E806F90630F4C701B6010F948A2A2901D5
:10EA30003A0183E5829DF001839DF00D1124EB5F87
:10EA4000F34FC18CD28CE38CF48CC114D104E1045B
:10EA5000F10451F16091C30B7091C40B8091C50B0F
:10EA60009091C60B6415750586059705E8F4C158A5
:10EA7000DF4F288139814A815B81CF57D0400F9485
:10EA80007A2A4B015C01A7019601C301B2010F94E0
:10EA90007A2A86169706A806B90630F4C501B4018D
:10EAA0000F948A2A29013A0183E5829DF001839D12
:10EAB000F00D1124EB5FF34FC58CD68CE78CF0A0E2
:10EAC000C114D104E104F10451F16091C70B7091BC
:10EAD000C80B8091C90B9091CA0B6415750586050A
:10EAE0009705E8F4C158DF4F288139814A815B815D
:10EAF000CF57D0400F947A2A4B015C01A7019601B1
:10EB0000C301B2010F947A2A86169706A806B906A1
:10EB100030F4C501B4010F948A2A29013A0183E532
:10EB2000829DF001839DF00D1124EB5FF34FC1A096
:10EB3000D2A0E3A0F4A0C114D104E104F10409F4CB
:10EB400051C16091CB0B7091CC0B8091CD0B90910A
:10EB5000CE0B641575058605970508F043C1C158AD
:10EB6000DF4F288139814A815B81CF57D0400F9494
:10EB70007A2A4B015C01A7019601C301B2010F94EF
:10EB80007A2A86169706A806B90608F02BC1C50191
:10EB9000B4010F948A2A29013A0124C181149104F5
:10EBA000A104B104D9F16091BF0B7091C00B8091A9
:10EBB000C10B9091C20B641575058605970570F51C
:10EBC0000F943924CD57DF4F288139814A815B81E9
:10EBD000C358D0400F949A246B017C01C501B40145
:10EBE0000F9439244B015C01C301B2010F94392405
:10EBF000A50194010F949A249B01AC01C701B601B1
:10EC00000F94342487FF0AC0A5019401C701B601FF
:10EC10000F94242C0F949D2C2B013C0183E5829DA5
:10EC2000F001839DF00D1124EB5FF34F818C928CEA
:10EC3000A38CB48C81149104A104B104D9F1609126
:10EC4000C30B7091C40B8091C50B9091C60B6415DA
:10EC500075058605970570F50F943924CD57DF4F5C
:10EC6000288139814A815B81C358D0400F949A240E
:10EC70006B017C01C501B4010F9439244B015C0187
:10EC8000C301B2010F943924A50194010F949A2471
:10EC90009B01AC01C701B6010F94342487FF0AC061
:10ECA000A5019401C701B6010F94242C0F949D2C4B
:10ECB0002B013C0183E5829DF001839DF00D112421
:10ECC000EB5FF34F858C968CA78CB0A081149104D8
:10ECD000A104B104D9F16091C70B7091C80B809168
:10ECE000C90B9091CA0B641575058605970570F5DB
:10ECF0000F943924CD57DF4F288139814A815B81B8
:10ED0000C358D0400F949A246B017C01C501B40113
:10ED10000F9439244B015C01C301B2010F943924D3
:10ED2000A50194010F949A249B01AC01C701B6017F
:10ED30000F94342487FF0AC0A5019401C701B601CE
:10ED40000F94242C0F949D2C2B013C0183E5829D74
:10ED5000F001839DF00D1124EB5FF34F81A092A091
:10ED6000A3A0B4A081149104A104B104D9F16091CD
:10ED7000CB0B7091CC0B8091CD0B9091CE0B641589
:10ED800075058605970570F50F943924CD57DF4F2B
:10ED9000288139814A815B81C358D0400F949A24DD
:10EDA0006B017C01C501B4010F9439244B015C0156
:10EDB000C301B2010F943924A50194010F949A2440
:10EDC0009B01AC01C701B6010F94342487FF0AC030
:10EDD000A5019401C701B6010F94242C0F949D2C1A
:10EDE0002B013C0183E5829D8001839D100D112440
:10EDF0000B5F134FF801E35BFF4F40825182628249
:10EE00007382C301B2010F9439246B017C01A79670
:10EE10002CAD3DAD4EAD5FADA7970F94242CE7967A
:10EE20006CAF7DAF8EAF9FAFE797D80151966D93D2
:10EE30007D938D939C9354972DEB37E346E051E4FB
:10EE4000C701B6010F949A240F949D2CF80161AB71
:10EE500072AB83AB94AB86A9882381F1FD962081A8
:10EE60003181428153816091010C7091020C80913B
:10EE7000030C9091040C0F949A24E7962CAD3DADB1
:10EE80004EAD5FADE7970F949A24209158113091C1
:10EE9000591140915A1150915B110F949A249B0182
:10EEA000AC0160E074E284EF99E40F94242C0F9499
:10EEB0009D2CD801D8967C936E93D79729A93AA90F
:10EEC0004BA95CA9EF966CAD7DAD8EAD9FADEF9774
:10EED0000F949A24EB966CAF7DAF8EAF9FAFEB97FC
:10EEE000698B7A8B8B8B9C8B2DA93EA94FA958AD32
:10EEF000EF966CAD7DAD8EAD9FADEF970F949A24DC
:10EF00002B013C016D8B7E8B8F8B988F29AD3AAD99
:10EF10004BAD5CADEF966CAD7DAD8EAD9FADEF971B
:10EF20000F949A244B015C01698F7A8F8B8F9C8F91
:10EF300021962CAD3DAD4EAD5FAD2197EF966CADFA
:10EF40007DAD8EAD9FADEF970F949A24EF966CAF89
:10EF50007DAF8EAF9FAFEF976D8F7E8F8F8F98A312
:10EF6000C557DF4FB881CB58D040BB2309F4DBC273
:10EF7000E0912D16A496EFAFA497F0912E16A896C7
:10EF8000FFAFA89720912F16E0962FAFE097309112
:10EF90003016AC963FAFAC972DEB37E346E855E320
:10EFA000BF01E0968FADE097AC969FADAC970F9404
:10EFB000342487FDB8C28091801190918111A09175
:10EFC0008211B0918311C158DF4F88839983AA833E
:10EFD000BB83CF57D040209184113091851140914F
:10EFE000861150918711CD57DF4F288339834A838B
:10EFF0005B83C358D0408091881190918911A09172
:10F000008A11B0918B11C957DF4F88839983AA83E6
:10F01000BB83C758D04020918C1130918D11409105
:10F020008E1150918F11C557DF4F288339834A8342
:10F030005B83CB58D040C158DF4F688179818A818A
:10F040009B81CF57D0409058EB962CAD3DAD4EAD47
:10F050005FADEB970F949A246B017C01CD57DF4F86
:10F06000288139814A815B81C358D040C301B201F4
:10F070000F949A249B01AC01C701B6010F94292B70
:10F080006B017C01C957DF4F288139814A815B813F
:10F09000C758D040C501B4010F949A249B01AC011C
:10F0A000C701B6010F94292B6B017C01C557DF4FB7
:10F0B000288139814A815B81CB58D040EF966CAD75
:10F0C0007DAD8EAD9FADEF970F949A249B01AC015F
:10F0D000C701B6010F94292B6B017C012FEE3FEF86
:10F0E0004FE75FE30F948A2D18160CF4BEC12FEE84
:10F0F0003FEF4FE75FEBC701B6010F94342487FF62
:10F1000008C03FEEC32EDD24DA943FE7E32E3FEB49
:10F11000F32EC158DF4F288139814A815B81CF5757
:10F12000D040EB966CAD7DAD8EAD9FADEB970F945F
:10F13000292B69837A838B839C83CD57DF4F28816A
:10F1400039814A815B81C358D040C301B2010F9419
:10F15000292B6D837E838F839887C957DF4F288142
:10F1600039814A815B81C758D040C501B4010F94F1
:10F17000292B69877A878B879C87C557DF4F288122
:10F1800039814A815B81CB58D040EF966CAD7DAD23
:10F190008EAD9FADEF970F94292B6D877E878F875C
:10F1A000988BAE014F5F5F4FE9965FAF4EAFE99727
:10F1B000CE014196A3969FAF8EAFA3978A01812C73
:10F1C000912C5401D8014D905D906D907D908D01F2
:10F1D00020E030E0A901C301B2010F943424882358
:10F1E00071F0A3019201C301B2010F949A249B0113
:10F1F000AC01C501B4010F942A2B4B015C01A3960D
:10F20000EEADFFADA397E017F107E1F6C501B4013C
:10F210000F94D82D9B01AC0160E070E080E89FE383
:10F220000F94242C4B015C01E9960EAD1FADE997BC
:10F23000A5019401D8016D917D918D919C910F94C0
:10F240009A24F80161937193819391938F01A3960E
:10F250002EAD3FADA3972E173F0751F708E311E1FD
:10F26000E4965FACE497E5966FACE597E6967FACE5
:10F27000E697E7964FACE797E996AEADBFADE99755
:10F280008D909D90AD90BD90E996BFAFAEAFE997E0
:10F2900020E030E0A901C501B4010F943424882393
:10F2A00031F1F80160817181828193810F94392459
:10F2B000A50194010F94242C4B015C0120E030E067
:10F2C000A9010F948A2D87FF04C0B7FAB094B7F84C
:10F2D000B094252D362D472D542DC501B4010F9422
:10F2E000342487FF04C0582C692C7A2C4B2C0C5FDB
:10F2F0001F4FA3962EAD3FADA397E9964EAD5FADE0
:10F30000E9972417350709F0B7CFA701960160E008
:10F3100070E080E89FE30F94292B20E030E040E08C
:10F320005FE30F949A240F94D82D4B015C01209138
:10F33000BB0B3091BC0B4091BD0B5091BE0B652DAA
:10F34000762D872D942D0F949A24A50194010F9466
:10F350009A24EB966CAF7DAF8EAF9FAFEB97A50174
:10F36000940160E070E080E89FE30F94292B9B01FB
:10F37000AC01EB966CAD7DAD8EAD9FADEB970F9470
:10F38000242CE8966FAFE897EC967FAFEC978C0152
:10F3900083E5829DF001839DF00D1124EB5FF34F17
:10F3A00085849684A784B08820E030E040E85FE35D
:10F3B000C501B4010F94342487FF61C0A7019601F1
:10F3C000C701B6010F949A2423EC38EB42E35FEBBC
:10F3D0000F949A2423EF36E64FE55FE30F94292B31
:10F3E000A70196010F949A242BED3FE049EC5FE3CF
:10F3F0000F942A2B2CEE31E548E35EE30F94292B82
:10F400006B017C0124EE3BEC46E150E40F948A2D25
:10F410001816ACF5A70196016BED7FE089E490E446
:10F420000F94292B9B01AC01C501B4010F94242C2E
:10F43000252D362D472D542D0F949A246B017C01D8
:10F440009B01AC01E8966FADE897EC967FADEC9729
:10F45000C8010F948A2D181694F4E896CFAEE89759
:10F46000EC96DFAEEC9787010AC05BE0E8965FAFF1
:10F47000E89787EDEC968FAFEC9703E21BE383E50B
:10F48000829DF001839DF00D1124EB5FF34FC1804D
:10F49000D280E380F4809601A701A4966FADA49773
:10F4A000A8967FADA897E0968FADE097AC969FADFC
:10F4B000AC970F948A2D181664F4A496CFAEA49737
:10F4C000A896DFAEA897E096EFAEE097AC96FFAEB9
:10F4D000AC97E8962FADE897EC963FADEC97A80176
:10F4E000A4966FADA497A8967FADA897E0968FAD30
:10F4F000E097AC969FADAC970F948A2D1816FCF44C
:10F50000E8969FADE897A4969FAFA497EC96AFAD11
:10F51000EC97A896AFAFA897E0960FAFE097AC96A0
:10F520001FAFAC970CC0A4961FAEA497A8961FAEB1
:10F53000A897E0961FAEE097AC961FAEAC9780E11F
:10F54000FE017196A0E8B1E101900D928A95E1F774
:10F5500083E5829D8001839D100D11240B5F134F65
:10F56000A4968FADA497A8969FADA897E096AFAD4F
:10F57000E097AC96BFADAC97F80181879287A387DF
:10F58000B487E7966CAD7DAD8EAD9FADE797905893
:10F590009B01AC010F942A2BD8011D962D913D9112
:10F5A0004D915C9150970F949A249B01AC016BE0B4
:10F5B00077ED83E29BE30F94292B2BE0C22E27EDFE
:10F5C000D22E23E2E22E2BE3F22EF801C582D68260
:10F5D000E782F086B080C180D280E380F480A7010A
:10F5E00096010F948A2D87FD02C083E001C081E05F
:10F5F0008B2993E5929DF001939DF00D1124EB5F13
:10F60000F34F808380E1FE01B196A1E3B6E1019062
:10F610000D928A95E1F7C0922D16D0922E16E092A7
:10F620002F16F092301680E1FE01EF5AFF4FA1E550
:10F63000B6E101900D928A95E1F780E1FE01EF5B62
:10F64000FF4FA1E4B6E101900D928A95E1F7909108
:10F650002B1680912C16981303C084E680932816ED
:10F66000C556DF4F8881CB59D0408F5F8F70809314
:10F670002B1680912B1690912A1681508F70891726
:10F6800009F4B3C0F0902B168FEF8F0D8F70A496F6
:10F690008FAFA497B0902A1680912B16B81609F454
:10F6A00073C0C12CD12CA496FFADA497FB1509F40F
:10F6B0006BC06F2E712C23E5269D8001279D100DB8
:10F6C00011240B5F134FD8018C9183FD3AC0E8964B
:10F6D0000FAFE897EC961FAFEC971996BC91A896E0
:10F6E000BFAFA897F801F285E096FFAFE097D80189
:10F6F0001B96BC91AC96BFAFAC97F801F485E4962D
:10F70000FFAFE497D80115962D903D904D905C90F9
:10F710001897A2019101A8966FADA897E0967FADCA
:10F72000E097AC968FADAC979F2F0F943424811146
:10F73000F4C1C114D10459F0F601808180FDEDC1FE
:10F7400006C0E896CFAEE897EC96DFAEEC97A496AD
:10F750008FADA49781508F70A4968FAFA49780919E
:10F760002A168B1107C0E896CFACE897EC96DFAC71
:10F77000EC9799CFA496FFADA497FB1529F081E0F3
:10F780008B0D8F70B82EEBCF20912A16A4962FAF39
:10F79000A497C12CD12C80912B16A4963FADA49791
:10F7A000831719F1832E912C43E5489D8001499DD3
:10F7B000100D11240B5F134FD8018C9183FD0AC0EB
:10F7C0005801C114D10439F0C6010F946B14811192
:10F7D00002C039C25601A4968FADA4978F5F8F7077
:10F7E000A4968FAFA4976501D6CF40912C16A4960E
:10F7F0004FAFA49750912B16A8965FAFA89723E51B
:10F80000A4968FADA497A8969FADA897891779F075
:10F81000892F81508F70289FF0011124EB5FF34FE7
:10F82000908193FF04C0A8968FAFA897E9CF812C51
:10F83000912CA12CB12CE0961FAEE097AC961FAE98
:10F84000AC97E4961FAEE497E8961FAEE897212C9C
:10F85000312C00E010E0A896AFADA897A496BFADFC
:10F86000A497AB1709F4D0C0E3E5EB9FC0011124C6
:10F870009C012B5F334F1901D9018C9183FD19C075
:10F8800015966D917D918D919C9118970F94D82D1F
:10F89000F62EE72ED82EC92E0115110509F49AC0AF
:10F8A000F801808180FD12C0D1018C9180FD0EC0D5
:10F8B00091C0E096FFACE097AC96EFACAC97E496C5
:10F8C000DFACE497E896CFACE89789C0F801808177
:10F8D00081608083C8010F946B14811177C0F80197
:10F8E00061817281838194810F94D82D2B013C0119
:10F8F0009B01AC0160E070E080E89FE30F94242C52
:10F900004B015C019B01AC016F2D7E2D8D2D9C2D3B
:10F910000F949A2469837A838B839C83E0962FAD1E
:10F92000E097AC963FADAC97E4964FADE497E89680
:10F930005FADE897C501B4010F949A24698B7A8B67
:10F940008B8B9C8BAE014F5F5F4FBE016F5E7F4F15
:10F95000C8010E943FC2D801D6968C918823B1F18C
:10F960002091010C3091020C4091030C5091040C39
:10F97000F801FD9660817181828193810F949A24B0
:10F98000209158113091591140915A1150915B11A9
:10F990000F949A244B015C019B01AC01C301B2019D
:10F9A0000F949A240F949D2CF80172AF61AFA501BA
:10F9B00094016F2D7E2D8D2D9C2D0F949A240F94E4
:10F9C0009D2CD801DC967C936E93DB97F8018081A7
:10F9D0008E7F80838F2C9E2CAD2CBC2C8101A49615
:10F9E0008FADA4978F5F8F70A4968FAFA497E0968A
:10F9F000FFAEE097AC96EFAEAC97E496DFAEE4973F
:10FA0000E896CFAEE89727CF2114310409F414C14A
:10FA1000D1018C9181608C93C8010F946B1481117A
:10FA20006BC0F10161817281838194810F94D82D23
:10FA30006B017C019B01AC0160E070E080E89FE31A
:10FA40000F94242C2B013C012DEC3CEC4CE45DE3A9
:10FA50000F949A2469837A838B839C839401A501F4
:10FA6000C301B2010F949A24698B7A8B8B8B9C8B88
:10FA7000AE014F5F5F4FBE016F5E7F4FC1010E94BD
:10FA80003FC2D101D6968C918823B1F12091010C0F
:10FA90003091020C4091030C5091040CF101FD9641
:10FAA00060817181828193810F949A2420915811F1
:10FAB0003091591140915A1150915B110F949A2431
:10FAC0004B015C019B01AC01C701B6010F949A2464
:10FAD0000F949D2CF10172AF61AF2DEC3CEC4CE426
:10FAE0005DE3C501B4010F949A240F949D2CD101BC
:10FAF000DC967C936E93DB97F10180818E7F80830F
:10FB00009BC080E022C1D0907C11E0907D11F090EC
:10FB10007E1110917F110C941C7123E5269DF0013C
:10FB2000279DF00D1124EB5FF34F808181FD4BC0C9
:10FB3000C114D10441F0D6011596CD90DD90ED9021
:10FB4000FC90189708C08BE0C82E87EDD82E83E272
:10FB5000E82E8BE3F82EB3E5B69DF001B79DF00DCE
:10FB60001124EB5FF34F81899289A389B489BC0189
:10FB7000CD0190589B01AC010F942A2BF8012585EB
:10FB80003685478550890F949A249B01AC01C701A3
:10FB9000B6010F94292BE62E872E982EA92E262FFC
:10FBA000372F482F592FA8966FADA897E0967FADB5
:10FBB000E097AC968FADAC97E4969FADE4970F9429
:10FBC000342487FF0CC0A896EFACA897E0968FACC2
:10FBD000E097AC969FACAC97E496AFACE4972E2D33
:10FBE000382D492D5A2DC201B1010F943424882398
:10FBF00009F4ADCDF3E5F69DC001F79D900D1124FC
:10FC00009C012B5F334F6901D9018C9181608C93EA
:10FC1000C8010F946B14882329F0F60180818E7F30
:10FC2000808395CD8E2D982DA92DBA2DF601858333
:10FC30009683A783B0878BCD80916F00826080937D
:10FC40006F0081E082C0D6018C9181FD58C0D60141
:10FC500015962D913D914D915C911897AB962CAFD7
:10FC60003DAF4EAF5FAFAB971501B5E02B0E311C2A
:10FC7000F8014580568067807084A3019201AB969D
:10FC80006CAD7DAD8EAD9FADAB970F94342487FFE7
:10FC900036C0F60181899289A389B489BC01CD015E
:10FCA00090589B01AC010F942A2BD6011D962D91E3
:10FCB0003D914D915C9150970F949A249B01AC011A
:10FCC000AB966CAD7DAD8EAD9FADAB970F94292BF0
:10FCD0006B017C019B01AC01C301B2010F948A2D21
:10FCE00018166CF4D8018C9181608C93C5010F9427
:10FCF0006B148823F1F0F80180818E7F808323E5E7
:10FD0000289DF001299DF00D1124EB5FF34F218513
:10FD100032854385548565817681878190850F94EE
:10FD20003424811158CDA4963FADA49730932A1660
:10FD300052CDD101CD92DD92ED92FC921397A49613
:10FD4000BFADA497B0932A16DACFC356DF4F0FB6D4
:10FD5000F894DEBF0FBECDBFDF91CF911F910F9101
:10FD6000FF90EF90DF90CF90BF90AF909F908F90DB
:10FD70007F906F905F904F903F902F900895CF921B
:10FD8000DF92EF92FF920F931F93CF93DF93CDB744
:10FD9000DEB764970FB6F894DEBF0FBECDBFC98A39
:10FDA000DA8AEB8AFC8AFC0180819181A281B3818D
:10FDB00089839A83AB83BC83FB0180819181A2817B
:10FDC000B3818D839E83AF83B887FA01808191814F
:10FDD000A281B38189879A87AB87BC87F90180812B
:10FDE0009181A281B3818D879E87AF87B88BAE0149
:10FDF000475F5F4FBE016B5F7F4FCE0101960E9450
:10FE000064C18091351190913611892B81F4CE0116
:10FE100041967C019E01235F3F4FAE01475F5F4FDC
:10FE2000BE016B5F7F4F40970E94AB6C01C080E0CA
:10FE300064960FB6F894DEBF0FBECDBFDF91CF91B1
:10FE40001F910F91FF90EF90DF90CF900895CF9387
:10FE5000DF93CDB7DEB760970FB6F894DEBF0FBE65
:10FE6000CDBFE7E7F2E080819181A281B3818983F0
:10FE70009A83AB83BC8384819581A681B7818D836E
:10FE80009E83AF83B88780859185A285B385898756
:10FE90009A87AB87BC8784859585A685B7858D872E
:10FEA0009E87AF87B88BAE01475F5F4FBE016B5F28
:10FEB0007F4FCE0101960E9464C19E01235F3F4F98
:10FEC000AE01475F5F4FBE016B5F7F4FCE01019672
:10FED0000E9489BF60960FB6F894DEBF0FBECDBFFB
:10FEE000DF91CF9108950F94860B6091B90B7091BB
:10FEF000BA0B8DEE92E10F946F0B8AEE92E10D94A6
:10FF00009D0A2F923F924F925F926F927F928F92B3
:10FF10009F92AF92BF92CF92DF92EF92FF920F9398
:10FF20001F93CF93DF93CDB7DEB7C154D1090FB67E
:10FF3000F894DEBF0FBECDBF2DB73EB73FA72EA7AB
:10FF40000E9497E881114FC461E086E50E94F0A607
:10FF50008D8B853018F081EE94E179C03D89332393
:10FF600021F081EC94E10F949D0A6AE080E50E9403
:10FF7000F0A6182F8CEF810F8F3218F08DE994E1E5
:10FF800066C060E085E40E941A8D811103C082E0A2
:10FF90008FA302C091E09FA36091770270917802D5
:10FFA0008091790290917A026D837E838F83988706
:10FFB000C0907B02D0907C02E0907D02F0907E02A7
:10FFC000C986DA86EB86FC862091C1133091C21374
:10FFD0004091C3135091C4130F942A2BAB01BC0161
:10FFE00088E50E943BC86D877E878F87988B29851F
:10FFF0003A854B855C856091C5137091C6138091DD
:020000021000EC
:10000000C7139091C8130F942A2BAB01BC0189E54B
:100010000E943BC8698B7A8B8B8B9C8BBE016F5E79
:100020007F4FCE010D960E94ACA5811103C085E8DB
:1000300094E10DC08CE40E94C48C082F882381F0C9
:100040000E94658C8E8B803128F082E594E10F94BC
:100050009D0AC9C3AE89A13021F4B2E0BE8B01C0B4
:100060001E8A60E083E50E941A8D8CAB882321F004
:10007000011102C0E7E0EE8BFD89F33020F088E348
:1000800094E10F949D0A2091B6182BAF80E00F9455
:1000900013080E9403DE812F90E09EAB8DABADB7BD
:1000A000BEB7E4E01E9FA019B10911240FB6F89461
:1000B000BEBF0FBEADBF2DB73EB72F5F3F4F3DA7B1
:1000C0002CA72D894FA1BE016F5E7F4FCE010D96EB
:1000D0000E9446E99B01AC010F941C2E8111ECC2D9
:1000E0000E94F1EE611571058105910511F00F94E3
:1000F000C51F33EF3F8B8FE4888F93EC998F37ECDC
:10010000232EA3EFAA8FBFE4BB8FE3ECEC8FF7E4C1
:10011000FD8F1EA233243394412C512C32014AA26C
:100120005BA26CA27DA22E89822F90E0DC01119748
:100130002296BFAFAEAF2297FEA1EF2FF0E0FF8F68
:10014000EE8F2DA93EA9E217F3070CF0CDC23E8930
:10015000332309F46EC10F94771F2AE030E040E0AA
:1001600050E00F94AC2A0F943B2420E030E040EAAA
:1001700050E40F948A2D18161CF001E010E002C024
:100180000FEF1FEF0F94771F28E631E040E050E0BB
:100190000F94AC2A0F943B244B015C010F94771F02
:1001A00028E230E040E050E00F94AC2A6B5F7F4FD4
:1001B0008F4F9F4F0F943B2468A779A78AA79BA7CF
:1001C0008D898430E1F448A559A56AA57BA58AE20A
:1001D00094E10F94510BB501A40182E294E10F94D4
:1001E000510B8CE194E10F949D0A0130110519F433
:1001F00083E40E94B95288E194E10F949D0A312C66
:10020000C801110FAA0BBB0B8FAB98AFA9AFBAAF48
:10021000832D90E02296AEADBFAD22978A179B0743
:100220000CF007C1BCA9BB2379F06FA978AD89ADEB
:100230009AAD0F943B249B01AC010F942A2B20E034
:1002400030E040E952E41AC00F94771F24E130E017
:1002500040E050E00F94AC2A675E7F4F8F4F9F4F76
:100260000F943B246B017C016FA978AD89AD9AADE9
:100270000F943B249B01AC01C701B6010F949A2453
:100280009B01AC01C501B4010F942A2B4B015C0109
:1002900020E030E044EB53E40F948A2D18164CF420
:1002A00020E030E044EB53E4C501B4010F94292B66
:1002B000EDCF20E030E0A901C501B4010F94342452
:1002C00087FF0BC020E030E044EB53E4C501B401EC
:1002D0000F942A2B4B015C01ECCF2BED3FE049E45E
:1002E00050E4C501B4010F949A2420E030E044E3C7
:1002F00053E40F94242C6B017C010F941F2C68ABEA
:1003000079AB8AAB9BAB2091C1133091C213409162
:10031000C3135091C4136D857E858F8598890F9482
:10032000292B6CAF7DAF8EAF9FAF28A939A94AA901
:100330005BA968A579A58AA59BA50F949A249B0122
:10034000AC016CAD7DAD8EAD9FAD0F942A2B6D834E
:100350007E838F839887C701B6010F94CA2D68AB3F
:1003600079AB8AAB9BAB2091C5133091C6134091FA
:10037000C7135091C81369897A898B899C890F9416
:10038000292B6B017C0128A939A94AA95BA968A579
:1003900079A58AA59BA50F949A249B01AC01C7015E
:1003A000B6010F942A2B69877A878B879C8748E64A
:1003B00051E060E070E0CE0105960F94A20F48E690
:1003C00051E060E070E0CE0109960F94A20FED8934
:1003D000E430F9F44D815E816F8178858CE094E1A1
:1003E0000F94510B49855A856B857C8589E094E192
:1003F0000F94510B40917F025091800260918102D5
:100400007091820286E094E10F94510B8AE00E9481
:10041000B95219821A821B821C82AE014F5F5F4F54
:10042000BE01675F7F4FCE0105960E94E3DE3394E5
:10043000EFCE20E04FA1BE016F5E7F4FCE010D9643
:100440000E9446E9D62EE72EF82E192FEE8DFF8D4D
:10045000EE0FFF1FEE0FFF1F2CA53DA5E20FF31FB0
:10046000862F9E2DAF2DB12F80839183A283B383DE
:10047000312C2D2D3E2D4F2D512F6D2D7E2D8F2D5D
:10048000912F0F941C2E811102C0332433942D2DF3
:100490003E2D4F2D512F6D2D7E2D8F2D912F0F9491
:1004A0001C2E811121C100E0412C512C3201ECA500
:1004B000FDA534E0039FE00DF11D11242081318161
:1004C00042815381C301B2010F942A2B2B013C01BD
:1004D0000F5F8EA1801758F78E8C9F8C9FEF891A23
:1004E000990A092C000CAA08BB08C501B4010F9495
:1004F0003B246E8F7F8F88A399A39B01AC01C3011E
:10050000B2010F94242C6AA37BA38CA39DA32A8DF4
:100510003B8D4C8D5D8D6D2D7E2D8F2D912F0F94EC
:10052000342487FF04C0DA8EEB8EFC8E1D8F2F895A
:10053000388D498D522D6D2D7E2D8F2D912F0F943D
:100540008A2D181624F4DF8AE88EF98E212EC12C0C
:10055000412C512C3201ECA5FDA5A4E0CA9EE00D72
:10056000F11D11242AA13BA14CA15DA160817181E3
:10057000828193810F94292B9B01AC010F949A24C3
:100580009B01AC01C301B2010F942A2B2B013C014A
:10059000C394BEA1BC15F8F62E8D3F8D48A159A17C
:1005A0000F94242C0F94D82D2B013C018D8982505F
:1005B0008E3708F07DC0C501B4010E942D536DA98E
:1005C0007EA981E094E10F94620B94E9A92E96E054
:1005D000B92EF50181915F01882319F00E94B9526B
:1005E000F8CF43E06D2D7E2D8F2D912F0E94495322
:1005F000FD89F23009F459C00AE916E0D8018D915D
:100600008D01882319F00E94B952F8CF44E06AA105
:100610007BA18CA19DA10E94495302EA16E0F8013A
:1006200081918F01882319F00E94B952F8CF46E0DA
:10063000C301B2010E9449530BEA16E0D8018D9123
:100640008D01882319F00E94B952F8CF43E06A8DDA
:100650007B8D8C8D9D8D0E94495302EB16E0F80135
:1006600081918F01882319F00E94B952F8CF43E09D
:100670006F89788D898D922D0E94495309EB16E080
:10068000D8018D918D01882319F00E94B952F8CFBD
:100690002A8D3B8D4C8D5D8D6F89788D898D922D46
:1006A0000F94292B43E00E9449538AE00E94B952DB
:1006B000BEA1BF5FBEA340CDE3EFEF8BFFE4F88F99
:1006C00023EC298F87EC282E33EF3A8F8FE48B8F22
:1006D00093EC9C8FA7E4AD8F312C412C512C32012F
:1006E0004AA25BA26CA27DA280E00E94FB9C332008
:1006F00009F46AC086EF93E10F949D0ABD89BB237C
:1007000009F44DC002EC16E0F80181918F018823B5
:1007100019F00E94B952F8CF46E06AA17BA18CA1E2
:100720009DA10E94495309EC16E0D8018D918D01DD
:10073000882319F00E94B952F8CF43E06A8D7B8D6F
:100740008C8D9D8D0E94495300ED16E0F80181913A
:100750008F01882319F00E94B952F8CF43E06F89C6
:10076000788D898D922D0E94495307ED16E0D801AE
:100770008D918D01882319F00E94B952F8CF2A8DEE
:100780003B8D4C8D5D8D6F89788D898D922D0F9469
:10079000292B43E00E9449538AE00E94B95200EE9F
:1007A00016E0F80181918F01882319F00E94B95257
:1007B000F8CF46E0C301B2010E9449538AE00E948B
:1007C000B9528AE00E94B9520E94EADD8BAD0F94C3
:1007D00013080E94B0DF2EA53FA50FB6F8943EBFC8
:1007E0000FBE2DBF07C08EA59FA50FB6F8949EBF64
:1007F0000FBE8DBFAEA5BFA50FB6F894BEBF0FBE8E
:10080000ADBFCF5BDF4F0FB6F894DEBF0FBECDBFDD
:10081000DF91CF911F910F91FF90EF90DF90CF90DC
:10082000BF90AF909F908F907F906F905F904F9010
:100830003F902F9008952F923F924F925F926F9228
:100840007F928F929F92AF92BF92CF92DF92EF9260
:10085000FF920F931F93CF93DF93CDB7DEB7E2974D
:100860000FB6F894DEBF0FBECDBF2091B6182F8B08
:1008700087E50E94C48C882309F4FAC080912D1466
:1008800090912E14892B29F40F94820B84EE93E11E
:1008900034C08AE50E940D8D882379F00E948D8CEA
:1008A0002091BD133091BE134091BF135091C013DE
:1008B0000F94292B6B017C0108C0C0907F02D0905F
:1008C0008002E0908102F090820220E030E040E27D
:1008D00051ECC701B6010F948A2D87FD0AC020E0B4
:1008E00030E040E251E4C701B6010F9434241816F9
:1008F0003CF40F94820B87ED93E10F949D0AC0C0E6
:1009000040E050E060EC7FE788E50E943BC8209122
:10091000B5133091B6134091B7135091B8130F949B
:10092000292B2B013C0140E050E060EC7FE789E59A
:100930000E943BC82091B9133091BA134091BB1368
:100940005091BC130F94292B4B015C016FEF89E48C
:100950000E94F0A6182F6FEF8AE40E94F0A6082FDD
:10096000A3019201C301B2010F941C2E811158C042
:10097000A5019401C501B4010F941C2E811150C032
:100980006091231470912414072E000C880B990B8E
:100990000F943B249B01AC01C301B2010F94292B9E
:1009A00020E030E0A9010F942A2B20E030E0A901DB
:1009B0000F94242C0F94962C162F6091251470916F
:1009C0002614072E000C880B990B0F943B249B01D7
:1009D000AC01C501B4010F94292B20E030E0A9013E
:1009E0000F942A2B20E030E0A9010F94242C0F94BF
:1009F000962C062F812F012E000C990B97FD04C019
:100A000005971CF014E001C010E0802F002E000CB0
:100A1000990B97FD04C005971CF004E001C000E0AD
:100A2000153070F5063060F580E00F94130835E05E
:100A30001302F0011124E00FF11D07FDFA95EE0FEE
:100A4000FF1FEE0FFF1FE75CFB4EC082D182E282E8
:100A5000F382A7019601602F812F0E940DC78F8915
:100A60000F9413086F89662359F00E94B0DF08C005
:100A70008AE40E94C48C182F882321F00E94C0921F
:100A800010E0CBC460E070E086E50E94E1A69A8F9A
:100A9000898F059718F08FEA93E195C260E084E4AE
:100AA0000E941A8D8B8F40E050E0BA018AE50E94C7
:100AB0003BC86AA77BA78CA79DA740E050E86BEBDB
:100AC00075E483E50E943BC820E030E040E752E453
:100AD0000F94242C609361027093620280936302EE
:100AE0009093640288E40E94C48C882309F4FCC0BB
:100AF0000E948D8C0F94962C6B017C014B012090F1
:100B0000C1133090C2134090C3135090C41320E01F
:100B100030E0A901C201B1010F942A2B762EA72E35
:100B2000B82E092F20E030E040E450E40F94342444
:100B300087FF05C0712CA12CF0E4BF2E00E4B601A4
:100B400097FE02C06F5F7F4F7595679571956195B0
:100B500071096C547F4F072E000C880B990B0F9472
:100B60003B244B01682E988F272D3A2D4B2D502F6B
:100B70000F948A2D181624F4782CA92CB62C088DE5
:100B8000672D7A2D8B2D902F0F94962C6B8B7C8B51
:100B90008D8B9E8B8B899C899A8B898B20E030E092
:100BA00044EB53E4C201B1010F942A2B762EA72EF9
:100BB000B82E092F20E030E842EB53E40F948A2D41
:100BC000181634F4712C50E8A52E62EBB62E03E40F
:100BD0006B897C896C0D7D1D072E000C880B990B91
:100BE0000F943B241B012C01272D3A2D4B2D502F08
:100BF0000F94342487FF04C0722CA32CB42C052D31
:100C0000672D7A2D8B2D902F0F94962C7C8B6B8BD0
:100C10002090C5133090C6134090C7135090C8134E
:100C200020E030E0A901C201B1010F942A2B762EF9
:100C3000A72EB82E092F20E030E040E450E40F94B6
:100C4000342487FF05C0712CA12C40E4B42E00E4AD
:100C5000272D3A2D4B2D502FB401862D988D0F94B2
:100C60008A2D181624F4782CA92CB62C088D672D03
:100C70007A2D8B2D902F0F94962C3B014C015B010C
:100C800020E030E044EB53E4C201B1010F942A2B81
:100C9000362E472E582E092F20E030E842EB53E441
:100CA0000F948A2D181634F4312C20E8422E32EBA2
:100CB000532E03E4C60CD71CB601DD0C880B990B30
:100CC0000F943B246B017C01232D342D452D502F97
:100CD0000F94342487FF04C03C2C4D2C5E2C0F2D28
:100CE000632D742D852D21C18CE40E940D8D8823E8
:100CF00069F00E948D8C2091B5133091B61340910C
:100D0000B7135091B8130F94292B2BC020E030E07B
:100D1000A9016091C1137091C2138091C313909186
:100D2000C4130F942A2B6B017C0120E030E040E4D7
:100D300050E40F94342487FD0DC020E030E0A90179
:100D4000C701B6010F94342487FF09C0C12CD12CF0
:100D5000760105C0C12CD12C90E4E92EFE2CC701F0
:100D6000B6010F94962C7A8B698B82E50E940D8DCB
:100D7000882369F00E948D8C2091B5133091B613B1
:100D80004091B7135091B8130F94292B3DC020E028
:100D900030E044EB53E46091C1137091C213809131
:100DA000C3139091C4130F942A2BD62EE72EF82E3E
:100DB000092F20E030E842EB53E40F948A2D1816F7
:100DC00034F4D12C00E8E02E82EBF82E03E469899C
:100DD0007A8968597E4F072E000C880B990B0F9467
:100DE0003B24962EA72EB82EC92E2D2D3E2D4F2DED
:100DF000502F0F94342487FF03C0D92C75010C2D7C
:100E00006D2D7E2D8F2D902F0F94962C7C8B6B8BC0
:100E100086E40E940D8D882369F00E948D8C2091BC
:100E2000B9133091BA134091BB135091BC130F9476
:100E3000292B2BC020E030E0A9016091C5137091EF
:100E4000C6138091C7139091C8130F942A2B6B017E
:100E50007C0120E030E040E450E40F94342487FD2E
:100E60000DC020E030E0A901C701B6010F94342481
:100E700087FF09C0C12CD12C760105C0C12CD12C13
:100E8000B0E4EB2EFE2CC701B6010F94962C5B014B
:100E900082E40E940D8D882369F00E948D8C209140
:100EA000B9133091BA134091BB135091BC130F94F6
:100EB000292B3CC020E030E044EB53E46091C513A3
:100EC0007091C6138091C7139091C8130F942A2B69
:100ED000D62EE72EF82E092F20E030E842EB53E41F
:100EE0000F948A2D181634F4D12CF0E8EF2EA2EBD3
:100EF000FA2E03E4B50168597E4F072E000C880BCB
:100F0000990B0F943B24762E872E982EC92E2D2DCB
:100F10003E2D4F2D502F0F94342487FF03C0D72C24
:100F200074010C2D6D2D7E2D8F2D902F0F94962CEE
:100F30007B01B5010B2C000C880B990B0F943B2403
:100F40006D8F7E8F8F8F98A369837A838B839C8329
:100F5000A989BA89BD01BB0F880B990B0F943B245B
:100F600069A37AA38BA39CA36D837E838F839887C9
:100F7000BE016F5F7F4FCE0105960E94ACA588230E
:100F800001F1B7010F2C000C880B990B0F943B2437
:100F900069877A878B879C872B893C89B901330FB6
:100FA000880B990B0F943B246D877E878F87988BD6
:100FB000BE01675F7F4FCE010D960E94ACA58130C8
:100FC00029F083E993E10F949D0A27C2898D9A8DB8
:100FD000892B71F08DE793E10F949D0A9B8D9923E6
:100FE00021F083E793E10F949D0A8AE00E94B952B1
:100FF0000E941CBF80E00F94130881E00E94FB9CBC
:10100000882321F08F890F9413083ACD0B891C890E
:10101000A989BA890A1B1B0B17FF02C00D5F1F4F5E
:101020001595079515950795B801012E000C880BAD
:10103000990B0F943B246DA37EA38FA398A7EA1866
:10104000FB08F7FE03C0B3E0EB0EF11C47019594DB
:10105000879495948794B401092C000C880B990B04
:101060000F943B246B017C010E9403DE60912D14E0
:1010700070912E14072E000C880B990B0F943B24B3
:101080009B01AC016DA17EA18FA198A50F94342482
:10109000811122C060912F1470913014072E000C22
:1010A000880B990B0F943B249B01AC01C701B6013F
:1010B0000F943424811110C0809123149091241432
:1010C00029893A892817390739F480912514909194
:1010D0002614A816B906A9F00E94C09210932E14E7
:1010E00000932D149092301480922F1489899A893C
:1010F0009093241480932314B0922614A092251464
:101100001F8A60E085E40E941A8D882319F091E01F
:1011100099A702C0A2E0A9A7B1E0BC8F212C312C75
:10112000812C912C540121E0298B31E0388F65E02E
:101130006B8B10E02EA6298931E02327298B0C8D9B
:10114000C101032C000CAA0BBB0B8FA798ABA9AB5A
:10115000BAAB9B89911709F4BEC0612F012E000C18
:10116000770B880B990B0F943B242DA13EA14FA127
:1011700058A50F949A2429A13AA14BA15CA10F94E0
:101180002A2B2B013C016FA578A989A99AA90F9454
:101190003B24A70196010F949A242D8D3E8D4F8DEF
:1011A00058A10F942A2B4B015C0120E030E0A901EB
:1011B000C301B2010F94342487FF04C020E030E063
:1011C000A90104C020E030E040E05FE3C301B201C8
:1011D0000F942A2B0F94CC2C69837A838B839C8366
:1011E00020E030E0A901C501B4010F94342487FF49
:1011F00004C020E030E0A90104C020E030E040E07D
:101200005FE3C501B4010F942A2B0F94CC2C6D839E
:101210007E838F839887A98DBA8DAB2B81F0602F49
:1012200070E08FE593E10F94620B69E170E08DE56A
:1012300093E10F94620B8AE593E10F949D0A1F924C
:10124000B9E1BF931F920F9326E433E13F932F93AD
:101250001F920E947DE8298D49A5BE016B5F7F4FDB
:10126000CE0101960E9446E94B015C010FB6F8944D
:10127000DEBF0FBECDBF9B01AC010F941C2E882397
:1012800021F08F890F94130833C0A50194016AA53A
:101290007BA58CA59DA50F942A2B9B01AC0165E035
:1012A0001603F0011124E20DF31DEE0FFF1FEE0FE8
:1012B000FF1FE75CFB4E20833183428353836EA57F
:1012C000812F0E940DC780E00E94E5530F5F888D3B
:1012D000180F1F8A3ECF94E02916310449F0A5016A
:1012E0009401C501B4010F941C2E882309F480C019
:1012F0000E94CDF580E00E94FB9C882351F08F89ED
:101300000F941308812C912C90ECA92E9FE7B92EF5
:1013100054C0A5019401C501B4010F941C2E811184
:101320004CC0AB8DAA2309F10F94AC0A0F94590855
:10133000BB8DB1113FC087E792E00F94FA059B0186
:10134000AC0160917F027091800280918102909146
:1013500082020F94292B60937F0270938002809306
:1013600081029093820281E026C012E084E0F82E90
:1013700002E0EF2CE11ADF2CD01A21E041E0602FCF
:10138000812F0F94C60821E04FEF602F8E2D0F9410
:10139000C6082FEF41E06D2D812F0F94C6082FEF67
:1013A0004FEF6D2D8E2D0F94C608015020F7115070
:1013B000F8F6BACF8F898093B6180E94EADD809143
:1013C000B61881110E94AEDF0E94B39C0E941CBF20
:1013D0008AE393E10E9480BB0E94B0DF11E0A50187
:1013E0009401C501B4010F941C2E811116C048CB85
:1013F0002989222361F081E0888F95E09B8B10E0A2
:10140000AFEF2A1A3A0ABC8DBB5FBC8F93CE3FEF79
:10141000388F6FEF6B8B14E0F3CF812FE2960FB60E
:10142000F894DEBF0FBECDBFDF91CF911F910F911A
:10143000FF90EF90DF90CF90BF90AF909F908F90F4
:101440007F906F905F904F903F902F900895809184
:10145000371183FD0FC08091E90B81110BC02091E2
:10146000F20B3091F30B8091190290911A02281718
:10147000390724F061E080E00C94FBD10F94860BD7
:101480008EE397E10F949D0A80E00895CF92DF925A
:10149000EF92FF920F931F93CF93DF937C018B0109
:1014A000109281090E944F50C7E7D2E020911502A7
:1014B000309116024091170250911802F701608195
:1014C0007181828193810F94242C2C853D854E85DA
:1014D0005F850F942A2B6C877D878E879F87C12C11
:1014E000D12C760123E832E04FE752E06BE772E05F
:1014F000CE010E94BF7EDF91CF911F910F91FF908F
:10150000EF90DF90CF900C941CBFCF92DF92EF92C0
:10151000FF92C0906502D0906602E0906702F09062
:101520006802FC0180819181A281B3818093650270
:1015300090936602A0936702B09368020E941FDB3B
:10154000C0926502D0926602E0926702F092680251
:10155000FF90EF90DF90CF9008952F923F924F929F
:101560005F926F927F928F929F92AF92BF92CF9233
:10157000DF92EF92FF920F931F93CF93DF93CDB73C
:10158000DEB76F970FB6F894DEBF0FBECDBF9C8F4E
:101590008B8F7E8F6D8F212C312C2FEF28873FEF83
:1015A0003F834FEF488B5FE4598B83EC8A8B97E442
:1015B0009B8B21E030E040E050E0022C04C0220F81
:1015C000331F441F551F0A94D2F72F8B388F498F32
:1015D0005A8F4AEF51E15B874A8700E010E02F8E77
:1015E000AA85BB858D919D91BB87AA87A0E0B0E0BD
:1015F0002F89388D498D5A8D82239323A423B523B7
:10160000892B8A2B8B2B09F0ECC080912D149091A3
:101610002E14289EB001299E700D389E700D112445
:101620008091231490912414680F791F072E000CC9
:10163000880B990B0F943B246C877D878E879F873F
:1016400080912F1490913014089FB001099F700D64
:10165000189F700D11248091251490912614680F05
:10166000791F072E000C880B990B0F943B246B01FC
:101670007C012C853D854E855F85AB8DBC8D6D9144
:101680007D918D919C910F94292B2B013C01A701F9
:101690009601ED8DFE8D60817181828193810F9421
:1016A000292B4B015C01A3019201C301B2010F94EC
:1016B0009A242B013C01A5019401C501B4010F94AA
:1016C0009A249B01AC01C301B2010F942A2B0F9401
:1016D000D82D4B015C012C853D854E855F85609141
:1016E0001E1270911F1280912012909121120F945E
:1016F000292B2B013C01A701960160911A127091D0
:101700001B1280911C1290911D120F94292B6B01BA
:101710007C01A3019201C301B2010F949A242B0111
:101720003C01A7019601C701B6010F949A249B01C1
:10173000AC01C301B2010F942A2B0F94D82D20E0E5
:1017400030E040E751E40F94242CA50194010F945C
:101750002A2B6B017C018090221290902312A09082
:101760002412B090251220E030E040E85FE3C5018C
:10177000B4010F948A2D1816FCF4C501B4010F941E
:10178000962C4B015C0116161706180619063CF438
:101790000F94771FA50194010F94AC2A03C060E059
:1017A00070E0CB010F943B249B01AC01B601C70153
:1017B0000F942A2B6B017C01288939894A895B891E
:1017C000B601C7010F94342487FF0BC0FF8DF88743
:1017D0000F83C986DC8AED8AFE8AC88AD98AEA8A9A
:1017E000FB8A0F5F1F4F0530110509F0F9CE2FEF6F
:1017F000221A320A35E02316310409F0DACE4F817D
:10180000E42FF0E0EE0FFF1FE650FE4E81E090E087
:10181000088402C0880F991F0A94E2F72081318161
:10182000822B932B9183808389859C89AD89BE8986
:101830008B839C83AD83BE83482F5C816D817E81C9
:1018400028853F8180E090E06F960FB6F894DEBF68
:101850000FBECDBFDF91CF911F910F91FF90EF9001
:10186000DF90CF90BF90AF909F908F907F906F90C0
:101870005F904F903F902F9008958C3891051CF009
:101880002CE880E002C0282F892F20938B098093B9
:101890008C090C944ED780E1E7E7F2E0A5EAB3E1CA
:1018A00001900D928A95E1F708958091F811909139
:1018B000F911009731F04AE050E060E070E00D94DB
:1018C0002A2160E070E0CB0108950E94558C97FDBD
:1018D0000CC00E94558C6F3F71058105910509F080
:1018E00034F40E94558C862F089580E008958FEF80
:1018F00008958091F8119091F911892B39F00E9487
:10190000658C91E0811103C090E001C091E0892FC6
:1019100008950E94558CCB0108950F931F93CF9388
:101920008091F8119091F911009711F1FC018F014C
:10193000C1912C2F2F7DA9F0C53411F0C536B9F710
:10194000F801108260E070E08091F8119091F91137
:101950000F94CE1FF801C083562F472F382F292F01
:101960000BC060E070E0CF911F910F910D94CE1FDE
:1019700050E040E030E020E0652F742F832F922F5D
:10198000CF911F910F91089581548A3108F042C080
:10199000E82FF0E040918A1250918B1260918C12E6
:1019A00070918D1204C076956795579547958A95E5
:1019B000D2F7842F817040FF2FC0E059FD4E9081F7
:1019C000992309F1E091B90BF091BA0BE90FF11DE0
:1019D000908120ED290F2A3098F09E3211F49181E8
:1019E0000CC09D3211F09B3271F4918120ED290FD2
:1019F0002A3030F09E3239F4928190539A3018F4A4
:101A00002E2F9F2F02C020E090E02093F81190939A
:101A1000F911089580E0089508950E94C48C8823E8
:101A200041F081E02091F8113091F911232B09F454
:101A300080E00895CF93DF93C82FD62F0E940D8D9D
:101A4000882321F0DF91CF910C94798C8C2F0E9408
:101A5000C48C811101C08D2FDF91CF9108950F9318
:101A60001F93CF938C01C62F8DE795E10F949D0AAC
:101A7000C8010F949D0ACC2331F08AE0CF911F91C9
:101A80000F910C94B952CF911F910F91089560E07E
:101A900082E995E10E942F8D8AE995E10F949D0AD4
:101AA0008AE00C94B95260E082E995E10E942F8DA2
:101AB0008EE895E10F949D0A8AE00C94B952EF925A
:101AC000FF920F931F93CF937C018B01C42F60E093
:101AD00082E995E10E942F8DC7010F949D0A80E253
:101AE0000E94B952C8010F949D0ACC2341F08AE0AC
:101AF000CF911F910F91FF90EF900C94B952CF911D
:101B00001F910F91FF90EF90089541E0BC0187E88D
:101B100095E10C945F8DCF93DF93C091911110925A
:101B20009111C230B9F118F4C13041F041C0C43054
:101B3000B1F1C530E9F5C5ECD5E13FC081111DC05B
:101B40000E94538D41E060E376E187E597E10E94D2
:101B50005F8D85E296E10E94858D809181098823C1
:101B600019F087E196E104C0C09391118EE096E1EF
:101B70000E94858D0E94478D1EC08130E1F48091C6
:101B800081098823C1F010921B02109281090E94E2
:101B90004F5011C010921414C1EED5E10EC08AE06E
:101BA00096E19093C0098093BF09C0EDD5E105C0CF
:101BB000C7EBD5E102C0CAEFD5E18FE995E10F94FB
:101BC0009D0ACE010F949D0A8AE0DF91CF910C947B
:101BD000B9520F931F93CF93DF938B01EA01809348
:101BE00091110E94538D41E0B80187E597E10E9471
:101BF0005F8D209719F0CE010E94858DDF91CF91E6
:101C00001F910F910C94478D0F931F93CF93DF93E8
